:020000040000FA
:10000000FFFF0401AA287201FFFF0401AA28720160
:10001000FFFF0401AA287201FFFF0401AA28720150
:10002000FFFF0401FE00FF01FFFF0401BBF210010E
:10003000FFFF0401BBF21901FFFF0401BBF2100135
:10004000FFFF04010A287201FFFF04010A28720160
:10005000FFFF04010A287201FFFF04010A28720150
:10006000FFFF04010A287201FFFF04010A28720140
:10007000FFFF04010A287201FFFF04010A28720130
:10008000FFFF0401AA287201FFFF0401AA287201E0
:10009000FFFF0401AA287201FFFF0401AA287201D0
:1000A000FFFF0401FE00FF01FFFF0401BBF210018E
:1000B000FFFF0401BBF21901FFFF0401BBF21001B5
:1000C000FFFF04010A287201FFFF04010A287201E0
:1000D000FFFF04010A287201FFFF04010A287201D0
:1000E000FFFF04010A287201FFFF04010A287201C0
:1000F000FFFF04010A287201FFFF04010A287201B0
:10010000FFFF0401AA287201FFFF0401AA2872015F
:10011000FFFF0401AA287201FFFF0401AA2872014F
:10012000FFFF040167142301FFFF0401BBF210016C
:10013000FFFF0401BBF21901FFFF0401BBF2100134
:10014000FFFF04010A287201FFFF04010A2872015F
:10015000FFFF04010A287201FFFF04010A2872014F
:10016000FFFF04010A287201FFFF04010A2872013F
:10017000FFFF04010A287201FFFF04010A2872012F
:10018000FFFF0401AA287201FFFF0401AA287201DF
:10019000FFFF0401AA287201FFFF0401AA287201CF
:1001A000FFFF0401FFFFF901FFFF0401BBF2100193
:1001B000FFFF0401BBF21901FFFF0401BBF21001B4
:1001C000FFFF04010A287201FFFF04010A287201DF
:1001D000FFFF04010A287201FFFF04010A287201CF
:1001E000FFFF04010A287201FFFF04010A287201BF
:1001F000FFFF04010A287201FFFF04010A287201AF
:10020000FFFF0401AA287201FFFF0401AA2872015E
:10021000FFFF0401AA287201FFFF0401AA2872014E
:10022000FFFF0401FE00FF01FFFF0401BBF210010C
:10023000FFFF0401BBF21901FFFF0401BBF2100133
:10024000FFFF04010A287201FFFF04010A2872015E
:10025000FFFF04010A287201FFFF04010A2872014E
:10026000FFFF04010A287201FFFF04010A2872013E
:10027000FFFF04010A287201FFFF04010A2872012E
:10028000FFFF0401AA287201FFFF0401AA287201DE
:10029000FFFF0401AA287201FFFF0401AA287201CE
:1002A000FFFF0401FE00FF01FFFF0401BBF210018C
:1002B000FFFF0401BBF21901FFFF0401BBF21001B3
:1002C000FFFF04010A287201FFFF04010A287201DE
:1002D000FFFF04010A287201FFFF04010A287201CE
:1002E000FFFF04010A287201FFFF04010A287201BE
:1002F000FFFF04010A287201FFFF04010A287201AE
:10030000FFFF0401AA287201FFFF0401AA2872015D
:10031000FFFF0401AA287201FFFF0401AA2872014D
:10032000FFFF04016A111E01FFFF0401BBF210016F
:10033000FFFF0401BBF21901FFFF0401BBF2100132
:10034000FFFF04010A287201FFFF04010A2872015D
:10035000FFFF04010A287201FFFF04010A2872014D
:10036000FFFF04010A287201FFFF04010A2872013D
:10037000FFFF04010A287201FFFF04010A2872012D
:10038000FFFF0401AA287201FFFF0401AA287201DD
:10039000FFFF0401AA287201FFFF0401AA287201CD
:1003A000FFFF04016A111E01FFFF0401BBF21001EF
:1003B000FFFF0401BBF21901FFFF0401BBF21001B2
:1003C000FFFF04010A287201FFFF04010A287201DD
:1003D000FFFF04010A287201FFFF04010A287201CD
:1003E000FFFF04010A287201FFFF04010A287201BD
:1003F000FFFF04010A287201FFFF04010A287201AD
:10040000FFFF0401AA287201FFFF0401AA2872015C
:10041000FFFF0401AA287201FFFF0401AA2872014C
:10042000FFFF0401FE00FF01FFFF0401BBF210010A
:10043000FFFF0401BBF21901FFFF0401BBF2100131
:10044000FFFF04010A287201FFFF04010A2872015C
:10045000FFFF04010A287201FFFF04010A2872014C
:10046000FFFF04010A287201FFFF04010A2872013C
:10047000FFFF04010A287201FFFF04010A2872012C
:10048000FFFF0401AA287201FFFF0401AA287201DC
:10049000FFFF0401AA287201FFFF0401AA287201CC
:1004A000FFFF0401FE00FF01FFFF0401BBF210018A
:1004B000FFFF0401BBF21901FFFF0401BBF21001B1
:1004C000FFFF04010A287201FFFF04010A287201DC
:1004D000FFFF04010A287201FFFF04010A287201CC
:1004E000FFFF04010A287201FFFF04010A287201BC
:1004F000FFFF04010A287201FFFF04010A287201AC
:10050000FFFF0401AA287201FFFF0401AA2872015B
:10051000FFFF0401AA287201FFFF0401AA2872014B
:10052000FFFF04012B282001FFFF0401BBF2100193
:10053000FFFF0401BBF21901FFFF0401BBF2100130
:10054000FFFF04010A287201FFFF04010A2872015B
:10055000FFFF04010A287201FFFF04010A2872014B
:10056000FFFF04010A287201FFFF04010A2872013B
:10057000FFFF04010A287201FFFF04010A2872012B
:10058000FFFF0401AA287201FFFF0401AA287201DB
:10059000FFFF0401AA287201FFFF0401AA287201CB
:1005A000FFFF04012B282001FFFF0401BBF2100113
:1005B000FFFF0401BBF21901FFFF0401BBF21001B0
:1005C000FFFF04010A287201FFFF04010A287201DB
:1005D000FFFF04010A287201FFFF04010A287201CB
:1005E000FFFF04010A287201FFFF04010A287201BB
:1005F000FFFF04010A287201FFFF04010A287201AB
:10060000FFFF0401AA287201FFFF0401AA2872015A
:10061000FFFF0401AA287201FFFF0401AA2872014A
:10062000FFFF0401FE00FF01FFFF0401BBF2100108
:10063000FFFF0401BBF21901FFFF0401BBF210012F
:10064000FFFF04010A287201FFFF04010A2872015A
:10065000FFFF04010A287201FFFF04010A2872014A
:10066000FFFF04010A287201FFFF04010A2872013A
:10067000FFFF04010A287201FFFF04010A2872012A
:10068000FFFF0401AA287201FFFF0401AA287201DA
:10069000FFFF0401AA287201FFFF0401AA287201CA
:1006A000FFFF0401FE00FF01FFFF0401BBF2100188
:1006B000FFFF0401BBF21901FFFF0401BBF21001AF
:1006C000FFFF04010A287201FFFF04010A287201DA
:1006D000FFFF04010A287201FFFF04010A287201CA
:1006E000FFFF04010A287201FFFF04010A287201BA
:1006F000FFFF04010A287201FFFF04010A287201AA
:10070000FFFF0401AA287201FFFF0401AA28720159
:10071000FFFF0401AA287201FFFF0401AA28720149
:10072000FFFF04016A111E01FFFF0401BBF210016B
:10073000FFFF0401BBF21901FFFF0401BBF210012E
:10074000FFFF04010A287201FFFF04010A28720159
:10075000FFFF04010A287201FFFF04010A28720149
:10076000FFFF04010A287201FFFF04010A28720139
:10077000FFFF04010A287201FFFF04010A28720129
:10078000FFFF0401AA287201FFFF0401AA287201D9
:10079000FFFF0401AA287201FFFF0401AA287201C9
:1007A000FFFF04016A111E01FFFF0401BBF21001EB
:1007B000FFFF0401BBF21901FFFF0401BBF21001AE
:1007C000FFFF04010A287201FFFF04010A287201D9
:1007D000FFFF04010A287201FFFF04010A287201C9
:1007E000FFFF04010A287201FFFF04010A287201B9
:1007F000FFFF04010A287201FFFF04010A287201A9
:10080000FFFF0401AA287201FFFF0401AA28720158
:10081000FFFF0401AA287201FFFF0401AA28720148
:10082000FFFF0401FE00FF01FFFF0401BBF2100106
:10083000FFFF0401BBF21901FFFF0401BBF210012D
:10084000FFFF04010A287201FFFF04010A28720158
:10085000FFFF04010A287201FFFF04010A28720148
:10086000FFFF04010A287201FFFF04010A28720138
:10087000FFFF04010A287201FFFF04010A28720128
:10088000FFFF0401AA287201FFFF0401AA287201D8
:10089000FFFF0401AA287201FFFF0401AA287201C8
:1008A000FFFF0401FE00FF01FFFF0401BBF2100186
:1008B000FFFF0401BBF21901FFFF0401BBF21001AD
:1008C000FFFF04010A287201FFFF04010A287201D8
:1008D000FFFF04010A287201FFFF04010A287201C8
:1008E000FFFF04010A287201FFFF04010A287201B8
:1008F000FFFF04010A287201FFFF04010A287201A8
:10090000FFFF0401AA287201FFFF0401AA28720157
:10091000FFFF0401AA287201FFFF0401AA28720147
:10092000FFFF04012B242001FFFF0401BBF2100193
:10093000FFFF0401BBF21901FFFF0401BBF210012C
:10094000FFFF04010A287201FFFF04010A28720157
:10095000FFFF04010A287201FFFF04010A28720147
:10096000FFFF04010A287201FFFF04010A28720137
:10097000FFFF04010A287201FFFF04010A28720127
:10098000FFFF0401AA287201FFFF0401AA287201D7
:10099000FFFF0401AA287201FFFF0401AA287201C7
:1009A000FFFF04012B242001FFFF0401BBF2100113
:1009B000FFFF0401BBF21901FFFF0401BBF21001AC
:1009C000FFFF04010A287201FFFF04010A287201D7
:1009D000FFFF04010A287201FFFF04010A287201C7
:1009E000FFFF04010A287201FFFF04010A287201B7
:1009F000FFFF04010A287201FFFF04010A287201A7
:100A0000FFFF0401AA287201FFFF0401AA28720156
:100A1000FFFF0401AA287201FFFF0401AA28720146
:100A2000FFFF0401FE00FF01FFFF0401BBF2100104
:100A3000FFFF0401BBF21901FFFF0401BBF210012B
:100A4000FFFF04010A287201FFFF04010A28720156
:100A5000FFFF04010A287201FFFF04010A28720146
:100A6000FFFF04010A287201FFFF04010A28720136
:100A7000FFFF04010A287201FFFF04010A28720126
:100A8000FFFF0401AA287201FFFF0401AA287201D6
:100A9000FFFF0401AA287201FFFF0401AA287201C6
:100AA000FFFF0401FE00FF01FFFF0401BBF2100184
:100AB000FFFF0401BBF21901FFFF0401BBF21001AB
:100AC000FFFF04010A287201FFFF04010A287201D6
:100AD000FFFF04010A287201FFFF04010A287201C6
:100AE000FFFF04010A287201FFFF04010A287201B6
:100AF000FFFF04010A287201FFFF04010A287201A6
:100B0000FFFF0401AA287201FFFF0401AA28720155
:100B1000FFFF0401AA287201FFFF0401AA28720145
:100B2000FFFF04016A111E01FFFF0401BBF2100167
:100B3000FFFF0401BBF21901FFFF0401BBF210012A
:100B4000FFFF04010A287201FFFF04010A28720155
:100B5000FFFF04010A287201FFFF04010A28720145
:100B6000FFFF04010A287201FFFF04010A28720135
:100B7000FFFF04010A287201FFFF04010A28720125
:100B8000FFFF0401AA287201FFFF0401AA287201D5
:100B9000FFFF0401AA287201FFFF0401AA287201C5
:100BA000FFFF04016A111E01FFFF0401BBF21001E7
:100BB000FFFF0401BBF21901FFFF0401BBF21001AA
:100BC000FFFF04010A287201FFFF04010A287201D5
:100BD000FFFF04010A287201FFFF04010A287201C5
:100BE000FFFF04010A287201FFFF04010A287201B5
:100BF000FFFF04010A287201FFFF04010A287201A5
:100C0000FFFF0401AA287201FFFF0401AA28720154
:100C1000FFFF0401AA287201FFFF0401AA28720144
:100C2000FFFF0401FE00FF01FFFF0401BBF2100102
:100C3000FFFF0401BBF21901FFFF0401BBF2100129
:100C4000FFFF04010A287201FFFF04010A28720154
:100C5000FFFF04010A287201FFFF04010A28720144
:100C6000FFFF04010A287201FFFF04010A28720134
:100C7000FFFF04010A287201FFFF04010A28720124
:100C8000FFFF0401AA287201FFFF0401AA287201D4
:100C9000FFFF0401AA287201FFFF0401AA287201C4
:100CA000FFFF0401FE00FF01FFFF0401BBF2100182
:100CB000FFFF0401BBF21901FFFF0401BBF21001A9
:100CC000FFFF04010A287201FFFF04010A287201D4
:100CD000FFFF04010A287201FFFF04010A287201C4
:100CE000FFFF04010A287201FFFF04010A287201B4
:100CF000FFFF04010A287201FFFF04010A287201A4
:100D0000FFFF0401AA287201FFFF0401AA28720153
:100D1000FFFF0401AA287201FFFF0401AA28720143
:100D2000FFFF04012B282001FFFF0401BBF210018B
:100D3000FFFF0401BBF21901FFFF0401BBF2100128
:100D4000FFFF04010A287201FFFF04010A28720153
:100D5000FFFF04010A287201FFFF04010A28720143
:100D6000FFFF04010A287201FFFF04010A28720133
:100D7000FFFF04010A287201FFFF04010A28720123
:100D8000FFFF0401AA287201FFFF0401AA287201D3
:100D9000FFFF0401AA287201FFFF0401AA287201C3
:100DA000FFFF04012B282001FFFF0401BBF210010B
:100DB000FFFF0401BBF21901FFFF0401BBF21001A8
:100DC000FFFF04010A287201FFFF04010A287201D3
:100DD000FFFF04010A287201FFFF04010A287201C3
:100DE000FFFF04010A287201FFFF04010A287201B3
:100DF000FFFF04010A287201FFFF04010A287201A3
:100E0000FFFF0401AA287201FFFF0401AA28720152
:100E1000FFFF0401AA287201FFFF0401AA28720142
:100E2000FFFF0401FE00FF01FFFF0401BBF2100100
:100E3000FFFF0401BBF21901FFFF0401BBF2100127
:100E4000FFFF04010A287201FFFF04010A28720152
:100E5000FFFF04010A287201FFFF04010A28720142
:100E6000FFFF04010A287201FFFF04010A28720132
:100E7000FFFF04010A287201FFFF04010A28720122
:100E8000FFFF0401AA287201FFFF0401AA287201D2
:100E9000FFFF0401AA287201FFFF0401AA287201C2
:100EA000FFFF0401FE00FF01FFFF0401BBF2100180
:100EB000FFFF0401BBF21901FFFF0401BBF21001A7
:100EC000FFFF04010A287201FFFF04010A287201D2
:100ED000FFFF04010A287201FFFF04010A287201C2
:100EE000FFFF04010A287201FFFF04010A287201B2
:100EF000FFFF04010A287201FFFF04010A287201A2
:100F0000FFFF0401AA287201FFFF0401AA28720151
:100F1000FFFF0401AA287201FFFF0401AA28720141
:100F2000FFFF04016A111E01FFFF0401BBF2100163
:100F3000FFFF0401BBF21901FFFF0401BBF2100126
:100F4000FFFF04010A287201FFFF04010A28720151
:100F5000FFFF04010A287201FFFF04010A28720141
:100F6000FFFF04010A287201FFFF04010A28720131
:100F7000FFFF04010A287201FFFF04010A28720121
:100F8000FFFF0401AA287201FFFF0401AA287201D1
:100F9000FFFF0401AA287201FFFF0401AA287201C1
:100FA000FFFF04016A111E01FFFF0401BBF21001E3
:100FB000FFFF0401BBF21901FFFF0401BBF21001A6
:100FC000FFFF04010A287201FFFF04010A287201D1
:100FD000FFFF04010A287201FFFF04010A287201C1
:100FE000FFFF04010A287201FFFF04010A287201B1
:100FF000FFFF04010A287201FFFF04010A287201A1
:10100000FFFF0401AA287201FFFF0401AA28720150
:10101000FFFF0401AA287201FFFF0401AA28720140
:10102000FFFF0401FE00FF01FFFF0401BBF21001FE
:10103000FFFF0401BBF21901FFFF0401BBF2100125
:10104000FFFF04010A287201FFFF04010A28720150
:10105000FFFF04010A287201FFFF04010A28720140
:10106000FFFF04010A287201FFFF04010A28720130
:10107000FFFF04010A287201FFFF04010A28720120
:10108000FFFF0401AA287201FFFF0401AA287201D0
:10109000FFFF0401AA287201FFFF0401AA287201C0
:1010A000FFFF0401FE00FF01FFFF0401BBF210017E
:1010B000FFFF0401BBF21901FFFF0401BBF21001A5
:1010C000FFFF04010A287201FFFF04010A287201D0
:1010D000FFFF04010A287201FFFF04010A287201C0
:1010E000FFFF04010A287201FFFF04010A287201B0
:1010F000FFFF04010A287201FFFF04010A287201A0
:10110000FFFF0401AA287201FFFF0401AA2872014F
:10111000FFFF0401AA287201FFFF0401AA2872013F
:10112000FFFF04012B222001FFFF0401BBF210018D
:10113000FFFF0401BBF21901FFFF0401BBF2100124
:10114000FFFF04010A287201FFFF04010A2872014F
:10115000FFFF04010A287201FFFF04010A2872013F
:10116000FFFF04010A287201FFFF04010A2872012F
:10117000FFFF04010A287201FFFF04010A2872011F
:10118000FFFF0401AA287201FFFF0401AA287201CF
:10119000FFFF0401AA287201FFFF0401AA287201BF
:1011A000FFFF04012B222001FFFF0401BBF210010D
:1011B000FFFF0401BBF21901FFFF0401BBF21001A4
:1011C000FFFF04010A287201FFFF04010A287201CF
:1011D000FFFF04010A287201FFFF04010A287201BF
:1011E000FFFF04010A287201FFFF04010A287201AF
:1011F000FFFF04010A287201FFFF04010A2872019F
:10120000FFFF0401AA287201FFFF0401AA2872014E
:10121000FFFF0401AA287201FFFF0401AA2872013E
:10122000FFFF0401FE00FF01FFFF0401BBF21001FC
:10123000FFFF0401BBF21901FFFF0401BBF2100123
:10124000FFFF04010A287201FFFF04010A2872014E
:10125000FFFF04010A287201FFFF04010A2872013E
:10126000FFFF04010A287201FFFF04010A2872012E
:10127000FFFF04010A287201FFFF04010A2872011E
:10128000FFFF0401AA287201FFFF0401AA287201CE
:10129000FFFF0401AA287201FFFF0401AA287201BE
:1012A000FFFF0401FE00FF01FFFF0401BBF210017C
:1012B000FFFF0401BBF21901FFFF0401BBF21001A3
:1012C000FFFF04010A287201FFFF04010A287201CE
:1012D000FFFF04010A287201FFFF04010A287201BE
:1012E000FFFF04010A287201FFFF04010A287201AE
:1012F000FFFF04010A287201FFFF04010A2872019E
:10130000FFFF0401AA287201FFFF0401AA2872014D
:10131000FFFF0401AA287201FFFF0401AA2872013D
:10132000FFFF04016A111E01FFFF0401BBF210015F
:10133000FFFF0401BBF21901FFFF0401BBF2100122
:10134000FFFF04010A287201FFFF04010A2872014D
:10135000FFFF04010A287201FFFF04010A2872013D
:10136000FFFF04010A287201FFFF04010A2872012D
:10137000FFFF04010A287201FFFF04010A2872011D
:10138000FFFF0401AA287201FFFF0401AA287201CD
:10139000FFFF0401AA287201FFFF0401AA287201BD
:1013A000FFFF04016A111E01FFFF0401BBF21001DF
:1013B000FFFF0401BBF21901FFFF0401BBF21001A2
:1013C000FFFF04010A287201FFFF04010A287201CD
:1013D000FFFF04010A287201FFFF04010A287201BD
:1013E000FFFF04010A287201FFFF04010A287201AD
:1013F000FFFF04010A287201FFFF04010A2872019D
:10140000FFFF0401AA287201FFFF0401AA2872014C
:10141000FFFF0401AA287201FFFF0401AA2872013C
:10142000FFFF0401FE00FF01FFFF0401BBF21001FA
:10143000FFFF0401BBF21901FFFF0401BBF2100121
:10144000FFFF04010A287201FFFF04010A2872014C
:10145000FFFF04010A287201FFFF04010A2872013C
:10146000FFFF04010A287201FFFF04010A2872012C
:10147000FFFF04010A287201FFFF04010A2872011C
:10148000FFFF0401AA287201FFFF0401AA287201CC
:10149000FFFF0401AA287201FFFF0401AA287201BC
:1014A000FFFF0401FE00FF01FFFF0401BBF210017A
:1014B000FFFF0401BBF21901FFFF0401BBF21001A1
:1014C000FFFF04010A287201FFFF04010A287201CC
:1014D000FFFF04010A287201FFFF04010A287201BC
:1014E000FFFF04010A287201FFFF04010A287201AC
:1014F000FFFF04010A287201FFFF04010A2872019C
:10150000FFFF0401AA287201FFFF0401AA2872014B
:10151000FFFF0401AA287201FFFF0401AA2872013B
:10152000FFFF04012B282001FFFF0401BBF2100183
:10153000FFFF0401BBF21901FFFF0401BBF2100120
:10154000FFFF04010A287201FFFF04010A2872014B
:10155000FFFF04010A287201FFFF04010A2872013B
:10156000FFFF04010A287201FFFF04010A2872012B
:10157000FFFF04010A287201FFFF04010A2872011B
:10158000FFFF0401AA287201FFFF0401AA287201CB
:10159000FFFF0401AA287201FFFF0401AA287201BB
:1015A000FFFF04012B282001FFFF0401BBF2100103
:1015B000FFFF0401BBF21901FFFF0401BBF21001A0
:1015C000FFFF04010A287201FFFF04010A287201CB
:1015D000FFFF04010A287201FFFF04010A287201BB
:1015E000FFFF04010A287201FFFF04010A287201AB
:1015F000FFFF04010A287201FFFF04010A2872019B
:10160000FFFF0401AA287201FFFF0401AA2872014A
:10161000FFFF0401AA287201FFFF0401AA2872013A
:10162000FFFF0401FE00FF01FFFF0401BBF21001F8
:10163000FFFF0401BBF21901FFFF0401BBF210011F
:10164000FFFF04010A287201FFFF04010A2872014A
:10165000FFFF04010A287201FFFF04010A2872013A
:10166000FFFF04010A287201FFFF04010A2872012A
:10167000FFFF04010A287201FFFF04010A2872011A
:10168000FFFF0401AA287201FFFF0401AA287201CA
:10169000FFFF0401AA287201FFFF0401AA287201BA
:1016A000FFFF0401FE00FF01FFFF0401BBF2100178
:1016B000FFFF0401BBF21901FFFF0401BBF210019F
:1016C000FFFF04010A287201FFFF04010A287201CA
:1016D000FFFF04010A287201FFFF04010A287201BA
:1016E000FFFF04010A287201FFFF04010A287201AA
:1016F000FFFF04010A287201FFFF04010A2872019A
:10170000FFFF0401AA287201FFFF0401AA28720149
:10171000FFFF0401AA287201FFFF0401AA28720139
:10172000FFFF04016A111E01FFFF0401BBF210015B
:10173000FFFF0401BBF21901FFFF0401BBF210011E
:10174000FFFF04010A287201FFFF04010A28720149
:10175000FFFF04010A287201FFFF04010A28720139
:10176000FFFF04010A287201FFFF04010A28720129
:10177000FFFF04010A287201FFFF04010A28720119
:10178000FFFF0401AA287201FFFF0401AA287201C9
:10179000FFFF0401AA287201FFFF0401AA287201B9
:1017A000FFFF04016A111E01FFFF0401BBF21001DB
:1017B000FFFF0401BBF21901FFFF0401BBF210019E
:1017C000FFFF04010A287201FFFF04010A287201C9
:1017D000FFFF04010A287201FFFF04010A287201B9
:1017E000FFFF04010A287201FFFF04010A287201A9
:1017F000FFFF04010A287201FFFF04010A28720199
:10180000FFFF0401AA287201FFFF0401AA28720148
:10181000FFFF0401AA287201FFFF0401AA28720138
:10182000FFFF0401FE00FF01FFFF0401BBF21001F6
:10183000FFFF0401BBF21901FFFF0401BBF210011D
:10184000FFFF04010A287201FFFF04010A28720148
:10185000FFFF04010A287201FFFF04010A28720138
:10186000FFFF04010A287201FFFF04010A28720128
:10187000FFFF04010A287201FFFF04010A28720118
:10188000FFFF0401AA287201FFFF0401AA287201C8
:10189000FFFF0401AA287201FFFF0401AA287201B8
:1018A000FFFF0401FE00FF01FFFF0401BBF2100176
:1018B000FFFF0401BBF21901FFFF0401BBF210019D
:1018C000FFFF04010A287201FFFF04010A287201C8
:1018D000FFFF04010A287201FFFF04010A287201B8
:1018E000FFFF04010A287201FFFF04010A287201A8
:1018F000FFFF04010A287201FFFF04010A28720198
:10190000FFFF0401AA287201FFFF0401AA28720147
:10191000FFFF0401AA287201FFFF0401AA28720137
:10192000FFFF04012B242001FFFF0401BBF2100183
:10193000FFFF0401BBF21901FFFF0401BBF210011C
:10194000FFFF04010A287201FFFF04010A28720147
:10195000FFFF04010A287201FFFF04010A28720137
:10196000FFFF04010A287201FFFF04010A28720127
:10197000FFFF04010A287201FFFF04010A28720117
:10198000FFFF0401AA287201FFFF0401AA287201C7
:10199000FFFF0401AA287201FFFF0401AA287201B7
:1019A000FFFF04012B242001FFFF0401BBF2100103
:1019B000FFFF0401BBF21901FFFF0401BBF210019C
:1019C000FFFF04010A287201FFFF04010A287201C7
:1019D000FFFF04010A287201FFFF04010A287201B7
:1019E000FFFF04010A287201FFFF04010A287201A7
:1019F000FFFF04010A287201FFFF04010A28720197
:101A0000FFFF0401AA287201FFFF0401AA28720146
:101A1000FFFF0401AA287201FFFF0401AA28720136
:101A2000FFFF0401FE00FF01FFFF0401BBF21001F4
:101A3000FFFF0401BBF21901FFFF0401BBF210011B
:101A4000FFFF04010A287201FFFF04010A28720146
:101A5000FFFF04010A287201FFFF04010A28720136
:101A6000FFFF04010A287201FFFF04010A28720126
:101A7000FFFF04010A287201FFFF04010A28720116
:101A8000FFFF0401AA287201FFFF0401AA287201C6
:101A9000FFFF0401AA287201FFFF0401AA287201B6
:101AA000FFFF0401FE00FF01FFFF0401BBF2100174
:101AB000FFFF0401BBF21901FFFF0401BBF210019B
:101AC000FFFF04010A287201FFFF04010A287201C6
:101AD000FFFF04010A287201FFFF04010A287201B6
:101AE000FFFF04010A287201FFFF04010A287201A6
:101AF000FFFF04010A287201FFFF04010A28720196
:101B0000FFFF0401AA287201FFFF0401AA28720145
:101B1000FFFF0401AA287201FFFF0401AA28720135
:101B2000FFFF04016A111E01FFFF0401BBF2100157
:101B3000FFFF0401BBF21901FFFF0401BBF210011A
:101B4000FFFF04010A287201FFFF04010A28720145
:101B5000FFFF04010A287201FFFF04010A28720135
:101B6000FFFF04010A287201FFFF04010A28720125
:101B7000FFFF04010A287201FFFF04010A28720115
:101B8000FFFF0401AA287201FFFF0401AA287201C5
:101B9000FFFF0401AA287201FFFF0401AA287201B5
:101BA000FFFF04016A111E01FFFF0401BBF21001D7
:101BB000FFFF0401BBF21901FFFF0401BBF210019A
:101BC000FFFF04010A287201FFFF04010A287201C5
:101BD000FFFF04010A287201FFFF04010A287201B5
:101BE000FFFF04010A287201FFFF04010A287201A5
:101BF000FFFF04010A287201FFFF04010A28720195
:101C0000FFFF0401AA287201FFFF0401AA28720144
:101C1000FFFF0401AA287201FFFF0401AA28720134
:101C2000FFFF0401FE00FF01FFFF0401BBF21001F2
:101C3000FFFF0401BBF21901FFFF0401BBF2100119
:101C4000FFFF04010A287201FFFF04010A28720144
:101C5000FFFF04010A287201FFFF04010A28720134
:101C6000FFFF04010A287201FFFF04010A28720124
:101C7000FFFF04010A287201FFFF04010A28720114
:101C8000FFFF0401AA287201FFFF0401AA287201C4
:101C9000FFFF0401AA287201FFFF0401AA287201B4
:101CA000FFFF0401FE00FF01FFFF0401BBF2100172
:101CB000FFFF0401BBF21901FFFF0401BBF2100199
:101CC000FFFF04010A287201FFFF04010A287201C4
:101CD000FFFF04010A287201FFFF04010A287201B4
:101CE000FFFF04010A287201FFFF04010A287201A4
:101CF000FFFF04010A287201FFFF04010A28720194
:101D0000FFFF0401AA287201FFFF0401AA28720143
:101D1000FFFF0401AA287201FFFF0401AA28720133
:101D2000FFFF04012B282001FFFF0401BBF210017B
:101D3000FFFF0401BBF21901FFFF0401BBF2100118
:101D4000FFFF04010A287201FFFF04010A28720143
:101D5000FFFF04010A287201FFFF04010A28720133
:101D6000FFFF04010A287201FFFF04010A28720123
:101D7000FFFF04010A287201FFFF04010A28720113
:101D8000FFFF0401AA287201FFFF0401AA287201C3
:101D9000FFFF0401AA287201FFFF0401AA287201B3
:101DA000FFFF04012B282001FFFF0401BBF21001FB
:101DB000FFFF0401BBF21901FFFF0401BBF2100198
:101DC000FFFF04010A287201FFFF04010A287201C3
:101DD000FFFF04010A287201FFFF04010A287201B3
:101DE000FFFF04010A287201FFFF04010A287201A3
:101DF000FFFF04010A287201FFFF04010A28720193
:101E0000FFFF0401AA287201FFFF0401AA28720142
:101E1000FFFF0401AA287201FFFF0401AA28720132
:101E2000FFFF0401FE00FF01FFFF0401BBF21001F0
:101E3000FFFF0401BBF21901FFFF0401BBF2100117
:101E4000FFFF04010A287201FFFF04010A28720142
:101E5000FFFF04010A287201FFFF04010A28720132
:101E6000FFFF04010A287201FFFF04010A28720122
:101E7000FFFF04010A287201FFFF04010A28720112
:101E8000FFFF0401AA287201FFFF0401AA287201C2
:101E9000FFFF0401AA287201FFFF0401AA287201B2
:101EA000FFFF0401FE00FF01FFFF0401BBF2100170
:101EB000FFFF0401BBF21901FFFF0401BBF2100197
:101EC000FFFF04010A287201FFFF04010A287201C2
:101ED000FFFF04010A287201FFFF04010A287201B2
:101EE000FFFF04010A287201FFFF04010A287201A2
:101EF000FFFF04010A287201FFFF04010A28720192
:101F0000FFFF0401AA287201FFFF0401AA28720141
:101F1000FFFF0401AA287201FFFF0401AA28720131
:101F2000FFFF04016A111E01FFFF0401BBF2100153
:101F3000FFFF0401BBF21901FFFF0401BBF2100116
:101F4000FFFF04010A287201FFFF04010A28720141
:101F5000FFFF04010A287201FFFF04010A28720131
:101F6000FFFF04010A287201FFFF04010A28720121
:101F7000FFFF04010A287201FFFF04010A28720111
:101F8000FFFF0401AA287201FFFF0401AA287201C1
:101F9000FFFF0401AA287201FFFF0401AA287201B1
:101FA000FFFF04016A111E01FFFF0401BBF21001D3
:101FB000FFFF0401BBF21901FFFF0401BBF2100196
:101FC000FFFF04010A287201FFFF04010A287201C1
:101FD000FFFF04010A287201FFFF04010A287201B1
:101FE000FFFF04010A287201FFFF04010A287201A1
:101FF000FFFF04010A287201FFFF04010A28720191
:10200000FFFF0401AA287201FFFF0401AA28720140
:10201000FFFF0401AA287201FFFF0401AA28720130
:10202000FFFF0401FE00FF01FFFF0401BBF21001EE
:10203000FFFF0401BBF21901FFFF0401BBF2100115
:10204000FFFF04010A287201FFFF04010A28720140
:10205000FFFF04010A287201FFFF04010A28720130
:10206000FFFF04010A287201FFFF04010A28720120
:10207000FFFF04010A287201FFFF04010A28720110
:10208000FFFF0401AA287201FFFF0401AA287201C0
:10209000FFFF0401AA287201FFFF0401AA287201B0
:1020A000FFFF0401FE00FF01FFFF0401BBF210016E
:1020B000FFFF0401BBF21901FFFF0401BBF2100195
:1020C000FFFF04010A287201FFFF04010A287201C0
:1020D000FFFF04010A287201FFFF04010A287201B0
:1020E000FFFF04010A287201FFFF04010A287201A0
:1020F000FFFF04010A287201FFFF04010A28720190
:10210000FFFF0401AA287201FFFF0401AA2872013F
:10211000FFFF0401AA287201FFFF0401AA2872012F
:10212000FFFF04012B212001FFFF0401BBF210017E
:10213000FFFF0401BBF21901FFFF0401BBF2100114
:10214000FFFF04010A287201FFFF04010A2872013F
:10215000FFFF04010A287201FFFF04010A2872012F
:10216000FFFF04010A287201FFFF04010A2872011F
:10217000FFFF04010A287201FFFF04010A2872010F
:10218000FFFF0401AA287201FFFF0401AA287201BF
:10219000FFFF0401AA287201FFFF0401AA287201AF
:1021A000FFFF04012B212001FFFF0401BBF21001FE
:1021B000FFFF0401BBF21901FFFF0401BBF2100194
:1021C000FFFF04010A287201FFFF04010A287201BF
:1021D000FFFF04010A287201FFFF04010A287201AF
:1021E000FFFF04010A287201FFFF04010A2872019F
:1021F000FFFF04010A287201FFFF04010A2872018F
:10220000FFFF0401AA287201FFFF0401AA2872013E
:10221000FFFF0401AA287201FFFF0401AA2872012E
:10222000FFFF0401FE00FF01FFFF0401BBF21001EC
:10223000FFFF0401BBF21901FFFF0401BBF2100113
:10224000FFFF04010A287201FFFF04010A2872013E
:10225000FFFF04010A287201FFFF04010A2872012E
:10226000FFFF04010A287201FFFF04010A2872011E
:10227000FFFF04010A287201FFFF04010A2872010E
:10228000FFFF0401AA287201FFFF0401AA287201BE
:10229000FFFF0401AA287201FFFF0401AA287201AE
:1022A000FFFF0401FE00FF01FFFF0401BBF210016C
:1022B000FFFF0401BBF21901FFFF0401BBF2100193
:1022C000FFFF04010A287201FFFF04010A287201BE
:1022D000FFFF04010A287201FFFF04010A287201AE
:1022E000FFFF04010A287201FFFF04010A2872019E
:1022F000FFFF04010A287201FFFF04010A2872018E
:10230000FFFF0401AA287201FFFF0401AA2872013D
:10231000FFFF0401AA287201FFFF0401AA2872012D
:10232000FFFF04016A111E01FFFF0401BBF210014F
:10233000FFFF0401BBF21901FFFF0401BBF2100112
:10234000FFFF04010A287201FFFF04010A2872013D
:10235000FFFF04010A287201FFFF04010A2872012D
:10236000FFFF04010A287201FFFF04010A2872011D
:10237000FFFF04010A287201FFFF04010A2872010D
:10238000FFFF0401AA287201FFFF0401AA287201BD
:10239000FFFF0401AA287201FFFF0401AA287201AD
:1023A000FFFF04016A111E01FFFF0401BBF21001CF
:1023B000FFFF0401BBF21901FFFF0401BBF2100192
:1023C000FFFF04010A287201FFFF04010A287201BD
:1023D000FFFF04010A287201FFFF04010A287201AD
:1023E000FFFF04010A287201FFFF04010A2872019D
:1023F000FFFF04010A287201FFFF04010A2872018D
:10240000FFFF0401AA287201FFFF0401AA2872013C
:10241000FFFF0401AA287201FFFF0401AA2872012C
:10242000FFFF0401FE00FF01FFFF0401BBF21001EA
:10243000FFFF0401BBF21901FFFF0401BBF2100111
:10244000FFFF04010A287201FFFF04010A2872013C
:10245000FFFF04010A287201FFFF04010A2872012C
:10246000FFFF04010A287201FFFF04010A2872011C
:10247000FFFF04010A287201FFFF04010A2872010C
:10248000FFFF0401AA287201FFFF0401AA287201BC
:10249000FFFF0401AA287201FFFF0401AA287201AC
:1024A000FFFF0401FE00FF01FFFF0401BBF210016A
:1024B000FFFF0401BBF21901FFFF0401BBF2100191
:1024C000FFFF04010A287201FFFF04010A287201BC
:1024D000FFFF04010A287201FFFF04010A287201AC
:1024E000FFFF04010A287201FFFF04010A2872019C
:1024F000FFFF04010A287201FFFF04010A2872018C
:10250000FFFF0401AA287201FFFF0401AA2872013B
:10251000FFFF0401AA287201FFFF0401AA2872012B
:10252000FFFF04012B282001FFFF0401BBF2100173
:10253000FFFF0401BBF21901FFFF0401BBF2100110
:10254000FFFF04010A287201FFFF04010A2872013B
:10255000FFFF04010A287201FFFF04010A2872012B
:10256000FFFF04010A287201FFFF04010A2872011B
:10257000FFFF04010A287201FFFF04010A2872010B
:10258000FFFF0401AA287201FFFF0401AA287201BB
:10259000FFFF0401AA287201FFFF0401AA287201AB
:1025A000FFFF04012B282001FFFF0401BBF21001F3
:1025B000FFFF0401BBF21901FFFF0401BBF2100190
:1025C000FFFF04010A287201FFFF04010A287201BB
:1025D000FFFF04010A287201FFFF04010A287201AB
:1025E000FFFF04010A287201FFFF04010A2872019B
:1025F000FFFF04010A287201FFFF04010A2872018B
:10260000FFFF0401AA287201FFFF0401AA2872013A
:10261000FFFF0401AA287201FFFF0401AA2872012A
:10262000FFFF0401FE00FF01FFFF0401BBF21001E8
:10263000FFFF0401BBF21901FFFF0401BBF210010F
:10264000FFFF04010A287201FFFF04010A2872013A
:10265000FFFF04010A287201FFFF04010A2872012A
:10266000FFFF04010A287201FFFF04010A2872011A
:10267000FFFF04010A287201FFFF04010A2872010A
:10268000FFFF0401AA287201FFFF0401AA287201BA
:10269000FFFF0401AA287201FFFF0401AA287201AA
:1026A000FFFF0401FE00FF01FFFF0401BBF2100168
:1026B000FFFF0401BBF21901FFFF0401BBF210018F
:1026C000FFFF04010A287201FFFF04010A287201BA
:1026D000FFFF04010A287201FFFF04010A287201AA
:1026E000FFFF04010A287201FFFF04010A2872019A
:1026F000FFFF04010A287201FFFF04010A2872018A
:10270000FFFF0401AA287201FFFF0401AA28720139
:10271000FFFF0401AA287201FFFF0401AA28720129
:10272000FFFF04016A111E01FFFF0401BBF210014B
:10273000FFFF0401BBF21901FFFF0401BBF210010E
:10274000FFFF04010A287201FFFF04010A28720139
:10275000FFFF04010A287201FFFF04010A28720129
:10276000FFFF04010A287201FFFF04010A28720119
:10277000FFFF04010A287201FFFF04010A28720109
:10278000FFFF0401AA287201FFFF0401AA287201B9
:10279000FFFF0401AA287201FFFF0401AA287201A9
:1027A000FFFF04016A111E01FFFF0401BBF21001CB
:1027B000FFFF0401BBF21901FFFF0401BBF210018E
:1027C000FFFF04010A287201FFFF04010A287201B9
:1027D000FFFF04010A287201FFFF04010A287201A9
:1027E000FFFF04010A287201FFFF04010A28720199
:1027F000FFFF04010A287201FFFF04010A28720189
:10280000FFFF0401AA287201FFFF0401AA28720138
:10281000FFFF0401AA287201FFFF0401AA28720128
:10282000FFFF0401FE00FF01FFFF0401BBF21001E6
:10283000FFFF0401BBF21901FFFF0401BBF210010D
:10284000FFFF04010A287201FFFF04010A28720138
:10285000FFFF04010A287201FFFF04010A28720128
:10286000FFFF04010A287201FFFF04010A28720118
:10287000FFFF04010A287201FFFF04010A28720108
:10288000FFFF0401AA287201FFFF0401AA287201B8
:10289000FFFF0401AA287201FFFF0401AA287201A8
:1028A000FFFF0401FE00FF01FFFF0401BBF2100166
:1028B000FFFF0401BBF21901FFFF0401BBF210018D
:1028C000FFFF04010A287201FFFF04010A287201B8
:1028D000FFFF04010A287201FFFF04010A287201A8
:1028E000FFFF04010A287201FFFF04010A28720198
:1028F000FFFF04010A287201FFFF04010A28720188
:10290000FFFF0401AA287201FFFF0401AA28720137
:10291000FFFF0401AA287201FFFF0401AA28720127
:10292000FFFF04012B242001FFFF0401BBF2100173
:10293000FFFF0401BBF21901FFFF0401BBF210010C
:10294000FFFF04010A287201FFFF04010A28720137
:10295000FFFF04010A287201FFFF04010A28720127
:10296000FFFF04010A287201FFFF04010A28720117
:10297000FFFF04010A287201FFFF04010A28720107
:10298000FFFF0401AA287201FFFF0401AA287201B7
:10299000FFFF0401AA287201FFFF0401AA287201A7
:1029A000FFFF04012B242001FFFF0401BBF21001F3
:1029B000FFFF0401BBF21901FFFF0401BBF210018C
:1029C000FFFF04010A287201FFFF04010A287201B7
:1029D000FFFF04010A287201FFFF04010A287201A7
:1029E000FFFF04010A287201FFFF04010A28720197
:1029F000FFFF04010A287201FFFF04010A28720187
:102A0000FFFF0401AA287201FFFF0401AA28720136
:102A1000FFFF0401AA287201FFFF0401AA28720126
:102A2000FFFF0401FE00FF01FFFF0401BBF21001E4
:102A3000FFFF0401BBF21901FFFF0401BBF210010B
:102A4000FFFF04010A287201FFFF04010A28720136
:102A5000FFFF04010A287201FFFF04010A28720126
:102A6000FFFF04010A287201FFFF04010A28720116
:102A7000FFFF04010A287201FFFF04010A28720106
:102A8000FFFF0401AA287201FFFF0401AA287201B6
:102A9000FFFF0401AA287201FFFF0401AA287201A6
:102AA000FFFF0401FE00FF01FFFF0401BBF2100164
:102AB000FFFF0401BBF21901FFFF0401BBF210018B
:102AC000FFFF04010A287201FFFF04010A287201B6
:102AD000FFFF04010A287201FFFF04010A287201A6
:102AE000FFFF04010A287201FFFF04010A28720196
:102AF000FFFF04010A287201FFFF04010A28720186
:102B0000FFFF0401AA287201FFFF0401AA28720135
:102B1000FFFF0401AA287201FFFF0401AA28720125
:102B2000FFFF04016A111E01FFFF0401BBF2100147
:102B3000FFFF0401BBF21901FFFF0401BBF210010A
:102B4000FFFF04010A287201FFFF04010A28720135
:102B5000FFFF04010A287201FFFF04010A28720125
:102B6000FFFF04010A287201FFFF04010A28720115
:102B7000FFFF04010A287201FFFF04010A28720105
:102B8000FFFF0401AA287201FFFF0401AA287201B5
:102B9000FFFF0401AA287201FFFF0401AA287201A5
:102BA000FFFF04016A111E01FFFF0401BBF21001C7
:102BB000FFFF0401BBF21901FFFF0401BBF210018A
:102BC000FFFF04010A287201FFFF04010A287201B5
:102BD000FFFF04010A287201FFFF04010A287201A5
:102BE000FFFF04010A287201FFFF04010A28720195
:102BF000FFFF04010A287201FFFF04010A28720185
:102C0000FFFF0401AA287201FFFF0401AA28720134
:102C1000FFFF0401AA287201FFFF0401AA28720124
:102C2000FFFF0401FE00FF01FFFF0401BBF21001E2
:102C3000FFFF0401BBF21901FFFF0401BBF2100109
:102C4000FFFF04010A287201FFFF04010A28720134
:102C5000FFFF04010A287201FFFF04010A28720124
:102C6000FFFF04010A287201FFFF04010A28720114
:102C7000FFFF04010A287201FFFF04010A28720104
:102C8000FFFF0401AA287201FFFF0401AA287201B4
:102C9000FFFF0401AA287201FFFF0401AA287201A4
:102CA000FFFF0401FE00FF01FFFF0401BBF2100162
:102CB000FFFF0401BBF21901FFFF0401BBF2100189
:102CC000FFFF04010A287201FFFF04010A287201B4
:102CD000FFFF04010A287201FFFF04010A287201A4
:102CE000FFFF04010A287201FFFF04010A28720194
:102CF000FFFF04010A287201FFFF04010A28720184
:102D0000FFFF0401AA287201FFFF0401AA28720133
:102D1000FFFF0401AA287201FFFF0401AA28720123
:102D2000FFFF04012B282001FFFF0401BBF210016B
:102D3000FFFF0401BBF21901FFFF0401BBF2100108
:102D4000FFFF04010A287201FFFF04010A28720133
:102D5000FFFF04010A287201FFFF04010A28720123
:102D6000FFFF04010A287201FFFF04010A28720113
:102D7000FFFF04010A287201FFFF04010A28720103
:102D8000FFFF0401AA287201FFFF0401AA287201B3
:102D9000FFFF0401AA287201FFFF0401AA287201A3
:102DA000FFFF04012B282001FFFF0401BBF21001EB
:102DB000FFFF0401BBF21901FFFF0401BBF2100188
:102DC000FFFF04010A287201FFFF04010A287201B3
:102DD000FFFF04010A287201FFFF04010A287201A3
:102DE000FFFF04010A287201FFFF04010A28720193
:102DF000FFFF04010A287201FFFF04010A28720183
:102E0000FFFF0401AA287201FFFF0401AA28720132
:102E1000FFFF0401AA287201FFFF0401AA28720122
:102E2000FFFF0401FE00FF01FFFF0401BBF21001E0
:102E3000FFFF0401BBF21901FFFF0401BBF2100107
:102E4000FFFF04010A287201FFFF04010A28720132
:102E5000FFFF04010A287201FFFF04010A28720122
:102E6000FFFF04010A287201FFFF04010A28720112
:102E7000FFFF04010A287201FFFF04010A28720102
:102E8000FFFF0401AA287201FFFF0401AA287201B2
:102E9000FFFF0401AA287201FFFF0401AA287201A2
:102EA000FFFF0401FE00FF01FFFF0401BBF2100160
:102EB000FFFF0401BBF21901FFFF0401BBF2100187
:102EC000FFFF04010A287201FFFF04010A287201B2
:102ED000FFFF04010A287201FFFF04010A287201A2
:102EE000FFFF04010A287201FFFF04010A28720192
:102EF000FFFF04010A287201FFFF04010A28720182
:102F0000FFFF0401AA287201FFFF0401AA28720131
:102F1000FFFF0401AA287201FFFF0401AA28720121
:102F2000FFFF04016A111E01FFFF0401BBF2100143
:102F3000FFFF0401BBF21901FFFF0401BBF2100106
:102F4000FFFF04010A287201FFFF04010A28720131
:102F5000FFFF04010A287201FFFF04010A28720121
:102F6000FFFF04010A287201FFFF04010A28720111
:102F7000FFFF04010A287201FFFF04010A28720101
:102F8000FFFF0401AA287201FFFF0401AA287201B1
:102F9000FFFF0401AA287201FFFF0401AA287201A1
:102FA000FFFF04016A111E01FFFF0401BBF21001C3
:102FB000FFFF0401BBF21901FFFF0401BBF2100186
:102FC000FFFF04010A287201FFFF04010A287201B1
:102FD000FFFF04010A287201FFFF04010A287201A1
:102FE000FFFF04010A287201FFFF04010A28720191
:102FF000FFFF04010A287201FFFF04010A28720181
:10300000FFFF0401AA287201FFFF0401AA28720130
:10301000FFFF0401AA287201FFFF0401AA28720120
:10302000FFFF0401FE00FF01FFFF0401BBF21001DE
:10303000FFFF0401BBF21901FFFF0401BBF2100105
:10304000FFFF04010A287201FFFF04010A28720130
:10305000FFFF04010A287201FFFF04010A28720120
:10306000FFFF04010A287201FFFF04010A28720110
:10307000FFFF04010A287201FFFF04010A28720100
:10308000FFFF0401AA287201FFFF0401AA287201B0
:10309000FFFF0401AA287201FFFF0401AA287201A0
:1030A000FFFF0401FE00FF01FFFF0401BBF210015E
:1030B000FFFF0401BBF21901FFFF0401BBF2100185
:1030C000FFFF04010A287201FFFF04010A287201B0
:1030D000FFFF04010A287201FFFF04010A287201A0
:1030E000FFFF04010A287201FFFF04010A28720190
:1030F000FFFF04010A287201FFFF04010A28720180
:10310000FFFF0401AA287201FFFF0401AA2872012F
:10311000FFFF0401AA287201FFFF0401AA2872011F
:10312000FFFF04012B222001FFFF0401BBF210016D
:10313000FFFF0401BBF21901FFFF0401BBF2100104
:10314000FFFF04010A287201FFFF04010A2872012F
:10315000FFFF04010A287201FFFF04010A2872011F
:10316000FFFF04010A287201FFFF04010A2872010F
:10317000FFFF04010A287201FFFF04010A287201FF
:10318000FFFF0401AA287201FFFF0401AA287201AF
:10319000FFFF0401AA287201FFFF0401AA2872019F
:1031A000FFFF04012B222001FFFF0401BBF21001ED
:1031B000FFFF0401BBF21901FFFF0401BBF2100184
:1031C000FFFF04010A287201FFFF04010A287201AF
:1031D000FFFF04010A287201FFFF04010A2872019F
:1031E000FFFF04010A287201FFFF04010A2872018F
:1031F000FFFF04010A287201FFFF04010A2872017F
:10320000FFFF0401AA287201FFFF0401AA2872012E
:10321000FFFF0401AA287201FFFF0401AA2872011E
:10322000FFFF0401FE00FF01FFFF0401BBF21001DC
:10323000FFFF0401BBF21901FFFF0401BBF2100103
:10324000FFFF04010A287201FFFF04010A2872012E
:10325000FFFF04010A287201FFFF04010A2872011E
:10326000FFFF04010A287201FFFF04010A2872010E
:10327000FFFF04010A287201FFFF04010A287201FE
:10328000FFFF0401AA287201FFFF0401AA287201AE
:10329000FFFF0401AA287201FFFF0401AA2872019E
:1032A000FFFF0401FE00FF01FFFF0401BBF210015C
:1032B000FFFF0401BBF21901FFFF0401BBF2100183
:1032C000FFFF04010A287201FFFF04010A287201AE
:1032D000FFFF04010A287201FFFF04010A2872019E
:1032E000FFFF04010A287201FFFF04010A2872018E
:1032F000FFFF04010A287201FFFF04010A2872017E
:10330000FFFF0401AA287201FFFF0401AA2872012D
:10331000FFFF0401AA287201FFFF0401AA2872011D
:10332000FFFF04016A111E01FFFF0401BBF210013F
:10333000FFFF0401BBF21901FFFF0401BBF2100102
:10334000FFFF04010A287201FFFF04010A2872012D
:10335000FFFF04010A287201FFFF04010A2872011D
:10336000FFFF04010A287201FFFF04010A2872010D
:10337000FFFF04010A287201FFFF04010A287201FD
:10338000FFFF0401AA287201FFFF0401AA287201AD
:10339000FFFF0401AA287201FFFF0401AA2872019D
:1033A000FFFF04016A111E01FFFF0401BBF21001BF
:1033B000FFFF0401BBF21901FFFF0401BBF2100182
:1033C000FFFF04010A287201FFFF04010A287201AD
:1033D000FFFF04010A287201FFFF04010A2872019D
:1033E000FFFF04010A287201FFFF04010A2872018D
:1033F000FFFF04010A287201FFFF04010A2872017D
:10340000FFFF0401AA287201FFFF0401AA2872012C
:10341000FFFF0401AA287201FFFF0401AA2872011C
:10342000FFFF0401FE00FF01FFFF0401BBF21001DA
:10343000FFFF0401BBF21901FFFF0401BBF2100101
:10344000FFFF04010A287201FFFF04010A2872012C
:10345000FFFF04010A287201FFFF04010A2872011C
:10346000FFFF04010A287201FFFF04010A2872010C
:10347000FFFF04010A287201FFFF04010A287201FC
:10348000FFFF0401AA287201FFFF0401AA287201AC
:10349000FFFF0401AA287201FFFF0401AA2872019C
:1034A000FFFF0401FE00FF01FFFF0401BBF210015A
:1034B000FFFF0401BBF21901FFFF0401BBF2100181
:1034C000FFFF04010A287201FFFF04010A287201AC
:1034D000FFFF04010A287201FFFF04010A2872019C
:1034E000FFFF04010A287201FFFF04010A2872018C
:1034F000FFFF04010A287201FFFF04010A2872017C
:10350000FFFF0401AA287201FFFF0401AA2872012B
:10351000FFFF0401AA287201FFFF0401AA2872011B
:10352000FFFF04012B282001FFFF0401BBF2100163
:10353000FFFF0401BBF21901FFFF0401BBF2100100
:10354000FFFF04010A287201FFFF04010A2872012B
:10355000FFFF04010A287201FFFF04010A2872011B
:10356000FFFF04010A287201FFFF04010A2872010B
:10357000FFFF04010A287201FFFF04010A287201FB
:10358000FFFF0401AA287201FFFF0401AA287201AB
:10359000FFFF0401AA287201FFFF0401AA2872019B
:1035A000FFFF04012B282001FFFF0401BBF21001E3
:1035B000FFFF0401BBF21901FFFF0401BBF2100180
:1035C000FFFF04010A287201FFFF04010A287201AB
:1035D000FFFF04010A287201FFFF04010A2872019B
:1035E000FFFF04010A287201FFFF04010A2872018B
:1035F000FFFF04010A287201FFFF04010A2872017B
:10360000FFFF0401AA287201FFFF0401AA2872012A
:10361000FFFF0401AA287201FFFF0401AA2872011A
:10362000FFFF0401FE00FF01FFFF0401BBF21001D8
:10363000FFFF0401BBF21901FFFF0401BBF21001FF
:10364000FFFF04010A287201FFFF04010A2872012A
:10365000FFFF04010A287201FFFF04010A2872011A
:10366000FFFF04010A287201FFFF04010A2872010A
:10367000FFFF04010A287201FFFF04010A287201FA
:10368000FFFF0401AA287201FFFF0401AA287201AA
:10369000FFFF0401AA287201FFFF0401AA2872019A
:1036A000FFFF0401FE00FF01FFFF0401BBF2100158
:1036B000FFFF0401BBF21901FFFF0401BBF210017F
:1036C000FFFF04010A287201FFFF04010A287201AA
:1036D000FFFF04010A287201FFFF04010A2872019A
:1036E000FFFF04010A287201FFFF04010A2872018A
:1036F000FFFF04010A287201FFFF04010A2872017A
:10370000FFFF0401AA287201FFFF0401AA28720129
:10371000FFFF0401AA287201FFFF0401AA28720119
:10372000FFFF04016A111E01FFFF0401BBF210013B
:10373000FFFF0401BBF21901FFFF0401BBF21001FE
:10374000FFFF04010A287201FFFF04010A28720129
:10375000FFFF04010A287201FFFF04010A28720119
:10376000FFFF04010A287201FFFF04010A28720109
:10377000FFFF04010A287201FFFF04010A287201F9
:10378000FFFF0401AA287201FFFF0401AA287201A9
:10379000FFFF0401AA287201FFFF0401AA28720199
:1037A000FFFF04016A111E01FFFF0401BBF21001BB
:1037B000FFFF0401BBF21901FFFF0401BBF210017E
:1037C000FFFF04010A287201FFFF04010A287201A9
:1037D000FFFF04010A287201FFFF04010A28720199
:1037E000FFFF04010A287201FFFF04010A28720189
:1037F000FFFF04010A287201FFFF04010A28720179
:10380000FFFF0401AA287201FFFF0401AA28720128
:10381000FFFF0401AA287201FFFF0401AA28720118
:10382000FFFF0401FE00FF01FFFF0401BBF21001D6
:10383000FFFF0401BBF21901FFFF0401BBF21001FD
:10384000FFFF04010A287201FFFF04010A28720128
:10385000FFFF04010A287201FFFF04010A28720118
:10386000FFFF04010A287201FFFF04010A28720108
:10387000FFFF04010A287201FFFF04010A287201F8
:10388000FFFF0401AA287201FFFF0401AA287201A8
:10389000FFFF0401AA287201FFFF0401AA28720198
:1038A000FFFF0401FE00FF01FFFF0401BBF2100156
:1038B000FFFF0401BBF21901FFFF0401BBF210017D
:1038C000FFFF04010A287201FFFF04010A287201A8
:1038D000FFFF04010A287201FFFF04010A28720198
:1038E000FFFF04010A287201FFFF04010A28720188
:1038F000FFFF04010A287201FFFF04010A28720178
:10390000FFFF0401AA287201FFFF0401AA28720127
:10391000FFFF0401AA287201FFFF0401AA28720117
:10392000FFFF04012B242001FFFF0401BBF2100163
:10393000FFFF0401BBF21901FFFF0401BBF21001FC
:10394000FFFF04010A287201FFFF04010A28720127
:10395000FFFF04010A287201FFFF04010A28720117
:10396000FFFF04010A287201FFFF04010A28720107
:10397000FFFF04010A287201FFFF04010A287201F7
:10398000FFFF0401AA287201FFFF0401AA287201A7
:10399000FFFF0401AA287201FFFF0401AA28720197
:1039A000FFFF04012B242001FFFF0401BBF21001E3
:1039B000FFFF0401BBF21901FFFF0401BBF210017C
:1039C000FFFF04010A287201FFFF04010A287201A7
:1039D000FFFF04010A287201FFFF04010A28720197
:1039E000FFFF04010A287201FFFF04010A28720187
:1039F000FFFF04010A287201FFFF04010A28720177
:103A0000FFFF0401AA287201FFFF0401AA28720126
:103A1000FFFF0401AA287201FFFF0401AA28720116
:103A2000FFFF0401FE00FF01FFFF0401BBF21001D4
:103A3000FFFF0401BBF21901FFFF0401BBF21001FB
:103A4000FFFF04010A287201FFFF04010A28720126
:103A5000FFFF04010A287201FFFF04010A28720116
:103A6000FFFF04010A287201FFFF04010A28720106
:103A7000FFFF04010A287201FFFF04010A287201F6
:103A8000FFFF0401AA287201FFFF0401AA287201A6
:103A9000FFFF0401AA287201FFFF0401AA28720196
:103AA000FFFF0401FE00FF01FFFF0401BBF2100154
:103AB000FFFF0401BBF21901FFFF0401BBF210017B
:103AC000FFFF04010A287201FFFF04010A287201A6
:103AD000FFFF04010A287201FFFF04010A28720196
:103AE000FFFF04010A287201FFFF04010A28720186
:103AF000FFFF04010A287201FFFF04010A28720176
:103B0000FFFF0401AA287201FFFF0401AA28720125
:103B1000FFFF0401AA287201FFFF0401AA28720115
:103B2000FFFF04016A111E01FFFF0401BBF2100137
:103B3000FFFF0401BBF21901FFFF0401BBF21001FA
:103B4000FFFF04010A287201FFFF04010A28720125
:103B5000FFFF04010A287201FFFF04010A28720115
:103B6000FFFF04010A287201FFFF04010A28720105
:103B7000FFFF04010A287201FFFF04010A287201F5
:103B8000FFFF0401AA287201FFFF0401AA287201A5
:103B9000FFFF0401AA287201FFFF0401AA28720195
:103BA000FFFF04016A111E01FFFF0401BBF21001B7
:103BB000FFFF0401BBF21901FFFF0401BBF210017A
:103BC000FFFF04010A287201FFFF04010A287201A5
:103BD000FFFF04010A287201FFFF04010A28720195
:103BE000FFFF04010A287201FFFF04010A28720185
:103BF000FFFF04010A287201FFFF04010A28720175
:103C0000FFFF0401AA287201FFFF0401AA28720124
:103C1000FFFF0401AA287201FFFF0401AA28720114
:103C2000FFFF0401FE00FF01FFFF0401BBF21001D2
:103C3000FFFF0401BBF21901FFFF0401BBF21001F9
:103C4000FFFF04010A287201FFFF04010A28720124
:103C5000FFFF04010A287201FFFF04010A28720114
:103C6000FFFF04010A287201FFFF04010A28720104
:103C7000FFFF04010A287201FFFF04010A287201F4
:103C8000FFFF0401AA287201FFFF0401AA287201A4
:103C9000FFFF0401AA287201FFFF0401AA28720194
:103CA000FFFF0401FE00FF01FFFF0401BBF2100152
:103CB000FFFF0401BBF21901FFFF0401BBF2100179
:103CC000FFFF04010A287201FFFF04010A287201A4
:103CD000FFFF04010A287201FFFF04010A28720194
:103CE000FFFF04010A287201FFFF04010A28720184
:103CF000FFFF04010A287201FFFF04010A28720174
:103D0000FFFF0401AA287201FFFF0401AA28720123
:103D1000FFFF0401AA287201FFFF0401AA28720113
:103D2000FFFF04012B282001FFFF0401BBF210015B
:103D3000FFFF0401BBF21901FFFF0401BBF21001F8
:103D4000FFFF04010A287201FFFF04010A28720123
:103D5000FFFF04010A287201FFFF04010A28720113
:103D6000FFFF04010A287201FFFF04010A28720103
:103D7000FFFF04010A287201FFFF04010A287201F3
:103D8000FFFF0401AA287201FFFF0401AA287201A3
:103D9000FFFF0401AA287201FFFF0401AA28720193
:103DA000FFFF04012B282001FFFF0401BBF21001DB
:103DB000FFFF0401BBF21901FFFF0401BBF2100178
:103DC000FFFF04010A287201FFFF04010A287201A3
:103DD000FFFF04010A287201FFFF04010A28720193
:103DE000FFFF04010A287201FFFF04010A28720183
:103DF000FFFF04010A287201FFFF04010A28720173
:103E0000FFFF0401AA287201FFFF0401AA28720122
:103E1000FFFF0401AA287201FFFF0401AA28720112
:103E2000FFFF0401FE00FF01FFFF0401BBF21001D0
:103E3000FFFF0401BBF21901FFFF0401BBF21001F7
:103E4000FFFF04010A287201FFFF04010A28720122
:103E5000FFFF04010A287201FFFF04010A28720112
:103E6000FFFF04010A287201FFFF04010A28720102
:103E7000FFFF04010A287201FFFF04010A287201F2
:103E8000FFFF0401AA287201FFFF0401AA287201A2
:103E9000FFFF0401AA287201FFFF0401AA28720192
:103EA000FFFF0401FE00FF01FFFF0401BBF2100150
:103EB000FFFF0401BBF21901FFFF0401BBF2100177
:103EC000FFFF04010A287201FFFF04010A287201A2
:103ED000FFFF04010A287201FFFF04010A28720192
:103EE000FFFF04010A287201FFFF04010A28720182
:103EF000FFFF04010A287201FFFF04010A28720172
:103F0000FFFF0401AA287201FFFF0401AA28720121
:103F1000FFFF0401AA287201FFFF0401AA28720111
:103F2000FFFF04016A111E01FFFF0401BBF2100133
:103F3000FFFF0401BBF21901FFFF0401BBF21001F6
:103F4000FFFF04010A287201FFFF04010A28720121
:103F5000FFFF04010A287201FFFF04010A28720111
:103F6000FFFF04010A287201FFFF04010A28720101
:103F7000FFFF04010A287201FFFF04010A287201F1
:103F8000FFFF0401AA287201FFFF0401AA287201A1
:103F9000FFFF0401AA287201FFFF0401AA28720191
:103FA000FFFF04016A111E01FFFF0401BBF21001B3
:103FB000FFFF0401BBF21901FFFF0401BBF2100176
:103FC000FFFF04010A287201FFFF04010A287201A1
:103FD000FFFF04010A287201FFFF04010A28720191
:103FE000FFFF04010A287201FFFF04010A28720181
:103FF000FFFF04010A287201FFFF04010A28720171
:10400000FFFF0401AA287201FFFF0401AA28720120
:10401000FFFF0401AA287201FFFF0401AA28720110
:10402000FFFF0401FE00FF01FFFF0401BBF21001CE
:10403000FFFF0401BBF21901FFFF0401BBF21001F5
:10404000FFFF04010A287201FFFF04010A28720120
:10405000FFFF04010A287201FFFF04010A28720110
:10406000FFFF04010A287201FFFF04010A28720100
:10407000FFFF04010A287201FFFF04010A287201F0
:10408000FFFF0401AA287201FFFF0401AA287201A0
:10409000FFFF0401AA287201FFFF0401AA28720190
:1040A000FFFF0401FE00FF01FFFF0401BBF210014E
:1040B000FFFF0401BBF21901FFFF0401BBF2100175
:1040C000FFFF04010A287201FFFF04010A287201A0
:1040D000FFFF04010A287201FFFF04010A28720190
:1040E000FFFF04010A287201FFFF04010A28720180
:1040F000FFFF04010A287201FFFF04010A28720170
:10410000FFFF0401AA287201FFFF0401AA2872011F
:10411000FFFF0401AA287201FFFF0401AA2872010F
:10412000FFFF04015A111F01FFFF0401BBF2100140
:10413000FFFF0401BBF21901FFFF0401BBF21001F4
:10414000FFFF04010A287201FFFF04010A2872011F
:10415000FFFF04010A287201FFFF04010A2872010F
:10416000FFFF04010A287201FFFF04010A287201FF
:10417000FFFF04010A287201FFFF04010A287201EF
:10418000FFFF0401AA287201FFFF0401AA2872019F
:10419000FFFF0401AA287201FFFF0401AA2872018F
:1041A000FFFF04015A111F01FFFF0401BBF21001C0
:1041B000FFFF0401BBF21901FFFF0401BBF2100174
:1041C000FFFF04010A287201FFFF04010A2872019F
:1041D000FFFF04010A287201FFFF04010A2872018F
:1041E000FFFF04010A287201FFFF04010A2872017F
:1041F000FFFF04010A287201FFFF04010A2872016F
:10420000FFFF0401AA287201FFFF0401AA2872011E
:10421000FFFF0401AA287201FFFF0401AA2872010E
:10422000FFFF0401FE00FF01FFFF0401BBF21001CC
:10423000FFFF0401BBF21901FFFF0401BBF21001F3
:10424000FFFF04010A287201FFFF04010A2872011E
:10425000FFFF04010A287201FFFF04010A2872010E
:10426000FFFF04010A287201FFFF04010A287201FE
:10427000FFFF04010A287201FFFF04010A287201EE
:10428000FFFF0401AA287201FFFF0401AA2872019E
:10429000FFFF0401AA287201FFFF0401AA2872018E
:1042A000FFFF0401FE00FF01FFFF0401BBF210014C
:1042B000FFFF0401BBF21901FFFF0401BBF2100173
:1042C000FFFF04010A287201FFFF04010A2872019E
:1042D000FFFF04010A287201FFFF04010A2872018E
:1042E000FFFF04010A287201FFFF04010A2872017E
:1042F000FFFF04010A287201FFFF04010A2872016E
:10430000FFFF0401AA287201FFFF0401AA2872011D
:10431000FFFF0401AA287201FFFF0401AA2872010D
:10432000FFFF04016A111E01FFFF0401BBF210012F
:10433000FFFF0401BBF21901FFFF0401BBF21001F2
:10434000FFFF04010A287201FFFF04010A2872011D
:10435000FFFF04010A287201FFFF04010A2872010D
:10436000FFFF04010A287201FFFF04010A287201FD
:10437000FFFF04010A287201FFFF04010A287201ED
:10438000FFFF0401AA287201FFFF0401AA2872019D
:10439000FFFF0401AA287201FFFF0401AA2872018D
:1043A000FFFF04016A111E01FFFF0401BBF21001AF
:1043B000FFFF0401BBF21901FFFF0401BBF2100172
:1043C000FFFF04010A287201FFFF04010A2872019D
:1043D000FFFF04010A287201FFFF04010A2872018D
:1043E000FFFF04010A287201FFFF04010A2872017D
:1043F000FFFF04010A287201FFFF04010A2872016D
:10440000FFFF0401AA287201FFFF0401AA2872011C
:10441000FFFF0401AA287201FFFF0401AA2872010C
:10442000FFFF0401FE00FF01FFFF0401BBF21001CA
:10443000FFFF0401BBF21901FFFF0401BBF21001F1
:10444000FFFF04010A287201FFFF04010A2872011C
:10445000FFFF04010A287201FFFF04010A2872010C
:10446000FFFF04010A287201FFFF04010A287201FC
:10447000FFFF04010A287201FFFF04010A287201EC
:10448000FFFF0401AA287201FFFF0401AA2872019C
:10449000FFFF0401AA287201FFFF0401AA2872018C
:1044A000FFFF0401FE00FF01FFFF0401BBF210014A
:1044B000FFFF0401BBF21901FFFF0401BBF2100171
:1044C000FFFF04010A287201FFFF04010A2872019C
:1044D000FFFF04010A287201FFFF04010A2872018C
:1044E000FFFF04010A287201FFFF04010A2872017C
:1044F000FFFF04010A287201FFFF04010A2872016C
:10450000FFFF0401AA287201FFFF0401AA2872011B
:10451000FFFF0401AA287201FFFF0401AA2872010B
:10452000FFFF04012B282001FFFF0401BBF2100153
:10453000FFFF0401BBF21901FFFF0401BBF21001F0
:10454000FFFF04010A287201FFFF04010A2872011B
:10455000FFFF04010A287201FFFF04010A2872010B
:10456000FFFF04010A287201FFFF04010A287201FB
:10457000FFFF04010A287201FFFF04010A287201EB
:10458000FFFF0401AA287201FFFF0401AA2872019B
:10459000FFFF0401AA287201FFFF0401AA2872018B
:1045A000FFFF04012B282001FFFF0401BBF21001D3
:1045B000FFFF0401BBF21901FFFF0401BBF2100170
:1045C000FFFF04010A287201FFFF04010A2872019B
:1045D000FFFF04010A287201FFFF04010A2872018B
:1045E000FFFF04010A287201FFFF04010A2872017B
:1045F000FFFF04010A287201FFFF04010A2872016B
:10460000FFFF0401AA287201FFFF0401AA2872011A
:10461000FFFF0401AA287201FFFF0401AA2872010A
:10462000FFFF0401FE00FF01FFFF0401BBF21001C8
:10463000FFFF0401BBF21901FFFF0401BBF21001EF
:10464000FFFF04010A287201FFFF04010A2872011A
:10465000FFFF04010A287201FFFF04010A2872010A
:10466000FFFF04010A287201FFFF04010A287201FA
:10467000FFFF04010A287201FFFF04010A287201EA
:10468000FFFF0401AA287201FFFF0401AA2872019A
:10469000FFFF0401AA287201FFFF0401AA2872018A
:1046A000FFFF0401FE00FF01FFFF0401BBF2100148
:1046B000FFFF0401BBF21901FFFF0401BBF210016F
:1046C000FFFF04010A287201FFFF04010A2872019A
:1046D000FFFF04010A287201FFFF04010A2872018A
:1046E000FFFF04010A287201FFFF04010A2872017A
:1046F000FFFF04010A287201FFFF04010A2872016A
:10470000FFFF0401AA287201FFFF0401AA28720119
:10471000FFFF0401AA287201FFFF0401AA28720109
:10472000FFFF04016A111E01FFFF0401BBF210012B
:10473000FFFF0401BBF21901FFFF0401BBF21001EE
:10474000FFFF04010A287201FFFF04010A28720119
:10475000FFFF04010A287201FFFF04010A28720109
:10476000FFFF04010A287201FFFF04010A287201F9
:10477000FFFF04010A287201FFFF04010A287201E9
:10478000FFFF0401AA287201FFFF0401AA28720199
:10479000FFFF0401AA287201FFFF0401AA28720189
:1047A000FFFF04016A111E01FFFF0401BBF21001AB
:1047B000FFFF0401BBF21901FFFF0401BBF210016E
:1047C000FFFF04010A287201FFFF04010A28720199
:1047D000FFFF04010A287201FFFF04010A28720189
:1047E000FFFF04010A287201FFFF04010A28720179
:1047F000FFFF04010A287201FFFF04010A28720169
:10480000FFFF0401AA287201FFFF0401AA28720118
:10481000FFFF0401AA287201FFFF0401AA28720108
:10482000FFFF0401FE00FF01FFFF0401BBF21001C6
:10483000FFFF0401BBF21901FFFF0401BBF21001ED
:10484000FFFF04010A287201FFFF04010A28720118
:10485000FFFF04010A287201FFFF04010A28720108
:10486000FFFF04010A287201FFFF04010A287201F8
:10487000FFFF04010A287201FFFF04010A287201E8
:10488000FFFF0401AA287201FFFF0401AA28720198
:10489000FFFF0401AA287201FFFF0401AA28720188
:1048A000FFFF0401FE00FF01FFFF0401BBF2100146
:1048B000FFFF0401BBF21901FFFF0401BBF210016D
:1048C000FFFF04010A287201FFFF04010A28720198
:1048D000FFFF04010A287201FFFF04010A28720188
:1048E000FFFF04010A287201FFFF04010A28720178
:1048F000FFFF04010A287201FFFF04010A28720168
:10490000FFFF0401AA287201FFFF0401AA28720117
:10491000FFFF0401AA287201FFFF0401AA28720107
:10492000FFFF04015A111F01FFFF0401BBF2100138
:10493000FFFF0401BBF21901FFFF0401BBF21001EC
:10494000FFFF04010A287201FFFF04010A28720117
:10495000FFFF04010A287201FFFF04010A28720107
:10496000FFFF04010A287201FFFF04010A287201F7
:10497000FFFF04010A287201FFFF04010A287201E7
:10498000FFFF0401AA287201FFFF0401AA28720197
:10499000FFFF0401AA287201FFFF0401AA28720187
:1049A000FFFF04015A111F01FFFF0401BBF21001B8
:1049B000FFFF0401BBF21901FFFF0401BBF210016C
:1049C000FFFF04010A287201FFFF04010A28720197
:1049D000FFFF04010A287201FFFF04010A28720187
:1049E000FFFF04010A287201FFFF04010A28720177
:1049F000FFFF04010A287201FFFF04010A28720167
:104A0000FFFF0401AA287201FFFF0401AA28720116
:104A1000FFFF0401AA287201FFFF0401AA28720106
:104A2000FFFF0401FE00FF01FFFF0401BBF21001C4
:104A3000FFFF0401BBF21901FFFF0401BBF21001EB
:104A4000FFFF04010A287201FFFF04010A28720116
:104A5000FFFF04010A287201FFFF04010A28720106
:104A6000FFFF04010A287201FFFF04010A287201F6
:104A7000FFFF04010A287201FFFF04010A287201E6
:104A8000FFFF0401AA287201FFFF0401AA28720196
:104A9000FFFF0401AA287201FFFF0401AA28720186
:104AA000FFFF0401FE00FF01FFFF0401BBF2100144
:104AB000FFFF0401BBF21901FFFF0401BBF210016B
:104AC000FFFF04010A287201FFFF04010A28720196
:104AD000FFFF04010A287201FFFF04010A28720186
:104AE000FFFF04010A287201FFFF04010A28720176
:104AF000FFFF04010A287201FFFF04010A28720166
:104B0000FFFF0401AA287201FFFF0401AA28720115
:104B1000FFFF0401AA287201FFFF0401AA28720105
:104B2000FFFF04016A111E01FFFF0401BBF2100127
:104B3000FFFF0401BBF21901FFFF0401BBF21001EA
:104B4000FFFF04010A287201FFFF04010A28720115
:104B5000FFFF04010A287201FFFF04010A28720105
:104B6000FFFF04010A287201FFFF04010A287201F5
:104B7000FFFF04010A287201FFFF04010A287201E5
:104B8000FFFF0401AA287201FFFF0401AA28720195
:104B9000FFFF0401AA287201FFFF0401AA28720185
:104BA000FFFF04016A111E01FFFF0401BBF21001A7
:104BB000FFFF0401BBF21901FFFF0401BBF210016A
:104BC000FFFF04010A287201FFFF04010A28720195
:104BD000FFFF04010A287201FFFF04010A28720185
:104BE000FFFF04010A287201FFFF04010A28720175
:104BF000FFFF04010A287201FFFF04010A28720165
:104C0000FFFF0401AA287201FFFF0401AA28720114
:104C1000FFFF0401AA287201FFFF0401AA28720104
:104C2000FFFF0401FE00FF01FFFF0401BBF21001C2
:104C3000FFFF0401BBF21901FFFF0401BBF21001E9
:104C4000FFFF04010A287201FFFF04010A28720114
:104C5000FFFF04010A287201FFFF04010A28720104
:104C6000FFFF04010A287201FFFF04010A287201F4
:104C7000FFFF04010A287201FFFF04010A287201E4
:104C8000FFFF0401AA287201FFFF0401AA28720194
:104C9000FFFF0401AA287201FFFF0401AA28720184
:104CA000FFFF0401FE00FF01FFFF0401BBF2100142
:104CB000FFFF0401BBF21901FFFF0401BBF2100169
:104CC000FFFF04010A287201FFFF04010A28720194
:104CD000FFFF04010A287201FFFF04010A28720184
:104CE000FFFF04010A287201FFFF04010A28720174
:104CF000FFFF04010A287201FFFF04010A28720164
:104D0000FFFF0401AA287201FFFF0401AA28720113
:104D1000FFFF0401AA287201FFFF0401AA28720103
:104D2000FFFF04012B282001FFFF0401BBF210014B
:104D3000FFFF0401BBF21901FFFF0401BBF21001E8
:104D4000FFFF04010A287201FFFF04010A28720113
:104D5000FFFF04010A287201FFFF04010A28720103
:104D6000FFFF04010A287201FFFF04010A287201F3
:104D7000FFFF04010A287201FFFF04010A287201E3
:104D8000FFFF0401AA287201FFFF0401AA28720193
:104D9000FFFF0401AA287201FFFF0401AA28720183
:104DA000FFFF04012B282001FFFF0401BBF21001CB
:104DB000FFFF0401BBF21901FFFF0401BBF2100168
:104DC000FFFF04010A287201FFFF04010A28720193
:104DD000FFFF04010A287201FFFF04010A28720183
:104DE000FFFF04010A287201FFFF04010A28720173
:104DF000FFFF04010A287201FFFF04010A28720163
:104E0000FFFF0401AA287201FFFF0401AA28720112
:104E1000FFFF0401AA287201FFFF0401AA28720102
:104E2000FFFF0401FE00FF01FFFF0401BBF21001C0
:104E3000FFFF0401BBF21901FFFF0401BBF21001E7
:104E4000FFFF04010A287201FFFF04010A28720112
:104E5000FFFF04010A287201FFFF04010A28720102
:104E6000FFFF04010A287201FFFF04010A287201F2
:104E7000FFFF04010A287201FFFF04010A287201E2
:104E8000FFFF0401AA287201FFFF0401AA28720192
:104E9000FFFF0401AA287201FFFF0401AA28720182
:104EA000FFFF0401FE00FF01FFFF0401BBF2100140
:104EB000FFFF0401BBF21901FFFF0401BBF2100167
:104EC000FFFF04010A287201FFFF04010A28720192
:104ED000FFFF04010A287201FFFF04010A28720182
:104EE000FFFF04010A287201FFFF04010A28720172
:104EF000FFFF04010A287201FFFF04010A28720162
:104F0000FFFF0401AA287201FFFF0401AA28720111
:104F1000FFFF0401AA287201FFFF0401AA28720101
:104F2000FFFF04016A111E01FFFF0401BBF2100123
:104F3000FFFF0401BBF21901FFFF0401BBF21001E6
:104F4000FFFF04010A287201FFFF04010A28720111
:104F5000FFFF04010A287201FFFF04010A28720101
:104F6000FFFF04010A287201FFFF04010A287201F1
:104F7000FFFF04010A287201FFFF04010A287201E1
:104F8000FFFF0401AA287201FFFF0401AA28720191
:104F9000FFFF0401AA287201FFFF0401AA28720181
:104FA000FFFF04016A111E01FFFF0401BBF21001A3
:104FB000FFFF0401BBF21901FFFF0401BBF2100166
:104FC000FFFF04010A287201FFFF04010A28720191
:104FD000FFFF04010A287201FFFF04010A28720181
:104FE000FFFF04010A287201FFFF04010A28720171
:104FF000FFFF04010A287201FFFF04010A28720161
:10500000FFFF0401AA287201FFFF0401AA28720110
:10501000FFFF0401AA287201FFFF0401AA28720100
:10502000FFFF0401FE00FF01FFFF0401BBF21001BE
:10503000FFFF0401BBF21901FFFF0401BBF21001E5
:10504000FFFF04010A287201FFFF04010A28720110
:10505000FFFF04010A287201FFFF04010A28720100
:10506000FFFF04010A287201FFFF04010A287201F0
:10507000FFFF04010A287201FFFF04010A287201E0
:10508000FFFF0401AA287201FFFF0401AA28720190
:10509000FFFF0401AA287201FFFF0401AA28720180
:1050A000FFFF0401FE00FF01FFFF0401BBF210013E
:1050B000FFFF0401BBF21901FFFF0401BBF2100165
:1050C000FFFF04010A287201FFFF04010A28720190
:1050D000FFFF04010A287201FFFF04010A28720180
:1050E000FFFF04010A287201FFFF04010A28720170
:1050F000FFFF04010A287201FFFF04010A28720160
:10510000FFFF0401AA287201FFFF0401AA2872010F
:10511000FFFF0401AA287201FFFF0401AA287201FF
:10512000FFFF04015A111F01FFFF0401BBF2100130
:10513000FFFF0401BBF21901FFFF0401BBF21001E4
:10514000FFFF04010A287201FFFF04010A2872010F
:10515000FFFF04010A287201FFFF04010A287201FF
:10516000FFFF04010A287201FFFF04010A287201EF
:10517000FFFF04010A287201FFFF04010A287201DF
:10518000FFFF0401AA287201FFFF0401AA2872018F
:10519000FFFF0401AA287201FFFF0401AA2872017F
:1051A000FFFF04015A111F01FFFF0401BBF21001B0
:1051B000FFFF0401BBF21901FFFF0401BBF2100164
:1051C000FFFF04010A287201FFFF04010A2872018F
:1051D000FFFF04010A287201FFFF04010A2872017F
:1051E000FFFF04010A287201FFFF04010A2872016F
:1051F000FFFF04010A287201FFFF04010A2872015F
:10520000FFFF0401AA287201FFFF0401AA2872010E
:10521000FFFF0401AA287201FFFF0401AA287201FE
:10522000FFFF0401FE00FF01FFFF0401BBF21001BC
:10523000FFFF0401BBF21901FFFF0401BBF21001E3
:10524000FFFF04010A287201FFFF04010A2872010E
:10525000FFFF04010A287201FFFF04010A287201FE
:10526000FFFF04010A287201FFFF04010A287201EE
:10527000FFFF04010A287201FFFF04010A287201DE
:10528000FFFF0401AA287201FFFF0401AA2872018E
:10529000FFFF0401AA287201FFFF0401AA2872017E
:1052A000FFFF0401FE00FF01FFFF0401BBF210013C
:1052B000FFFF0401BBF21901FFFF0401BBF2100163
:1052C000FFFF04010A287201FFFF04010A2872018E
:1052D000FFFF04010A287201FFFF04010A2872017E
:1052E000FFFF04010A287201FFFF04010A2872016E
:1052F000FFFF04010A287201FFFF04010A2872015E
:10530000FFFF0401AA287201FFFF0401AA2872010D
:10531000FFFF0401AA287201FFFF0401AA287201FD
:10532000FFFF04016A111E01FFFF0401BBF210011F
:10533000FFFF0401BBF21901FFFF0401BBF21001E2
:10534000FFFF04010A287201FFFF04010A2872010D
:10535000FFFF04010A287201FFFF04010A287201FD
:10536000FFFF04010A287201FFFF04010A287201ED
:10537000FFFF04010A287201FFFF04010A287201DD
:10538000FFFF0401AA287201FFFF0401AA2872018D
:10539000FFFF0401AA287201FFFF0401AA2872017D
:1053A000FFFF04016A111E01FFFF0401BBF210019F
:1053B000FFFF0401BBF21901FFFF0401BBF2100162
:1053C000FFFF04010A287201FFFF04010A2872018D
:1053D000FFFF04010A287201FFFF04010A2872017D
:1053E000FFFF04010A287201FFFF04010A2872016D
:1053F000FFFF04010A287201FFFF04010A2872015D
:10540000FFFF0401AA287201FFFF0401AA2872010C
:10541000FFFF0401AA287201FFFF0401AA287201FC
:10542000FFFF0401FE00FF01FFFF0401BBF21001BA
:10543000FFFF0401BBF21901FFFF0401BBF21001E1
:10544000FFFF04010A287201FFFF04010A2872010C
:10545000FFFF04010A287201FFFF04010A287201FC
:10546000FFFF04010A287201FFFF04010A287201EC
:10547000FFFF04010A287201FFFF04010A287201DC
:10548000FFFF0401AA287201FFFF0401AA2872018C
:10549000FFFF0401AA287201FFFF0401AA2872017C
:1054A000FFFF0401FE00FF01FFFF0401BBF210013A
:1054B000FFFF0401BBF21901FFFF0401BBF2100161
:1054C000FFFF04010A287201FFFF04010A2872018C
:1054D000FFFF04010A287201FFFF04010A2872017C
:1054E000FFFF04010A287201FFFF04010A2872016C
:1054F000FFFF04010A287201FFFF04010A2872015C
:10550000FFFF0401AA287201FFFF0401AA2872010B
:10551000FFFF0401AA287201FFFF0401AA287201FB
:10552000FFFF04012B282001FFFF0401BBF2100143
:10553000FFFF0401BBF21901FFFF0401BBF21001E0
:10554000FFFF04010A287201FFFF04010A2872010B
:10555000FFFF04010A287201FFFF04010A287201FB
:10556000FFFF04010A287201FFFF04010A287201EB
:10557000FFFF04010A287201FFFF04010A287201DB
:10558000FFFF0401AA287201FFFF0401AA2872018B
:10559000FFFF0401AA287201FFFF0401AA2872017B
:1055A000FFFF04012B282001FFFF0401BBF21001C3
:1055B000FFFF0401BBF21901FFFF0401BBF2100160
:1055C000FFFF04010A287201FFFF04010A2872018B
:1055D000FFFF04010A287201FFFF04010A2872017B
:1055E000FFFF04010A287201FFFF04010A2872016B
:1055F000FFFF04010A287201FFFF04010A2872015B
:10560000FFFF0401AA287201FFFF0401AA2872010A
:10561000FFFF0401AA287201FFFF0401AA287201FA
:10562000FFFF0401FE00FF01FFFF0401BBF21001B8
:10563000FFFF0401BBF21901FFFF0401BBF21001DF
:10564000FFFF04010A287201FFFF04010A2872010A
:10565000FFFF04010A287201FFFF04010A287201FA
:10566000FFFF04010A287201FFFF04010A287201EA
:10567000FFFF04010A287201FFFF04010A287201DA
:10568000FFFF0401AA287201FFFF0401AA2872018A
:10569000FFFF0401AA287201FFFF0401AA2872017A
:1056A000FFFF0401FE00FF01FFFF0401BBF2100138
:1056B000FFFF0401BBF21901FFFF0401BBF210015F
:1056C000FFFF04010A287201FFFF04010A2872018A
:1056D000FFFF04010A287201FFFF04010A2872017A
:1056E000FFFF04010A287201FFFF04010A2872016A
:1056F000FFFF04010A287201FFFF04010A2872015A
:10570000FFFF0401AA287201FFFF0401AA28720109
:10571000FFFF0401AA287201FFFF0401AA287201F9
:10572000FFFF04016A111E01FFFF0401BBF210011B
:10573000FFFF0401BBF21901FFFF0401BBF21001DE
:10574000FFFF04010A287201FFFF04010A28720109
:10575000FFFF04010A287201FFFF04010A287201F9
:10576000FFFF04010A287201FFFF04010A287201E9
:10577000FFFF04010A287201FFFF04010A287201D9
:10578000FFFF0401AA287201FFFF0401AA28720189
:10579000FFFF0401AA287201FFFF0401AA28720179
:1057A000FFFF04016A111E01FFFF0401BBF210019B
:1057B000FFFF0401BBF21901FFFF0401BBF210015E
:1057C000FFFF04010A287201FFFF04010A28720189
:1057D000FFFF04010A287201FFFF04010A28720179
:1057E000FFFF04010A287201FFFF04010A28720169
:1057F000FFFF04010A287201FFFF04010A28720159
:10580000FFFF0401AA287201FFFF0401AA28720108
:10581000FFFF0401AA287201FFFF0401AA287201F8
:10582000FFFF0401FE00FF01FFFF0401BBF21001B6
:10583000FFFF0401BBF21901FFFF0401BBF21001DD
:10584000FFFF04010A287201FFFF04010A28720108
:10585000FFFF04010A287201FFFF04010A287201F8
:10586000FFFF04010A287201FFFF04010A287201E8
:10587000FFFF04010A287201FFFF04010A287201D8
:10588000FFFF0401AA287201FFFF0401AA28720188
:10589000FFFF0401AA287201FFFF0401AA28720178
:1058A000FFFF0401FE00FF01FFFF0401BBF2100136
:1058B000FFFF0401BBF21901FFFF0401BBF210015D
:1058C000FFFF04010A287201FFFF04010A28720188
:1058D000FFFF04010A287201FFFF04010A28720178
:1058E000FFFF04010A287201FFFF04010A28720168
:1058F000FFFF04010A287201FFFF04010A28720158
:10590000FFFF0401AA287201FFFF0401AA28720107
:10591000FFFF0401AA287201FFFF0401AA287201F7
:10592000FFFF04015A111F01FFFF0401BBF2100128
:10593000FFFF0401BBF21901FFFF0401BBF21001DC
:10594000FFFF04010A287201FFFF04010A28720107
:10595000FFFF04010A287201FFFF04010A287201F7
:10596000FFFF04010A287201FFFF04010A287201E7
:10597000FFFF04010A287201FFFF04010A287201D7
:10598000FFFF0401AA287201FFFF0401AA28720187
:10599000FFFF0401AA287201FFFF0401AA28720177
:1059A000FFFF04015A111F01FFFF0401BBF21001A8
:1059B000FFFF0401BBF21901FFFF0401BBF210015C
:1059C000FFFF04010A287201FFFF04010A28720187
:1059D000FFFF04010A287201FFFF04010A28720177
:1059E000FFFF04010A287201FFFF04010A28720167
:1059F000FFFF04010A287201FFFF04010A28720157
:105A0000FFFF0401AA287201FFFF0401AA28720106
:105A1000FFFF0401AA287201FFFF0401AA287201F6
:105A2000FFFF0401FE00FF01FFFF0401BBF21001B4
:105A3000FFFF0401BBF21901FFFF0401BBF21001DB
:105A4000FFFF04010A287201FFFF04010A28720106
:105A5000FFFF04010A287201FFFF04010A287201F6
:105A6000FFFF04010A287201FFFF04010A287201E6
:105A7000FFFF04010A287201FFFF04010A287201D6
:105A8000FFFF0401AA287201FFFF0401AA28720186
:105A9000FFFF0401AA287201FFFF0401AA28720176
:105AA000FFFF0401FE00FF01FFFF0401BBF2100134
:105AB000FFFF0401BBF21901FFFF0401BBF210015B
:105AC000FFFF04010A287201FFFF04010A28720186
:105AD000FFFF04010A287201FFFF04010A28720176
:105AE000FFFF04010A287201FFFF04010A28720166
:105AF000FFFF04010A287201FFFF04010A28720156
:105B0000FFFF0401AA287201FFFF0401AA28720105
:105B1000FFFF0401AA287201FFFF0401AA287201F5
:105B2000FFFF04016A111E01FFFF0401BBF2100117
:105B3000FFFF0401BBF21901FFFF0401BBF21001DA
:105B4000FFFF04010A287201FFFF04010A28720105
:105B5000FFFF04010A287201FFFF04010A287201F5
:105B6000FFFF04010A287201FFFF04010A287201E5
:105B7000FFFF04010A287201FFFF04010A287201D5
:105B8000FFFF0401AA287201FFFF0401AA28720185
:105B9000FFFF0401AA287201FFFF0401AA28720175
:105BA000FFFF04016A111E01FFFF0401BBF2100197
:105BB000FFFF0401BBF21901FFFF0401BBF210015A
:105BC000FFFF04010A287201FFFF04010A28720185
:105BD000FFFF04010A287201FFFF04010A28720175
:105BE000FFFF04010A287201FFFF04010A28720165
:105BF000FFFF04010A287201FFFF04010A28720155
:105C0000FFFF0401AA287201FFFF0401AA28720104
:105C1000FFFF0401AA287201FFFF0401AA287201F4
:105C2000FFFF0401FE00FF01FFFF0401BBF21001B2
:105C3000FFFF0401BBF21901FFFF0401BBF21001D9
:105C4000FFFF04010A287201FFFF04010A28720104
:105C5000FFFF04010A287201FFFF04010A287201F4
:105C6000FFFF04010A287201FFFF04010A287201E4
:105C7000FFFF04010A287201FFFF04010A287201D4
:105C8000FFFF0401AA287201FFFF0401AA28720184
:105C9000FFFF0401AA287201FFFF0401AA28720174
:105CA000FFFF0401FE00FF01FFFF0401BBF2100132
:105CB000FFFF0401BBF21901FFFF0401BBF2100159
:105CC000FFFF04010A287201FFFF04010A28720184
:105CD000FFFF04010A287201FFFF04010A28720174
:105CE000FFFF04010A287201FFFF04010A28720164
:105CF000FFFF04010A287201FFFF04010A28720154
:105D0000FFFF0401AA287201FFFF0401AA28720103
:105D1000FFFF0401AA287201FFFF0401AA287201F3
:105D2000FFFF04012B282001FFFF0401BBF210013B
:105D3000FFFF0401BBF21901FFFF0401BBF21001D8
:105D4000FFFF04010A287201FFFF04010A28720103
:105D5000FFFF04010A287201FFFF04010A287201F3
:105D6000FFFF04010A287201FFFF04010A287201E3
:105D7000FFFF04010A287201FFFF04010A287201D3
:105D8000FFFF0401AA287201FFFF0401AA28720183
:105D9000FFFF0401AA287201FFFF0401AA28720173
:105DA000FFFF04012B282001FFFF0401BBF21001BB
:105DB000FFFF0401BBF21901FFFF0401BBF2100158
:105DC000FFFF04010A287201FFFF04010A28720183
:105DD000FFFF04010A287201FFFF04010A28720173
:105DE000FFFF04010A287201FFFF04010A28720163
:105DF000FFFF04010A287201FFFF04010A28720153
:105E0000FFFF0401AA287201FFFF0401AA28720102
:105E1000FFFF0401AA287201FFFF0401AA287201F2
:105E2000FFFF0401FE00FF01FFFF0401BBF21001B0
:105E3000FFFF0401BBF21901FFFF0401BBF21001D7
:105E4000FFFF04010A287201FFFF04010A28720102
:105E5000FFFF04010A287201FFFF04010A287201F2
:105E6000FFFF04010A287201FFFF04010A287201E2
:105E7000FFFF04010A287201FFFF04010A287201D2
:105E8000FFFF0401AA287201FFFF0401AA28720182
:105E9000FFFF0401AA287201FFFF0401AA28720172
:105EA000FFFF0401FE00FF01FFFF0401BBF2100130
:105EB000FFFF0401BBF21901FFFF0401BBF2100157
:105EC000FFFF04010A287201FFFF04010A28720182
:105ED000FFFF04010A287201FFFF04010A28720172
:105EE000FFFF04010A287201FFFF04010A28720162
:105EF000FFFF04010A287201FFFF04010A28720152
:105F0000FFFF0401AA287201FFFF0401AA28720101
:105F1000FFFF0401AA287201FFFF0401AA287201F1
:105F2000FFFF04016A111E01FFFF0401BBF2100113
:105F3000FFFF0401BBF21901FFFF0401BBF21001D6
:105F4000FFFF04010A287201FFFF04010A28720101
:105F5000FFFF04010A287201FFFF04010A287201F1
:105F6000FFFF04010A287201FFFF04010A287201E1
:105F7000FFFF04010A287201FFFF04010A287201D1
:105F8000FFFF0401AA287201FFFF0401AA28720181
:105F9000FFFF0401AA287201FFFF0401AA28720171
:105FA000FFFF04016A111E01FFFF0401BBF2100193
:105FB000FFFF0401BBF21901FFFF0401BBF2100156
:105FC000FFFF04010A287201FFFF04010A28720181
:105FD000FFFF04010A287201FFFF04010A28720171
:105FE000FFFF04010A287201FFFF04010A28720161
:105FF000FFFF04010A287201FFFF04010A28720151
:10600000FFFF0401AA287201FFFF0401AA28720100
:10601000FFFF0401AA287201FFFF0401AA287201F0
:10602000FFFF0401FE00FF01FFFF0401BBF21001AE
:10603000FFFF0401BBF21901FFFF0401BBF21001D5
:10604000FFFF04010A287201FFFF04010A28720100
:10605000FFFF04010A287201FFFF04010A287201F0
:10606000FFFF04010A287201FFFF04010A287201E0
:10607000FFFF04010A287201FFFF04010A287201D0
:10608000FFFF0401AA287201FFFF0401AA28720180
:10609000FFFF0401AA287201FFFF0401AA28720170
:1060A000FFFF0401FE00FF01FFFF0401BBF210012E
:1060B000FFFF0401BBF21901FFFF0401BBF2100155
:1060C000FFFF04010A287201FFFF04010A28720180
:1060D000FFFF04010A287201FFFF04010A28720170
:1060E000FFFF04010A287201FFFF04010A28720160
:1060F000FFFF04010A287201FFFF04010A28720150
:10610000FFFF0401AA287201FFFF0401AA287201FF
:10611000FFFF0401AA287201FFFF0401AA287201EF
:10612000FFFF04015A111F01FFFF0401BBF2100120
:10613000FFFF0401BBF21901FFFF0401BBF21001D4
:10614000FFFF04010A287201FFFF04010A287201FF
:10615000FFFF04010A287201FFFF04010A287201EF
:10616000FFFF04010A287201FFFF04010A287201DF
:10617000FFFF04010A287201FFFF04010A287201CF
:10618000FFFF0401AA287201FFFF0401AA2872017F
:10619000FFFF0401AA287201FFFF0401AA2872016F
:1061A000FFFF04015A111F01FFFF0401BBF21001A0
:1061B000FFFF0401BBF21901FFFF0401BBF2100154
:1061C000FFFF04010A287201FFFF04010A2872017F
:1061D000FFFF04010A287201FFFF04010A2872016F
:1061E000FFFF04010A287201FFFF04010A2872015F
:1061F000FFFF04010A287201FFFF04010A2872014F
:10620000FFFF0401AA287201FFFF0401AA287201FE
:10621000FFFF0401AA287201FFFF0401AA287201EE
:10622000FFFF0401FE00FF01FFFF0401BBF21001AC
:10623000FFFF0401BBF21901FFFF0401BBF21001D3
:10624000FFFF04010A287201FFFF04010A287201FE
:10625000FFFF04010A287201FFFF04010A287201EE
:10626000FFFF04010A287201FFFF04010A287201DE
:10627000FFFF04010A287201FFFF04010A287201CE
:10628000FFFF0401AA287201FFFF0401AA2872017E
:10629000FFFF0401AA287201FFFF0401AA2872016E
:1062A000FFFF0401FE00FF01FFFF0401BBF210012C
:1062B000FFFF0401BBF21901FFFF0401BBF2100153
:1062C000FFFF04010A287201FFFF04010A2872017E
:1062D000FFFF04010A287201FFFF04010A2872016E
:1062E000FFFF04010A287201FFFF04010A2872015E
:1062F000FFFF04010A287201FFFF04010A2872014E
:10630000FFFF0401AA287201FFFF0401AA287201FD
:10631000FFFF0401AA287201FFFF0401AA287201ED
:10632000FFFF04016A111E01FFFF0401BBF210010F
:10633000FFFF0401BBF21901FFFF0401BBF21001D2
:10634000FFFF04010A287201FFFF04010A287201FD
:10635000FFFF04010A287201FFFF04010A287201ED
:10636000FFFF04010A287201FFFF04010A287201DD
:10637000FFFF04010A287201FFFF04010A287201CD
:10638000FFFF0401AA287201FFFF0401AA2872017D
:10639000FFFF0401AA287201FFFF0401AA2872016D
:1063A000FFFF04016A111E01FFFF0401BBF210018F
:1063B000FFFF0401BBF21901FFFF0401BBF2100152
:1063C000FFFF04010A287201FFFF04010A2872017D
:1063D000FFFF04010A287201FFFF04010A2872016D
:1063E000FFFF04010A287201FFFF04010A2872015D
:1063F000FFFF04010A287201FFFF04010A2872014D
:10640000FFFF0401AA287201FFFF0401AA287201FC
:10641000FFFF0401AA287201FFFF0401AA287201EC
:10642000FFFF0401FE00FF01FFFF0401BBF21001AA
:10643000FFFF0401BBF21901FFFF0401BBF21001D1
:10644000FFFF04010A287201FFFF04010A287201FC
:10645000FFFF04010A287201FFFF04010A287201EC
:10646000FFFF04010A287201FFFF04010A287201DC
:10647000FFFF04010A287201FFFF04010A287201CC
:10648000FFFF0401AA287201FFFF0401AA2872017C
:10649000FFFF0401AA287201FFFF0401AA2872016C
:1064A000FFFF0401FE00FF01FFFF0401BBF210012A
:1064B000FFFF0401BBF21901FFFF0401BBF2100151
:1064C000FFFF04010A287201FFFF04010A2872017C
:1064D000FFFF04010A287201FFFF04010A2872016C
:1064E000FFFF04010A287201FFFF04010A2872015C
:1064F000FFFF04010A287201FFFF04010A2872014C
:10650000FFFF0401AA287201FFFF0401AA287201FB
:10651000FFFF0401AA287201FFFF0401AA287201EB
:10652000FFFF04012B282001FFFF0401BBF2100133
:10653000FFFF0401BBF21901FFFF0401BBF21001D0
:10654000FFFF04010A287201FFFF04010A287201FB
:10655000FFFF04010A287201FFFF04010A287201EB
:10656000FFFF04010A287201FFFF04010A287201DB
:10657000FFFF04010A287201FFFF04010A287201CB
:10658000FFFF0401AA287201FFFF0401AA2872017B
:10659000FFFF0401AA287201FFFF0401AA2872016B
:1065A000FFFF04012B282001FFFF0401BBF21001B3
:1065B000FFFF0401BBF21901FFFF0401BBF2100150
:1065C000FFFF04010A287201FFFF04010A2872017B
:1065D000FFFF04010A287201FFFF04010A2872016B
:1065E000FFFF04010A287201FFFF04010A2872015B
:1065F000FFFF04010A287201FFFF04010A2872014B
:10660000FFFF0401AA287201FFFF0401AA287201FA
:10661000FFFF0401AA287201FFFF0401AA287201EA
:10662000FFFF0401FE00FF01FFFF0401BBF21001A8
:10663000FFFF0401BBF21901FFFF0401BBF21001CF
:10664000FFFF04010A287201FFFF04010A287201FA
:10665000FFFF04010A287201FFFF04010A287201EA
:10666000FFFF04010A287201FFFF04010A287201DA
:10667000FFFF04010A287201FFFF04010A287201CA
:10668000FFFF0401AA287201FFFF0401AA2872017A
:10669000FFFF0401AA287201FFFF0401AA2872016A
:1066A000FFFF0401FE00FF01FFFF0401BBF2100128
:1066B000FFFF0401BBF21901FFFF0401BBF210014F
:1066C000FFFF04010A287201FFFF04010A2872017A
:1066D000FFFF04010A287201FFFF04010A2872016A
:1066E000FFFF04010A287201FFFF04010A2872015A
:1066F000FFFF04010A287201FFFF04010A2872014A
:10670000FFFF0401AA287201FFFF0401AA287201F9
:10671000FFFF0401AA287201FFFF0401AA287201E9
:10672000FFFF04016A111E01FFFF0401BBF210010B
:10673000FFFF0401BBF21901FFFF0401BBF21001CE
:10674000FFFF04010A287201FFFF04010A287201F9
:10675000FFFF04010A287201FFFF04010A287201E9
:10676000FFFF04010A287201FFFF04010A287201D9
:10677000FFFF04010A287201FFFF04010A287201C9
:10678000FFFF0401AA287201FFFF0401AA28720179
:10679000FFFF0401AA287201FFFF0401AA28720169
:1067A000FFFF04016A111E01FFFF0401BBF210018B
:1067B000FFFF0401BBF21901FFFF0401BBF210014E
:1067C000FFFF04010A287201FFFF04010A28720179
:1067D000FFFF04010A287201FFFF04010A28720169
:1067E000FFFF04010A287201FFFF04010A28720159
:1067F000FFFF04010A287201FFFF04010A28720149
:10680000FFFF0401AA287201FFFF0401AA287201F8
:10681000FFFF0401AA287201FFFF0401AA287201E8
:10682000FFFF0401FE00FF01FFFF0401BBF21001A6
:10683000FFFF0401BBF21901FFFF0401BBF21001CD
:10684000FFFF04010A287201FFFF04010A287201F8
:10685000FFFF04010A287201FFFF04010A287201E8
:10686000FFFF04010A287201FFFF04010A287201D8
:10687000FFFF04010A287201FFFF04010A287201C8
:10688000FFFF0401AA287201FFFF0401AA28720178
:10689000FFFF0401AA287201FFFF0401AA28720168
:1068A000FFFF0401FE00FF01FFFF0401BBF2100126
:1068B000FFFF0401BBF21901FFFF0401BBF210014D
:1068C000FFFF04010A287201FFFF04010A28720178
:1068D000FFFF04010A287201FFFF04010A28720168
:1068E000FFFF04010A287201FFFF04010A28720158
:1068F000FFFF04010A287201FFFF04010A28720148
:10690000FFFF0401AA287201FFFF0401AA287201F7
:10691000FFFF0401AA287201FFFF0401AA287201E7
:10692000FFFF04015A111F01FFFF0401BBF2100118
:10693000FFFF0401BBF21901FFFF0401BBF21001CC
:10694000FFFF04010A287201FFFF04010A287201F7
:10695000FFFF04010A287201FFFF04010A287201E7
:10696000FFFF04010A287201FFFF04010A287201D7
:10697000FFFF04010A287201FFFF04010A287201C7
:10698000FFFF0401AA287201FFFF0401AA28720177
:10699000FFFF0401AA287201FFFF0401AA28720167
:1069A000FFFF04015A111F01FFFF0401BBF2100198
:1069B000FFFF0401BBF21901FFFF0401BBF210014C
:1069C000FFFF04010A287201FFFF04010A28720177
:1069D000FFFF04010A287201FFFF04010A28720167
:1069E000FFFF04010A287201FFFF04010A28720157
:1069F000FFFF04010A287201FFFF04010A28720147
:106A0000FFFF0401AA287201FFFF0401AA287201F6
:106A1000FFFF0401AA287201FFFF0401AA287201E6
:106A2000FFFF0401FE00FF01FFFF0401BBF21001A4
:106A3000FFFF0401BBF21901FFFF0401BBF21001CB
:106A4000FFFF04010A287201FFFF04010A287201F6
:106A5000FFFF04010A287201FFFF04010A287201E6
:106A6000FFFF04010A287201FFFF04010A287201D6
:106A7000FFFF04010A287201FFFF04010A287201C6
:106A8000FFFF0401AA287201FFFF0401AA28720176
:106A9000FFFF0401AA287201FFFF0401AA28720166
:106AA000FFFF0401FE00FF01FFFF0401BBF2100124
:106AB000FFFF0401BBF21901FFFF0401BBF210014B
:106AC000FFFF04010A287201FFFF04010A28720176
:106AD000FFFF04010A287201FFFF04010A28720166
:106AE000FFFF04010A287201FFFF04010A28720156
:106AF000FFFF04010A287201FFFF04010A28720146
:106B0000FFFF0401AA287201FFFF0401AA287201F5
:106B1000FFFF0401AA287201FFFF0401AA287201E5
:106B2000FFFF04016A111E01FFFF0401BBF2100107
:106B3000FFFF0401BBF21901FFFF0401BBF21001CA
:106B4000FFFF04010A287201FFFF04010A287201F5
:106B5000FFFF04010A287201FFFF04010A287201E5
:106B6000FFFF04010A287201FFFF04010A287201D5
:106B7000FFFF04010A287201FFFF04010A287201C5
:106B8000FFFF0401AA287201FFFF0401AA28720175
:106B9000FFFF0401AA287201FFFF0401AA28720165
:106BA000FFFF04016A111E01FFFF0401BBF2100187
:106BB000FFFF0401BBF21901FFFF0401BBF210014A
:106BC000FFFF04010A287201FFFF04010A28720175
:106BD000FFFF04010A287201FFFF04010A28720165
:106BE000FFFF04010A287201FFFF04010A28720155
:106BF000FFFF04010A287201FFFF04010A28720145
:106C0000FFFF0401AA287201FFFF0401AA287201F4
:106C1000FFFF0401AA287201FFFF0401AA287201E4
:106C2000FFFF0401FE00FF01FFFF0401BBF21001A2
:106C3000FFFF0401BBF21901FFFF0401BBF21001C9
:106C4000FFFF04010A287201FFFF04010A287201F4
:106C5000FFFF04010A287201FFFF04010A287201E4
:106C6000FFFF04010A287201FFFF04010A287201D4
:106C7000FFFF04010A287201FFFF04010A287201C4
:106C8000FFFF0401AA287201FFFF0401AA28720174
:106C9000FFFF0401AA287201FFFF0401AA28720164
:106CA000FFFF0401FE00FF01FFFF0401BBF2100122
:106CB000FFFF0401BBF21901FFFF0401BBF2100149
:106CC000FFFF04010A287201FFFF04010A28720174
:106CD000FFFF04010A287201FFFF04010A28720164
:106CE000FFFF04010A287201FFFF04010A28720154
:106CF000FFFF04010A287201FFFF04010A28720144
:106D0000FFFF0401AA287201FFFF0401AA287201F3
:106D1000FFFF0401AA287201FFFF0401AA287201E3
:106D2000FFFF04012B282001FFFF0401BBF210012B
:106D3000FFFF0401BBF21901FFFF0401BBF21001C8
:106D4000FFFF04010A287201FFFF04010A287201F3
:106D5000FFFF04010A287201FFFF04010A287201E3
:106D6000FFFF04010A287201FFFF04010A287201D3
:106D7000FFFF04010A287201FFFF04010A287201C3
:106D8000FFFF0401AA287201FFFF0401AA28720173
:106D9000FFFF0401AA287201FFFF0401AA28720163
:106DA000FFFF04012B282001FFFF0401BBF21001AB
:106DB000FFFF0401BBF21901FFFF0401BBF2100148
:106DC000FFFF04010A287201FFFF04010A28720173
:106DD000FFFF04010A287201FFFF04010A28720163
:106DE000FFFF04010A287201FFFF04010A28720153
:106DF000FFFF04010A287201FFFF04010A28720143
:106E0000FFFF0401AA287201FFFF0401AA287201F2
:106E1000FFFF0401AA287201FFFF0401AA287201E2
:106E2000FFFF0401FE00FF01FFFF0401BBF21001A0
:106E3000FFFF0401BBF21901FFFF0401BBF21001C7
:106E4000FFFF04010A287201FFFF04010A287201F2
:106E5000FFFF04010A287201FFFF04010A287201E2
:106E6000FFFF04010A287201FFFF04010A287201D2
:106E7000FFFF04010A287201FFFF04010A287201C2
:106E8000FFFF0401AA287201FFFF0401AA28720172
:106E9000FFFF0401AA287201FFFF0401AA28720162
:106EA000FFFF0401FE00FF01FFFF0401BBF2100120
:106EB000FFFF0401BBF21901FFFF0401BBF2100147
:106EC000FFFF04010A287201FFFF04010A28720172
:106ED000FFFF04010A287201FFFF04010A28720162
:106EE000FFFF04010A287201FFFF04010A28720152
:106EF000FFFF04010A287201FFFF04010A28720142
:106F0000FFFF0401AA287201FFFF0401AA287201F1
:106F1000FFFF0401AA287201FFFF0401AA287201E1
:106F2000FFFF04016A111E01FFFF0401BBF2100103
:106F3000FFFF0401BBF21901FFFF0401BBF21001C6
:106F4000FFFF04010A287201FFFF04010A287201F1
:106F5000FFFF04010A287201FFFF04010A287201E1
:106F6000FFFF04010A287201FFFF04010A287201D1
:106F7000FFFF04010A287201FFFF04010A287201C1
:106F8000FFFF0401AA287201FFFF0401AA28720171
:106F9000FFFF0401AA287201FFFF0401AA28720161
:106FA000FFFF04016A111E01FFFF0401BBF2100183
:106FB000FFFF0401BBF21901FFFF0401BBF2100146
:106FC000FFFF04010A287201FFFF04010A28720171
:106FD000FFFF04010A287201FFFF04010A28720161
:106FE000FFFF04010A287201FFFF04010A28720151
:106FF000FFFF04010A287201FFFF04010A28720141
:10700000FFFF0401AA287201FFFF0401AA287201F0
:10701000FFFF0401AA287201FFFF0401AA287201E0
:10702000FFFF0401FE00FF01FFFF0401BBF210019E
:10703000FFFF0401BBF21901FFFF0401BBF21001C5
:10704000FFFF04010A287201FFFF04010A287201F0
:10705000FFFF04010A287201FFFF04010A287201E0
:10706000FFFF04010A287201FFFF04010A287201D0
:10707000FFFF04010A287201FFFF04010A287201C0
:10708000FFFF0401AA287201FFFF0401AA28720170
:10709000FFFF0401AA287201FFFF0401AA28720160
:1070A000FFFF0401FE00FF01FFFF0401BBF210011E
:1070B000FFFF0401BBF21901FFFF0401BBF2100145
:1070C000FFFF04010A287201FFFF04010A28720170
:1070D000FFFF04010A287201FFFF04010A28720160
:1070E000FFFF04010A287201FFFF04010A28720150
:1070F000FFFF04010A287201FFFF04010A28720140
:10710000FFFF0401AA287201FFFF0401AA287201EF
:10711000FFFF0401AA287201FFFF0401AA287201DF
:10712000FFFF04015A111F01FFFF0401BBF2100110
:10713000FFFF0401BBF21901FFFF0401BBF21001C4
:10714000FFFF04010A287201FFFF04010A287201EF
:10715000FFFF04010A287201FFFF04010A287201DF
:10716000FFFF04010A287201FFFF04010A287201CF
:10717000FFFF04010A287201FFFF04010A287201BF
:10718000FFFF0401AA287201FFFF0401AA2872016F
:10719000FFFF0401AA287201FFFF0401AA2872015F
:1071A000FFFF04015A111F01FFFF0401BBF2100190
:1071B000FFFF0401BBF21901FFFF0401BBF2100144
:1071C000FFFF04010A287201FFFF04010A2872016F
:1071D000FFFF04010A287201FFFF04010A2872015F
:1071E000FFFF04010A287201FFFF04010A2872014F
:1071F000FFFF04010A287201FFFF04010A2872013F
:10720000FFFF0401AA287201FFFF0401AA287201EE
:10721000FFFF0401AA287201FFFF0401AA287201DE
:10722000FFFF0401FE00FF01FFFF0401BBF210019C
:10723000FFFF0401BBF21901FFFF0401BBF21001C3
:10724000FFFF04010A287201FFFF04010A287201EE
:10725000FFFF04010A287201FFFF04010A287201DE
:10726000FFFF04010A287201FFFF04010A287201CE
:10727000FFFF04010A287201FFFF04010A287201BE
:10728000FFFF0401AA287201FFFF0401AA2872016E
:10729000FFFF0401AA287201FFFF0401AA2872015E
:1072A000FFFF0401FE00FF01FFFF0401BBF210011C
:1072B000FFFF0401BBF21901FFFF0401BBF2100143
:1072C000FFFF04010A287201FFFF04010A2872016E
:1072D000FFFF04010A287201FFFF04010A2872015E
:1072E000FFFF04010A287201FFFF04010A2872014E
:1072F000FFFF04010A287201FFFF04010A2872013E
:10730000FFFF0401AA287201FFFF0401AA287201ED
:10731000FFFF0401AA287201FFFF0401AA287201DD
:10732000FFFF04016A111E01FFFF0401BBF21001FF
:10733000FFFF0401BBF21901FFFF0401BBF21001C2
:10734000FFFF04010A287201FFFF04010A287201ED
:10735000FFFF04010A287201FFFF04010A287201DD
:10736000FFFF04010A287201FFFF04010A287201CD
:10737000FFFF04010A287201FFFF04010A287201BD
:10738000FFFF0401AA287201FFFF0401AA2872016D
:10739000FFFF0401AA287201FFFF0401AA2872015D
:1073A000FFFF04016A111E01FFFF0401BBF210017F
:1073B000FFFF0401BBF21901FFFF0401BBF2100142
:1073C000FFFF04010A287201FFFF04010A2872016D
:1073D000FFFF04010A287201FFFF04010A2872015D
:1073E000FFFF04010A287201FFFF04010A2872014D
:1073F000FFFF04010A287201FFFF04010A2872013D
:10740000FFFF0401AA287201FFFF0401AA287201EC
:10741000FFFF0401AA287201FFFF0401AA287201DC
:10742000FFFF0401FE00FF01FFFF0401BBF210019A
:10743000FFFF0401BBF21901FFFF0401BBF21001C1
:10744000FFFF04010A287201FFFF04010A287201EC
:10745000FFFF04010A287201FFFF04010A287201DC
:10746000FFFF04010A287201FFFF04010A287201CC
:10747000FFFF04010A287201FFFF04010A287201BC
:10748000FFFF0401AA287201FFFF0401AA2872016C
:10749000FFFF0401AA287201FFFF0401AA2872015C
:1074A000FFFF0401FE00FF01FFFF0401BBF210011A
:1074B000FFFF0401BBF21901FFFF0401BBF2100141
:1074C000FFFF04010A287201FFFF04010A2872016C
:1074D000FFFF04010A287201FFFF04010A2872015C
:1074E000FFFF04010A287201FFFF04010A2872014C
:1074F000FFFF04010A287201FFFF04010A2872013C
:10750000FFFF0401AA287201FFFF0401AA287201EB
:10751000FFFF0401AA287201FFFF0401AA287201DB
:10752000FFFF04012B282001FFFF0401BBF2100123
:10753000FFFF0401BBF21901FFFF0401BBF21001C0
:10754000FFFF04010A287201FFFF04010A287201EB
:10755000FFFF04010A287201FFFF04010A287201DB
:10756000FFFF04010A287201FFFF04010A287201CB
:10757000FFFF04010A287201FFFF04010A287201BB
:10758000FFFF0401AA287201FFFF0401AA2872016B
:10759000FFFF0401AA287201FFFF0401AA2872015B
:1075A000FFFF04012B282001FFFF0401BBF21001A3
:1075B000FFFF0401BBF21901FFFF0401BBF2100140
:1075C000FFFF04010A287201FFFF04010A2872016B
:1075D000FFFF04010A287201FFFF04010A2872015B
:1075E000FFFF04010A287201FFFF04010A2872014B
:1075F000FFFF04010A287201FFFF04010A2872013B
:10760000FFFF0401AA287201FFFF0401AA287201EA
:10761000FFFF0401AA287201FFFF0401AA287201DA
:10762000FFFF0401FE00FF01FFFF0401BBF2100198
:10763000FFFF0401BBF21901FFFF0401BBF21001BF
:10764000FFFF04010A287201FFFF04010A287201EA
:10765000FFFF04010A287201FFFF04010A287201DA
:10766000FFFF04010A287201FFFF04010A287201CA
:10767000FFFF04010A287201FFFF04010A287201BA
:10768000FFFF0401AA287201FFFF0401AA2872016A
:10769000FFFF0401AA287201FFFF0401AA2872015A
:1076A000FFFF0401FE00FF01FFFF0401BBF2100118
:1076B000FFFF0401BBF21901FFFF0401BBF210013F
:1076C000FFFF04010A287201FFFF04010A2872016A
:1076D000FFFF04010A287201FFFF04010A2872015A
:1076E000FFFF04010A287201FFFF04010A2872014A
:1076F000FFFF04010A287201FFFF04010A2872013A
:10770000FFFF0401AA287201FFFF0401AA287201E9
:10771000FFFF0401AA287201FFFF0401AA287201D9
:10772000FFFF04016A111E01FFFF0401BBF21001FB
:10773000FFFF0401BBF21901FFFF0401BBF21001BE
:10774000FFFF04010A287201FFFF04010A287201E9
:10775000FFFF04010A287201FFFF04010A287201D9
:10776000FFFF04010A287201FFFF04010A287201C9
:10777000FFFF04010A287201FFFF04010A287201B9
:10778000FFFF0401AA287201FFFF0401AA28720169
:10779000FFFF0401AA287201FFFF0401AA28720159
:1077A000FFFF04016A111E01FFFF0401BBF210017B
:1077B000FFFF0401BBF21901FFFF0401BBF210013E
:1077C000FFFF04010A287201FFFF04010A28720169
:1077D000FFFF04010A287201FFFF04010A28720159
:1077E000FFFF04010A287201FFFF04010A28720149
:1077F000FFFF04010A287201FFFF04010A28720139
:10780000FFFF0401AA287201FFFF0401AA287201E8
:10781000FFFF0401AA287201FFFF0401AA287201D8
:10782000FFFF0401FE00FF01FFFF0401BBF2100196
:10783000FFFF0401BBF21901FFFF0401BBF21001BD
:10784000FFFF04010A287201FFFF04010A287201E8
:10785000FFFF04010A287201FFFF04010A287201D8
:10786000FFFF04010A287201FFFF04010A287201C8
:10787000FFFF04010A287201FFFF04010A287201B8
:10788000FFFF0401AA287201FFFF0401AA28720168
:10789000FFFF0401AA287201FFFF0401AA28720158
:1078A000FFFF0401FE00FF01FFFF0401BBF2100116
:1078B000FFFF0401BBF21901FFFF0401BBF210013D
:1078C000FFFF04010A287201FFFF04010A28720168
:1078D000FFFF04010A287201FFFF04010A28720158
:1078E000FFFF04010A287201FFFF04010A28720148
:1078F000FFFF04010A287201FFFF04010A28720138
:10790000FFFF0401AA287201FFFF0401AA287201E7
:10791000FFFF0401AA287201FFFF0401AA287201D7
:10792000FFFF04015A111F01FFFF0401BBF2100108
:10793000FFFF0401BBF21901FFFF0401BBF21001BC
:10794000FFFF04010A287201FFFF04010A287201E7
:10795000FFFF04010A287201FFFF04010A287201D7
:10796000FFFF04010A287201FFFF04010A287201C7
:10797000FFFF04010A287201FFFF04010A287201B7
:10798000FFFF0401AA287201FFFF0401AA28720167
:10799000FFFF0401AA287201FFFF0401AA28720157
:1079A000FFFF04015A111F01FFFF0401BBF2100188
:1079B000FFFF0401BBF21901FFFF0401BBF210013C
:1079C000FFFF04010A287201FFFF04010A28720167
:1079D000FFFF04010A287201FFFF04010A28720157
:1079E000FFFF04010A287201FFFF04010A28720147
:1079F000FFFF04010A287201FFFF04010A28720137
:107A0000FFFF0401AA287201FFFF0401AA287201E6
:107A1000FFFF0401AA287201FFFF0401AA287201D6
:107A2000FFFF0401FE00FF01FFFF0401BBF2100194
:107A3000FFFF0401BBF21901FFFF0401BBF21001BB
:107A4000FFFF04010A287201FFFF04010A287201E6
:107A5000FFFF04010A287201FFFF04010A287201D6
:107A6000FFFF04010A287201FFFF04010A287201C6
:107A7000FFFF04010A287201FFFF04010A287201B6
:107A8000FFFF0401AA287201FFFF0401AA28720166
:107A9000FFFF0401AA287201FFFF0401AA28720156
:107AA000FFFF0401FE00FF01FFFF0401BBF2100114
:107AB000FFFF0401BBF21901FFFF0401BBF210013B
:107AC000FFFF04010A287201FFFF04010A28720166
:107AD000FFFF04010A287201FFFF04010A28720156
:107AE000FFFF04010A287201FFFF04010A28720146
:107AF000FFFF04010A287201FFFF04010A28720136
:107B0000FFFF0401AA287201FFFF0401AA287201E5
:107B1000FFFF0401AA287201FFFF0401AA287201D5
:107B2000FFFF04016A111E01FFFF0401BBF21001F7
:107B3000FFFF0401BBF21901FFFF0401BBF21001BA
:107B4000FFFF04010A287201FFFF04010A287201E5
:107B5000FFFF04010A287201FFFF04010A287201D5
:107B6000FFFF04010A287201FFFF04010A287201C5
:107B7000FFFF04010A287201FFFF04010A287201B5
:107B8000FFFF0401AA287201FFFF0401AA28720165
:107B9000FFFF0401AA287201FFFF0401AA28720155
:107BA000FFFF04016A111E01FFFF0401BBF2100177
:107BB000FFFF0401BBF21901FFFF0401BBF210013A
:107BC000FFFF04010A287201FFFF04010A28720165
:107BD000FFFF04010A287201FFFF04010A28720155
:107BE000FFFF04010A287201FFFF04010A28720145
:107BF000FFFF04010A287201FFFF04010A28720135
:107C0000FFFF0401AA287201FFFF0401AA287201E4
:107C1000FFFF0401AA287201FFFF0401AA287201D4
:107C2000FFFF0401FE00FF01FFFF0401BBF2100192
:107C3000FFFF0401BBF21901FFFF0401BBF21001B9
:107C4000FFFF04010A287201FFFF04010A287201E4
:107C5000FFFF04010A287201FFFF04010A287201D4
:107C6000FFFF04010A287201FFFF04010A287201C4
:107C7000FFFF04010A287201FFFF04010A287201B4
:107C8000FFFF0401AA287201FFFF0401AA28720164
:107C9000FFFF0401AA287201FFFF0401AA28720154
:107CA000FFFF0401FE00FF01FFFF0401BBF2100112
:107CB000FFFF0401BBF21901FFFF0401BBF2100139
:107CC000FFFF04010A287201FFFF04010A28720164
:107CD000FFFF04010A287201FFFF04010A28720154
:107CE000FFFF04010A287201FFFF04010A28720144
:107CF000FFFF04010A287201FFFF04010A28720134
:107D0000FFFF0401AA287201FFFF0401AA287201E3
:107D1000FFFF0401AA287201FFFF0401AA287201D3
:107D2000FFFF04012B282001FFFF0401BBF210011B
:107D3000FFFF0401BBF21901FFFF0401BBF21001B8
:107D4000FFFF04010A287201FFFF04010A287201E3
:107D5000FFFF04010A287201FFFF04010A287201D3
:107D6000FFFF04010A287201FFFF04010A287201C3
:107D7000FFFF04010A287201FFFF04010A287201B3
:107D8000FFFF0401AA287201FFFF0401AA28720163
:107D9000FFFF0401AA287201FFFF0401AA28720153
:107DA000FFFF04012B282001FFFF0401BBF210019B
:107DB000FFFF0401BBF21901FFFF0401BBF2100138
:107DC000FFFF04010A287201FFFF04010A28720163
:107DD000FFFF04010A287201FFFF04010A28720153
:107DE000FFFF04010A287201FFFF04010A28720143
:107DF000FFFF04010A287201FFFF04010A28720133
:107E0000FFFF0401AA287201FFFF0401AA287201E2
:107E1000FFFF0401AA287201FFFF0401AA287201D2
:107E2000FFFF0401FE00FF01FFFF0401BBF2100190
:107E3000FFFF0401BBF21901FFFF0401BBF21001B7
:107E4000FFFF04010A287201FFFF04010A287201E2
:107E5000FFFF04010A287201FFFF04010A287201D2
:107E6000FFFF04010A287201FFFF04010A287201C2
:107E7000FFFF04010A287201FFFF04010A287201B2
:107E8000FFFF0401AA287201FFFF0401AA28720162
:107E9000FFFF0401AA287201FFFF0401AA28720152
:107EA000FFFF0401FE00FF01FFFF0401BBF2100110
:107EB000FFFF0401BBF21901FFFF0401BBF2100137
:107EC000FFFF04010A287201FFFF04010A28720162
:107ED000FFFF04010A287201FFFF04010A28720152
:107EE000FFFF04010A287201FFFF04010A28720142
:107EF000FFFF04010A287201FFFF04010A28720132
:107F0000FFFF0401AA287201FFFF0401AA287201E1
:107F1000FFFF0401AA287201FFFF0401AA287201D1
:107F2000FFFF04016A111E01FFFF0401BBF21001F3
:107F3000FFFF0401BBF21901FFFF0401BBF21001B6
:107F4000FFFF04010A287201FFFF04010A287201E1
:107F5000FFFF04010A287201FFFF04010A287201D1
:107F6000FFFF04010A287201FFFF04010A287201C1
:107F7000FFFF04010A287201FFFF04010A287201B1
:107F8000FFFF0401AA287201FFFF0401AA28720161
:107F9000FFFF0401AA287201FFFF0401AA28720151
:107FA000FFFF04016A111E01FFFF0401BBF2100173
:107FB000FFFF0401BBF21901FFFF0401BBF2100136
:107FC000FFFF04010A287201FFFF04010A28720161
:107FD000FFFF04010A287201FFFF04010A28720151
:107FE000FFFF04010A287201FFFF04010A28720141
:107FF000FFFF04010A287201FFFF04010A28720131
:10800000FFFF0401AA287201FFFF0401AA287201E0
:10801000FFFF0401AA287201FFFF0401AA287201D0
:10802000FFFF0401FE00FF01FFFF0401BBF210018E
:10803000FFFF0401BBF21901FFFF0401BBF21001B5
:10804000FFFF04010A287201FFFF04010A287201E0
:10805000FFFF04010A287201FFFF04010A287201D0
:10806000FFFF04010A287201FFFF04010A287201C0
:10807000FFFF04010A287201FFFF04010A287201B0
:10808000FFFF0401AA287201FFFF0401AA28720160
:10809000FFFF0401AA287201FFFF0401AA28720150
:1080A000FFFF0401FE00FF01FFFF0401BBF210010E
:1080B000FFFF0401BBF21901FFFF0401BBF2100135
:1080C000FFFF04010A287201FFFF04010A28720160
:1080D000FFFF04010A287201FFFF04010A28720150
:1080E000FFFF04010A287201FFFF04010A28720140
:1080F000FFFF04010A287201FFFF04010A28720130
:10810000FFFF0401AA287201FFFF0401AA287201DF
:10811000FFFF0401AA287201FFFF0401AA287201CF
:10812000FFFF04010A247201FFFF0401BBF21001EA
:10813000FFFF0401BBF21901FFFF0401BBF21001B4
:10814000FFFF04010A287201FFFF04010A287201DF
:10815000FFFF04010A287201FFFF04010A287201CF
:10816000FFFF04010A287201FFFF04010A287201BF
:10817000FFFF04010A287201FFFF04010A287201AF
:10818000FFFF0401AA287201FFFF0401AA2872015F
:10819000FFFF0401AA287201FFFF0401AA2872014F
:1081A000FFFF04010A247201FFFF0401BBF210016A
:1081B000FFFF0401BBF21901FFFF0401BBF2100134
:1081C000FFFF04010A287201FFFF04010A2872015F
:1081D000FFFF04010A287201FFFF04010A2872014F
:1081E000FFFF04010A287201FFFF04010A2872013F
:1081F000FFFF04010A287201FFFF04010A2872012F
:10820000FFFF0401AA287201FFFF0401AA287201DE
:10821000FFFF0401AA287201FFFF0401AA287201CE
:10822000FFFF0401FE00FF01FFFF0401BBF210018C
:10823000FFFF0401BBF21901FFFF0401BBF21001B3
:10824000FFFF04010A287201FFFF04010A287201DE
:10825000FFFF04010A287201FFFF04010A287201CE
:10826000FFFF04010A287201FFFF04010A287201BE
:10827000FFFF04010A287201FFFF04010A287201AE
:10828000FFFF0401AA287201FFFF0401AA2872015E
:10829000FFFF0401AA287201FFFF0401AA2872014E
:1082A000FFFF0401FE00FF01FFFF0401BBF210010C
:1082B000FFFF0401BBF21901FFFF0401BBF2100133
:1082C000FFFF04010A287201FFFF04010A2872015E
:1082D000FFFF04010A287201FFFF04010A2872014E
:1082E000FFFF04010A287201FFFF04010A2872013E
:1082F000FFFF04010A287201FFFF04010A2872012E
:10830000FFFF0401AA287201FFFF0401AA287201DD
:10831000FFFF0401AA287201FFFF0401AA287201CD
:10832000FFFF04010A247201FFFF0401BBF21001E8
:10833000FFFF0401BBF21901FFFF0401BBF21001B2
:10834000FFFF04010A287201FFFF04010A287201DD
:10835000FFFF04010A287201FFFF04010A287201CD
:10836000FFFF04010A287201FFFF04010A287201BD
:10837000FFFF04010A287201FFFF04010A287201AD
:10838000FFFF0401AA287201FFFF0401AA2872015D
:10839000FFFF0401AA287201FFFF0401AA2872014D
:1083A000FFFF04010A247201FFFF0401BBF2100168
:1083B000FFFF0401BBF21901FFFF0401BBF2100132
:1083C000FFFF04010A287201FFFF04010A2872015D
:1083D000FFFF04010A287201FFFF04010A2872014D
:1083E000FFFF04010A287201FFFF04010A2872013D
:1083F000FFFF04010A287201FFFF04010A2872012D
:10840000FFFF0401AA287201FFFF0401AA287201DC
:10841000FFFF0401AA287201FFFF0401AA287201CC
:10842000FFFF0401FE00FF01FFFF0401BBF210018A
:10843000FFFF0401BBF21901FFFF0401BBF21001B1
:10844000FFFF04010A287201FFFF04010A287201DC
:10845000FFFF04010A287201FFFF04010A287201CC
:10846000FFFF04010A287201FFFF04010A287201BC
:10847000FFFF04010A287201FFFF04010A287201AC
:10848000FFFF0401AA287201FFFF0401AA2872015C
:10849000FFFF0401AA287201FFFF0401AA2872014C
:1084A000FFFF0401FE00FF01FFFF0401BBF210010A
:1084B000FFFF0401BBF21901FFFF0401BBF2100131
:1084C000FFFF04010A287201FFFF04010A2872015C
:1084D000FFFF04010A287201FFFF04010A2872014C
:1084E000FFFF04010A287201FFFF04010A2872013C
:1084F000FFFF04010A287201FFFF04010A2872012C
:10850000FFFF0401AA287201FFFF0401AA287201DB
:10851000FFFF0401AA287201FFFF0401AA287201CB
:10852000FFFF04010A247201FFFF0401BBF21001E6
:10853000FFFF0401BBF21901FFFF0401BBF21001B0
:10854000FFFF04010A287201FFFF04010A287201DB
:10855000FFFF04010A287201FFFF04010A287201CB
:10856000FFFF04010A287201FFFF04010A287201BB
:10857000FFFF04010A287201FFFF04010A287201AB
:10858000FFFF0401AA287201FFFF0401AA2872015B
:10859000FFFF0401AA287201FFFF0401AA2872014B
:1085A000FFFF04010A247201FFFF0401BBF2100166
:1085B000FFFF0401BBF21901FFFF0401BBF2100130
:1085C000FFFF04010A287201FFFF04010A2872015B
:1085D000FFFF04010A287201FFFF04010A2872014B
:1085E000FFFF04010A287201FFFF04010A2872013B
:1085F000FFFF04010A287201FFFF04010A2872012B
:10860000FFFF0401AA287201FFFF0401AA287201DA
:10861000FFFF0401AA287201FFFF0401AA287201CA
:10862000FFFF0401FE00FF01FFFF0401BBF2100188
:10863000FFFF0401BBF21901FFFF0401BBF21001AF
:10864000FFFF04010A287201FFFF04010A287201DA
:10865000FFFF04010A287201FFFF04010A287201CA
:10866000FFFF04010A287201FFFF04010A287201BA
:10867000FFFF04010A287201FFFF04010A287201AA
:10868000FFFF0401AA287201FFFF0401AA2872015A
:10869000FFFF0401AA287201FFFF0401AA2872014A
:1086A000FFFF0401FE00FF01FFFF0401BBF2100108
:1086B000FFFF0401BBF21901FFFF0401BBF210012F
:1086C000FFFF04010A287201FFFF04010A2872015A
:1086D000FFFF04010A287201FFFF04010A2872014A
:1086E000FFFF04010A287201FFFF04010A2872013A
:1086F000FFFF04010A287201FFFF04010A2872012A
:10870000FFFF0401AA287201FFFF0401AA287201D9
:10871000FFFF0401AA287201FFFF0401AA287201C9
:10872000FFFF04010A247201FFFF0401BBF21001E4
:10873000FFFF0401BBF21901FFFF0401BBF21001AE
:10874000FFFF04010A287201FFFF04010A287201D9
:10875000FFFF04010A287201FFFF04010A287201C9
:10876000FFFF04010A287201FFFF04010A287201B9
:10877000FFFF04010A287201FFFF04010A287201A9
:10878000FFFF0401AA287201FFFF0401AA28720159
:10879000FFFF0401AA287201FFFF0401AA28720149
:1087A000FFFF04010A247201FFFF0401BBF2100164
:1087B000FFFF0401BBF21901FFFF0401BBF210012E
:1087C000FFFF04010A287201FFFF04010A28720159
:1087D000FFFF04010A287201FFFF04010A28720149
:1087E000FFFF04010A287201FFFF04010A28720139
:1087F000FFFF04010A287201FFFF04010A28720129
:10880000FFFF0401AA287201FFFF0401AA287201D8
:10881000FFFF0401AA287201FFFF0401AA287201C8
:10882000FFFF0401FE00FF01FFFF0401BBF2100186
:10883000FFFF0401BBF21901FFFF0401BBF21001AD
:10884000FFFF04010A287201FFFF04010A287201D8
:10885000FFFF04010A287201FFFF04010A287201C8
:10886000FFFF04010A287201FFFF04010A287201B8
:10887000FFFF04010A287201FFFF04010A287201A8
:10888000FFFF0401AA287201FFFF0401AA28720158
:10889000FFFF0401AA287201FFFF0401AA28720148
:1088A000FFFF0401FE00FF01FFFF0401BBF2100106
:1088B000FFFF0401BBF21901FFFF0401BBF210012D
:1088C000FFFF04010A287201FFFF04010A28720158
:1088D000FFFF04010A287201FFFF04010A28720148
:1088E000FFFF04010A287201FFFF04010A28720138
:1088F000FFFF04010A287201FFFF04010A28720128
:10890000FFFF0401AA287201FFFF0401AA287201D7
:10891000FFFF0401AA287201FFFF0401AA287201C7
:10892000FFFF04010A247201FFFF0401BBF21001E2
:10893000FFFF0401BBF21901FFFF0401BBF21001AC
:10894000FFFF04010A287201FFFF04010A287201D7
:10895000FFFF04010A287201FFFF04010A287201C7
:10896000FFFF04010A287201FFFF04010A287201B7
:10897000FFFF04010A287201FFFF04010A287201A7
:10898000FFFF0401AA287201FFFF0401AA28720157
:10899000FFFF0401AA287201FFFF0401AA28720147
:1089A000FFFF04010A247201FFFF0401BBF2100162
:1089B000FFFF0401BBF21901FFFF0401BBF210012C
:1089C000FFFF04010A287201FFFF04010A28720157
:1089D000FFFF04010A287201FFFF04010A28720147
:1089E000FFFF04010A287201FFFF04010A28720137
:1089F000FFFF04010A287201FFFF04010A28720127
:108A0000FFFF0401AA287201FFFF0401AA287201D6
:108A1000FFFF0401AA287201FFFF0401AA287201C6
:108A2000FFFF0401FE00FF01FFFF0401BBF2100184
:108A3000FFFF0401BBF21901FFFF0401BBF21001AB
:108A4000FFFF04010A287201FFFF04010A287201D6
:108A5000FFFF04010A287201FFFF04010A287201C6
:108A6000FFFF04010A287201FFFF04010A287201B6
:108A7000FFFF04010A287201FFFF04010A287201A6
:108A8000FFFF0401AA287201FFFF0401AA28720156
:108A9000FFFF0401AA287201FFFF0401AA28720146
:108AA000FFFF0401FE00FF01FFFF0401BBF2100104
:108AB000FFFF0401BBF21901FFFF0401BBF210012B
:108AC000FFFF04010A287201FFFF04010A28720156
:108AD000FFFF04010A287201FFFF04010A28720146
:108AE000FFFF04010A287201FFFF04010A28720136
:108AF000FFFF04010A287201FFFF04010A28720126
:108B0000FFFF0401AA287201FFFF0401AA287201D5
:108B1000FFFF0401AA287201FFFF0401AA287201C5
:108B2000FFFF04010A247201FFFF0401BBF21001E0
:108B3000FFFF0401BBF21901FFFF0401BBF21001AA
:108B4000FFFF04010A287201FFFF04010A287201D5
:108B5000FFFF04010A287201FFFF04010A287201C5
:108B6000FFFF04010A287201FFFF04010A287201B5
:108B7000FFFF04010A287201FFFF04010A287201A5
:108B8000FFFF0401AA287201FFFF0401AA28720155
:108B9000FFFF0401AA287201FFFF0401AA28720145
:108BA000FFFF04010A247201FFFF0401BBF2100160
:108BB000FFFF0401BBF21901FFFF0401BBF210012A
:108BC000FFFF04010A287201FFFF04010A28720155
:108BD000FFFF04010A287201FFFF04010A28720145
:108BE000FFFF04010A287201FFFF04010A28720135
:108BF000FFFF04010A287201FFFF04010A28720125
:108C0000FFFF0401AA287201FFFF0401AA287201D4
:108C1000FFFF0401AA287201FFFF0401AA287201C4
:108C2000FFFF0401FE00FF01FFFF0401BBF2100182
:108C3000FFFF0401BBF21901FFFF0401BBF21001A9
:108C4000FFFF04010A287201FFFF04010A287201D4
:108C5000FFFF04010A287201FFFF04010A287201C4
:108C6000FFFF04010A287201FFFF04010A287201B4
:108C7000FFFF04010A287201FFFF04010A287201A4
:108C8000FFFF0401AA287201FFFF0401AA28720154
:108C9000FFFF0401AA287201FFFF0401AA28720144
:108CA000FFFF0401FE00FF01FFFF0401BBF2100102
:108CB000FFFF0401BBF21901FFFF0401BBF2100129
:108CC000FFFF04010A287201FFFF04010A28720154
:108CD000FFFF04010A287201FFFF04010A28720144
:108CE000FFFF04010A287201FFFF04010A28720134
:108CF000FFFF04010A287201FFFF04010A28720124
:108D0000FFFF0401AA287201FFFF0401AA287201D3
:108D1000FFFF0401AA287201FFFF0401AA287201C3
:108D2000FFFF04010A247201FFFF0401BBF21001DE
:108D3000FFFF0401BBF21901FFFF0401BBF21001A8
:108D4000FFFF04010A287201FFFF04010A287201D3
:108D5000FFFF04010A287201FFFF04010A287201C3
:108D6000FFFF04010A287201FFFF04010A287201B3
:108D7000FFFF04010A287201FFFF04010A287201A3
:108D8000FFFF0401AA287201FFFF0401AA28720153
:108D9000FFFF0401AA287201FFFF0401AA28720143
:108DA000FFFF04010A247201FFFF0401BBF210015E
:108DB000FFFF0401BBF21901FFFF0401BBF2100128
:108DC000FFFF04010A287201FFFF04010A28720153
:108DD000FFFF04010A287201FFFF04010A28720143
:108DE000FFFF04010A287201FFFF04010A28720133
:108DF000FFFF04010A287201FFFF04010A28720123
:108E0000FFFF0401AA287201FFFF0401AA287201D2
:108E1000FFFF0401AA287201FFFF0401AA287201C2
:108E2000FFFF0401FE00FF01FFFF0401BBF2100180
:108E3000FFFF0401BBF21901FFFF0401BBF21001A7
:108E4000FFFF04010A287201FFFF04010A287201D2
:108E5000FFFF04010A287201FFFF04010A287201C2
:108E6000FFFF04010A287201FFFF04010A287201B2
:108E7000FFFF04010A287201FFFF04010A287201A2
:108E8000FFFF0401AA287201FFFF0401AA28720152
:108E9000FFFF0401AA287201FFFF0401AA28720142
:108EA000FFFF0401FE00FF01FFFF0401BBF2100100
:108EB000FFFF0401BBF21901FFFF0401BBF2100127
:108EC000FFFF04010A287201FFFF04010A28720152
:108ED000FFFF04010A287201FFFF04010A28720142
:108EE000FFFF04010A287201FFFF04010A28720132
:108EF000FFFF04010A287201FFFF04010A28720122
:108F0000FFFF0401AA287201FFFF0401AA287201D1
:108F1000FFFF0401AA287201FFFF0401AA287201C1
:108F2000FFFF04010A247201FFFF0401BBF21001DC
:108F3000FFFF0401BBF21901FFFF0401BBF21001A6
:108F4000FFFF04010A287201FFFF04010A287201D1
:108F5000FFFF04010A287201FFFF04010A287201C1
:108F6000FFFF04010A287201FFFF04010A287201B1
:108F7000FFFF04010A287201FFFF04010A287201A1
:108F8000FFFF0401AA287201FFFF0401AA28720151
:108F9000FFFF0401AA287201FFFF0401AA28720141
:108FA000FFFF04010A247201FFFF0401BBF210015C
:108FB000FFFF0401BBF21901FFFF0401BBF2100126
:108FC000FFFF04010A287201FFFF04010A28720151
:108FD000FFFF04010A287201FFFF04010A28720141
:108FE000FFFF04010A287201FFFF04010A28720131
:108FF000FFFF04010A287201FFFF04010A28720121
:10900000FFFF0401AA287201FFFF0401AA287201D0
:10901000FFFF0401AA287201FFFF0401AA287201C0
:10902000FFFF0401FE00FF01FFFF0401BBF210017E
:10903000FFFF0401BBF21901FFFF0401BBF21001A5
:10904000FFFF04010A287201FFFF04010A287201D0
:10905000FFFF04010A287201FFFF04010A287201C0
:10906000FFFF04010A287201FFFF04010A287201B0
:10907000FFFF04010A287201FFFF04010A287201A0
:10908000FFFF0401AA287201FFFF0401AA28720150
:10909000FFFF0401AA287201FFFF0401AA28720140
:1090A000FFFF0401FE00FF01FFFF0401BBF21001FE
:1090B000FFFF0401BBF21901FFFF0401BBF2100125
:1090C000FFFF04010A287201FFFF04010A28720150
:1090D000FFFF04010A287201FFFF04010A28720140
:1090E000FFFF04010A287201FFFF04010A28720130
:1090F000FFFF04010A287201FFFF04010A28720120
:10910000FFFF0401AA287201FFFF0401AA287201CF
:10911000FFFF0401AA287201FFFF0401AA287201BF
:10912000FFFF04010A247201FFFF0401BBF21001DA
:10913000FFFF0401BBF21901FFFF0401BBF21001A4
:10914000FFFF04010A287201FFFF04010A287201CF
:10915000FFFF04010A287201FFFF04010A287201BF
:10916000FFFF04010A287201FFFF04010A287201AF
:10917000FFFF04010A287201FFFF04010A2872019F
:10918000FFFF0401AA287201FFFF0401AA2872014F
:10919000FFFF0401AA287201FFFF0401AA2872013F
:1091A000FFFF04010A247201FFFF0401BBF210015A
:1091B000FFFF0401BBF21901FFFF0401BBF2100124
:1091C000FFFF04010A287201FFFF04010A2872014F
:1091D000FFFF04010A287201FFFF04010A2872013F
:1091E000FFFF04010A287201FFFF04010A2872012F
:1091F000FFFF04010A287201FFFF04010A2872011F
:10920000FFFF0401AA287201FFFF0401AA287201CE
:10921000FFFF0401AA287201FFFF0401AA287201BE
:10922000FFFF0401FE00FF01FFFF0401BBF210017C
:10923000FFFF0401BBF21901FFFF0401BBF21001A3
:10924000FFFF04010A287201FFFF04010A287201CE
:10925000FFFF04010A287201FFFF04010A287201BE
:10926000FFFF04010A287201FFFF04010A287201AE
:10927000FFFF04010A287201FFFF04010A2872019E
:10928000FFFF0401AA287201FFFF0401AA2872014E
:10929000FFFF0401AA287201FFFF0401AA2872013E
:1092A000FFFF0401FE00FF01FFFF0401BBF21001FC
:1092B000FFFF0401BBF21901FFFF0401BBF2100123
:1092C000FFFF04010A287201FFFF04010A2872014E
:1092D000FFFF04010A287201FFFF04010A2872013E
:1092E000FFFF04010A287201FFFF04010A2872012E
:1092F000FFFF04010A287201FFFF04010A2872011E
:10930000FFFF0401AA287201FFFF0401AA287201CD
:10931000FFFF0401AA287201FFFF0401AA287201BD
:10932000FFFF04010A247201FFFF0401BBF21001D8
:10933000FFFF0401BBF21901FFFF0401BBF21001A2
:10934000FFFF04010A287201FFFF04010A287201CD
:10935000FFFF04010A287201FFFF04010A287201BD
:10936000FFFF04010A287201FFFF04010A287201AD
:10937000FFFF04010A287201FFFF04010A2872019D
:10938000FFFF0401AA287201FFFF0401AA2872014D
:10939000FFFF0401AA287201FFFF0401AA2872013D
:1093A000FFFF04010A247201FFFF0401BBF2100158
:1093B000FFFF0401BBF21901FFFF0401BBF2100122
:1093C000FFFF04010A287201FFFF04010A2872014D
:1093D000FFFF04010A287201FFFF04010A2872013D
:1093E000FFFF04010A287201FFFF04010A2872012D
:1093F000FFFF04010A287201FFFF04010A2872011D
:10940000FFFF0401AA287201FFFF0401AA287201CC
:10941000FFFF0401AA287201FFFF0401AA287201BC
:10942000FFFF0401FE00FF01FFFF0401BBF210017A
:10943000FFFF0401BBF21901FFFF0401BBF21001A1
:10944000FFFF04010A287201FFFF04010A287201CC
:10945000FFFF04010A287201FFFF04010A287201BC
:10946000FFFF04010A287201FFFF04010A287201AC
:10947000FFFF04010A287201FFFF04010A2872019C
:10948000FFFF0401AA287201FFFF0401AA2872014C
:10949000FFFF0401AA287201FFFF0401AA2872013C
:1094A000FFFF0401FE00FF01FFFF0401BBF21001FA
:1094B000FFFF0401BBF21901FFFF0401BBF2100121
:1094C000FFFF04010A287201FFFF04010A2872014C
:1094D000FFFF04010A287201FFFF04010A2872013C
:1094E000FFFF04010A287201FFFF04010A2872012C
:1094F000FFFF04010A287201FFFF04010A2872011C
:10950000FFFF0401AA287201FFFF0401AA287201CB
:10951000FFFF0401AA287201FFFF0401AA287201BB
:10952000FFFF04010A247201FFFF0401BBF21001D6
:10953000FFFF0401BBF21901FFFF0401BBF21001A0
:10954000FFFF04010A287201FFFF04010A287201CB
:10955000FFFF04010A287201FFFF04010A287201BB
:10956000FFFF04010A287201FFFF04010A287201AB
:10957000FFFF04010A287201FFFF04010A2872019B
:10958000FFFF0401AA287201FFFF0401AA2872014B
:10959000FFFF0401AA287201FFFF0401AA2872013B
:1095A000FFFF04010A247201FFFF0401BBF2100156
:1095B000FFFF0401BBF21901FFFF0401BBF2100120
:1095C000FFFF04010A287201FFFF04010A2872014B
:1095D000FFFF04010A287201FFFF04010A2872013B
:1095E000FFFF04010A287201FFFF04010A2872012B
:1095F000FFFF04010A287201FFFF04010A2872011B
:10960000FFFF0401AA287201FFFF0401AA287201CA
:10961000FFFF0401AA287201FFFF0401AA287201BA
:10962000FFFF0401FE00FF01FFFF0401BBF2100178
:10963000FFFF0401BBF21901FFFF0401BBF210019F
:10964000FFFF04010A287201FFFF04010A287201CA
:10965000FFFF04010A287201FFFF04010A287201BA
:10966000FFFF04010A287201FFFF04010A287201AA
:10967000FFFF04010A287201FFFF04010A2872019A
:10968000FFFF0401AA287201FFFF0401AA2872014A
:10969000FFFF0401AA287201FFFF0401AA2872013A
:1096A000FFFF0401FE00FF01FFFF0401BBF21001F8
:1096B000FFFF0401BBF21901FFFF0401BBF210011F
:1096C000FFFF04010A287201FFFF04010A2872014A
:1096D000FFFF04010A287201FFFF04010A2872013A
:1096E000FFFF04010A287201FFFF04010A2872012A
:1096F000FFFF04010A287201FFFF04010A2872011A
:10970000FFFF0401AA287201FFFF0401AA287201C9
:10971000FFFF0401AA287201FFFF0401AA287201B9
:10972000FFFF04010A247201FFFF0401BBF21001D4
:10973000FFFF0401BBF21901FFFF0401BBF210019E
:10974000FFFF04010A287201FFFF04010A287201C9
:10975000FFFF04010A287201FFFF04010A287201B9
:10976000FFFF04010A287201FFFF04010A287201A9
:10977000FFFF04010A287201FFFF04010A28720199
:10978000FFFF0401AA287201FFFF0401AA28720149
:10979000FFFF0401AA287201FFFF0401AA28720139
:1097A000FFFF04010A247201FFFF0401BBF2100154
:1097B000FFFF0401BBF21901FFFF0401BBF210011E
:1097C000FFFF04010A287201FFFF04010A28720149
:1097D000FFFF04010A287201FFFF04010A28720139
:1097E000FFFF04010A287201FFFF04010A28720129
:1097F000FFFF04010A287201FFFF04010A28720119
:10980000FFFF0401AA287201FFFF0401AA287201C8
:10981000FFFF0401AA287201FFFF0401AA287201B8
:10982000FFFF0401FE00FF01FFFF0401BBF2100176
:10983000FFFF0401BBF21901FFFF0401BBF210019D
:10984000FFFF04010A287201FFFF04010A287201C8
:10985000FFFF04010A287201FFFF04010A287201B8
:10986000FFFF04010A287201FFFF04010A287201A8
:10987000FFFF04010A287201FFFF04010A28720198
:10988000FFFF0401AA287201FFFF0401AA28720148
:10989000FFFF0401AA287201FFFF0401AA28720138
:1098A000FFFF0401FE00FF01FFFF0401BBF21001F6
:1098B000FFFF0401BBF21901FFFF0401BBF210011D
:1098C000FFFF04010A287201FFFF04010A28720148
:1098D000FFFF04010A287201FFFF04010A28720138
:1098E000FFFF04010A287201FFFF04010A28720128
:1098F000FFFF04010A287201FFFF04010A28720118
:10990000FFFF0401AA287201FFFF0401AA287201C7
:10991000FFFF0401AA287201FFFF0401AA287201B7
:10992000FFFF04010A247201FFFF0401BBF21001D2
:10993000FFFF0401BBF21901FFFF0401BBF210019C
:10994000FFFF04010A287201FFFF04010A287201C7
:10995000FFFF04010A287201FFFF04010A287201B7
:10996000FFFF04010A287201FFFF04010A287201A7
:10997000FFFF04010A287201FFFF04010A28720197
:10998000FFFF0401AA287201FFFF0401AA28720147
:10999000FFFF0401AA287201FFFF0401AA28720137
:1099A000FFFF04010A247201FFFF0401BBF2100152
:1099B000FFFF0401BBF21901FFFF0401BBF210011C
:1099C000FFFF04010A287201FFFF04010A28720147
:1099D000FFFF04010A287201FFFF04010A28720137
:1099E000FFFF04010A287201FFFF04010A28720127
:1099F000FFFF04010A287201FFFF04010A28720117
:109A0000FFFF0401AA287201FFFF0401AA287201C6
:109A1000FFFF0401AA287201FFFF0401AA287201B6
:109A2000FFFF0401FE00FF01FFFF0401BBF2100174
:109A3000FFFF0401BBF21901FFFF0401BBF210019B
:109A4000FFFF04010A287201FFFF04010A287201C6
:109A5000FFFF04010A287201FFFF04010A287201B6
:109A6000FFFF04010A287201FFFF04010A287201A6
:109A7000FFFF04010A287201FFFF04010A28720196
:109A8000FFFF0401AA287201FFFF0401AA28720146
:109A9000FFFF0401AA287201FFFF0401AA28720136
:109AA000FFFF0401FE00FF01FFFF0401BBF21001F4
:109AB000FFFF0401BBF21901FFFF0401BBF210011B
:109AC000FFFF04010A287201FFFF04010A28720146
:109AD000FFFF04010A287201FFFF04010A28720136
:109AE000FFFF04010A287201FFFF04010A28720126
:109AF000FFFF04010A287201FFFF04010A28720116
:109B0000FFFF0401AA287201FFFF0401AA287201C5
:109B1000FFFF0401AA287201FFFF0401AA287201B5
:109B2000FFFF04010A247201FFFF0401BBF21001D0
:109B3000FFFF0401BBF21901FFFF0401BBF210019A
:109B4000FFFF04010A287201FFFF04010A287201C5
:109B5000FFFF04010A287201FFFF04010A287201B5
:109B6000FFFF04010A287201FFFF04010A287201A5
:109B7000FFFF04010A287201FFFF04010A28720195
:109B8000FFFF0401AA287201FFFF0401AA28720145
:109B9000FFFF0401AA287201FFFF0401AA28720135
:109BA000FFFF04010A247201FFFF0401BBF2100150
:109BB000FFFF0401BBF21901FFFF0401BBF210011A
:109BC000FFFF04010A287201FFFF04010A28720145
:109BD000FFFF04010A287201FFFF04010A28720135
:109BE000FFFF04010A287201FFFF04010A28720125
:109BF000FFFF04010A287201FFFF04010A28720115
:109C0000FFFF0401AA287201FFFF0401AA287201C4
:109C1000FFFF0401AA287201FFFF0401AA287201B4
:109C2000FFFF0401FE00FF01FFFF0401BBF2100172
:109C3000FFFF0401BBF21901FFFF0401BBF2100199
:109C4000FFFF04010A287201FFFF04010A287201C4
:109C5000FFFF04010A287201FFFF04010A287201B4
:109C6000FFFF04010A287201FFFF04010A287201A4
:109C7000FFFF04010A287201FFFF04010A28720194
:109C8000FFFF0401AA287201FFFF0401AA28720144
:109C9000FFFF0401AA287201FFFF0401AA28720134
:109CA000FFFF0401FE00FF01FFFF0401BBF21001F2
:109CB000FFFF0401BBF21901FFFF0401BBF2100119
:109CC000FFFF04010A287201FFFF04010A28720144
:109CD000FFFF04010A287201FFFF04010A28720134
:109CE000FFFF04010A287201FFFF04010A28720124
:109CF000FFFF04010A287201FFFF04010A28720114
:109D0000FFFF0401AA287201FFFF0401AA287201C3
:109D1000FFFF0401AA287201FFFF0401AA287201B3
:109D2000FFFF04010A247201FFFF0401BBF21001CE
:109D3000FFFF0401BBF21901FFFF0401BBF2100198
:109D4000FFFF04010A287201FFFF04010A287201C3
:109D5000FFFF04010A287201FFFF04010A287201B3
:109D6000FFFF04010A287201FFFF04010A287201A3
:109D7000FFFF04010A287201FFFF04010A28720193
:109D8000FFFF0401AA287201FFFF0401AA28720143
:109D9000FFFF0401AA287201FFFF0401AA28720133
:109DA000FFFF04010A247201FFFF0401BBF210014E
:109DB000FFFF0401BBF21901FFFF0401BBF2100118
:109DC000FFFF04010A287201FFFF04010A28720143
:109DD000FFFF04010A287201FFFF04010A28720133
:109DE000FFFF04010A287201FFFF04010A28720123
:109DF000FFFF04010A287201FFFF04010A28720113
:109E0000FFFF0401AA287201FFFF0401AA287201C2
:109E1000FFFF0401AA287201FFFF0401AA287201B2
:109E2000FFFF0401FE00FF01FFFF0401BBF2100170
:109E3000FFFF0401BBF21901FFFF0401BBF2100197
:109E4000FFFF04010A287201FFFF04010A287201C2
:109E5000FFFF04010A287201FFFF04010A287201B2
:109E6000FFFF04010A287201FFFF04010A287201A2
:109E7000FFFF04010A287201FFFF04010A28720192
:109E8000FFFF0401AA287201FFFF0401AA28720142
:109E9000FFFF0401AA287201FFFF0401AA28720132
:109EA000FFFF0401FE00FF01FFFF0401BBF21001F0
:109EB000FFFF0401BBF21901FFFF0401BBF2100117
:109EC000FFFF04010A287201FFFF04010A28720142
:109ED000FFFF04010A287201FFFF04010A28720132
:109EE000FFFF04010A287201FFFF04010A28720122
:109EF000FFFF04010A287201FFFF04010A28720112
:109F0000FFFF0401AA287201FFFF0401AA287201C1
:109F1000FFFF0401AA287201FFFF0401AA287201B1
:109F2000FFFF04010A247201FFFF0401BBF21001CC
:109F3000FFFF0401BBF21901FFFF0401BBF2100196
:109F4000FFFF04010A287201FFFF04010A287201C1
:109F5000FFFF04010A287201FFFF04010A287201B1
:109F6000FFFF04010A287201FFFF04010A287201A1
:109F7000FFFF04010A287201FFFF04010A28720191
:109F8000FFFF0401AA287201FFFF0401AA28720141
:109F9000FFFF0401AA287201FFFF0401AA28720131
:109FA000FFFF04010A247201FFFF0401BBF210014C
:109FB000FFFF0401BBF21901FFFF0401BBF2100116
:109FC000FFFF04010A287201FFFF04010A28720141
:109FD000FFFF04010A287201FFFF04010A28720131
:109FE000FFFF04010A287201FFFF04010A28720121
:109FF000FFFF04010A287201FFFF04010A28720111
:10A00000FFFF0401AA287201FFFF0401AA287201C0
:10A01000FFFF0401AA287201FFFF0401AA287201B0
:10A02000FFFF0401FE00FF01FFFF0401BBF210016E
:10A03000FFFF0401BBF21901FFFF0401BBF2100195
:10A04000FFFF04010A287201FFFF04010A287201C0
:10A05000FFFF04010A287201FFFF04010A287201B0
:10A06000FFFF04010A287201FFFF04010A287201A0
:10A07000FFFF04010A287201FFFF04010A28720190
:10A08000FFFF0401AA287201FFFF0401AA28720140
:10A09000FFFF0401AA287201FFFF0401AA28720130
:10A0A000FFFF0401FE00FF01FFFF0401BBF21001EE
:10A0B000FFFF0401BBF21901FFFF0401BBF2100115
:10A0C000FFFF04010A287201FFFF04010A28720140
:10A0D000FFFF04010A287201FFFF04010A28720130
:10A0E000FFFF04010A287201FFFF04010A28720120
:10A0F000FFFF04010A287201FFFF04010A28720110
:10A10000FFFF0401AA287201FFFF0401AA287201BF
:10A11000FFFF0401AA287201FFFF0401AA287201AF
:10A12000FFFF04010A247201FFFF0401BBF21001CA
:10A13000FFFF0401BBF21901FFFF0401BBF2100194
:10A14000FFFF04010A287201FFFF04010A287201BF
:10A15000FFFF04010A287201FFFF04010A287201AF
:10A16000FFFF04010A287201FFFF04010A2872019F
:10A17000FFFF04010A287201FFFF04010A2872018F
:10A18000FFFF0401AA287201FFFF0401AA2872013F
:10A19000FFFF0401AA287201FFFF0401AA2872012F
:10A1A000FFFF04010A247201FFFF0401BBF210014A
:10A1B000FFFF0401BBF21901FFFF0401BBF2100114
:10A1C000FFFF04010A287201FFFF04010A2872013F
:10A1D000FFFF04010A287201FFFF04010A2872012F
:10A1E000FFFF04010A287201FFFF04010A2872011F
:10A1F000FFFF04010A287201FFFF04010A2872010F
:10A20000FFFF0401AA287201FFFF0401AA287201BE
:10A21000FFFF0401AA287201FFFF0401AA287201AE
:10A22000FFFF0401FE00FF01FFFF0401BBF210016C
:10A23000FFFF0401BBF21901FFFF0401BBF2100193
:10A24000FFFF04010A287201FFFF04010A287201BE
:10A25000FFFF04010A287201FFFF04010A287201AE
:10A26000FFFF04010A287201FFFF04010A2872019E
:10A27000FFFF04010A287201FFFF04010A2872018E
:10A28000FFFF0401AA287201FFFF0401AA2872013E
:10A29000FFFF0401AA287201FFFF0401AA2872012E
:10A2A000FFFF0401FE00FF01FFFF0401BBF21001EC
:10A2B000FFFF0401BBF21901FFFF0401BBF2100113
:10A2C000FFFF04010A287201FFFF04010A2872013E
:10A2D000FFFF04010A287201FFFF04010A2872012E
:10A2E000FFFF04010A287201FFFF04010A2872011E
:10A2F000FFFF04010A287201FFFF04010A2872010E
:10A30000FFFF0401AA287201FFFF0401AA287201BD
:10A31000FFFF0401AA287201FFFF0401AA287201AD
:10A32000FFFF04010A247201FFFF0401BBF21001C8
:10A33000FFFF0401BBF21901FFFF0401BBF2100192
:10A34000FFFF04010A287201FFFF04010A287201BD
:10A35000FFFF04010A287201FFFF04010A287201AD
:10A36000FFFF04010A287201FFFF04010A2872019D
:10A37000FFFF04010A287201FFFF04010A2872018D
:10A38000FFFF0401AA287201FFFF0401AA2872013D
:10A39000FFFF0401AA287201FFFF0401AA2872012D
:10A3A000FFFF04010A247201FFFF0401BBF2100148
:10A3B000FFFF0401BBF21901FFFF0401BBF2100112
:10A3C000FFFF04010A287201FFFF04010A2872013D
:10A3D000FFFF04010A287201FFFF04010A2872012D
:10A3E000FFFF04010A287201FFFF04010A2872011D
:10A3F000FFFF04010A287201FFFF04010A2872010D
:10A40000FFFF0401AA287201FFFF0401AA287201BC
:10A41000FFFF0401AA287201FFFF0401AA287201AC
:10A42000FFFF0401FE00FF01FFFF0401BBF210016A
:10A43000FFFF0401BBF21901FFFF0401BBF2100191
:10A44000FFFF04010A287201FFFF04010A287201BC
:10A45000FFFF04010A287201FFFF04010A287201AC
:10A46000FFFF04010A287201FFFF04010A2872019C
:10A47000FFFF04010A287201FFFF04010A2872018C
:10A48000FFFF0401AA287201FFFF0401AA2872013C
:10A49000FFFF0401AA287201FFFF0401AA2872012C
:10A4A000FFFF0401FE00FF01FFFF0401BBF21001EA
:10A4B000FFFF0401BBF21901FFFF0401BBF2100111
:10A4C000FFFF04010A287201FFFF04010A2872013C
:10A4D000FFFF04010A287201FFFF04010A2872012C
:10A4E000FFFF04010A287201FFFF04010A2872011C
:10A4F000FFFF04010A287201FFFF04010A2872010C
:10A50000FFFF0401AA287201FFFF0401AA287201BB
:10A51000FFFF0401AA287201FFFF0401AA287201AB
:10A52000FFFF04010A247201FFFF0401BBF21001C6
:10A53000FFFF0401BBF21901FFFF0401BBF2100190
:10A54000FFFF04010A287201FFFF04010A287201BB
:10A55000FFFF04010A287201FFFF04010A287201AB
:10A56000FFFF04010A287201FFFF04010A2872019B
:10A57000FFFF04010A287201FFFF04010A2872018B
:10A58000FFFF0401AA287201FFFF0401AA2872013B
:10A59000FFFF0401AA287201FFFF0401AA2872012B
:10A5A000FFFF04010A247201FFFF0401BBF2100146
:10A5B000FFFF0401BBF21901FFFF0401BBF2100110
:10A5C000FFFF04010A287201FFFF04010A2872013B
:10A5D000FFFF04010A287201FFFF04010A2872012B
:10A5E000FFFF04010A287201FFFF04010A2872011B
:10A5F000FFFF04010A287201FFFF04010A2872010B
:10A60000FFFF0401AA287201FFFF0401AA287201BA
:10A61000FFFF0401AA287201FFFF0401AA287201AA
:10A62000FFFF0401FE00FF01FFFF0401BBF2100168
:10A63000FFFF0401BBF21901FFFF0401BBF210018F
:10A64000FFFF04010A287201FFFF04010A287201BA
:10A65000FFFF04010A287201FFFF04010A287201AA
:10A66000FFFF04010A287201FFFF04010A2872019A
:10A67000FFFF04010A287201FFFF04010A2872018A
:10A68000FFFF0401AA287201FFFF0401AA2872013A
:10A69000FFFF0401AA287201FFFF0401AA2872012A
:10A6A000FFFF0401FE00FF01FFFF0401BBF21001E8
:10A6B000FFFF0401BBF21901FFFF0401BBF210010F
:10A6C000FFFF04010A287201FFFF04010A2872013A
:10A6D000FFFF04010A287201FFFF04010A2872012A
:10A6E000FFFF04010A287201FFFF04010A2872011A
:10A6F000FFFF04010A287201FFFF04010A2872010A
:10A70000FFFF0401AA287201FFFF0401AA287201B9
:10A71000FFFF0401AA287201FFFF0401AA287201A9
:10A72000FFFF04010A247201FFFF0401BBF21001C4
:10A73000FFFF0401BBF21901FFFF0401BBF210018E
:10A74000FFFF04010A287201FFFF04010A287201B9
:10A75000FFFF04010A287201FFFF04010A287201A9
:10A76000FFFF04010A287201FFFF04010A28720199
:10A77000FFFF04010A287201FFFF04010A28720189
:10A78000FFFF0401AA287201FFFF0401AA28720139
:10A79000FFFF0401AA287201FFFF0401AA28720129
:10A7A000FFFF04010A247201FFFF0401BBF2100144
:10A7B000FFFF0401BBF21901FFFF0401BBF210010E
:10A7C000FFFF04010A287201FFFF04010A28720139
:10A7D000FFFF04010A287201FFFF04010A28720129
:10A7E000FFFF04010A287201FFFF04010A28720119
:10A7F000FFFF04010A287201FFFF04010A28720109
:10A80000FFFF0401AA287201FFFF0401AA287201B8
:10A81000FFFF0401AA287201FFFF0401AA287201A8
:10A82000FFFF0401FE00FF01FFFF0401BBF2100166
:10A83000FFFF0401BBF21901FFFF0401BBF210018D
:10A84000FFFF04010A287201FFFF04010A287201B8
:10A85000FFFF04010A287201FFFF04010A287201A8
:10A86000FFFF04010A287201FFFF04010A28720198
:10A87000FFFF04010A287201FFFF04010A28720188
:10A88000FFFF0401AA287201FFFF0401AA28720138
:10A89000FFFF0401AA287201FFFF0401AA28720128
:10A8A000FFFF0401FE00FF01FFFF0401BBF21001E6
:10A8B000FFFF0401BBF21901FFFF0401BBF210010D
:10A8C000FFFF04010A287201FFFF04010A28720138
:10A8D000FFFF04010A287201FFFF04010A28720128
:10A8E000FFFF04010A287201FFFF04010A28720118
:10A8F000FFFF04010A287201FFFF04010A28720108
:10A90000FFFF0401AA287201FFFF0401AA287201B7
:10A91000FFFF0401AA287201FFFF0401AA287201A7
:10A92000FFFF04010A247201FFFF0401BBF21001C2
:10A93000FFFF0401BBF21901FFFF0401BBF210018C
:10A94000FFFF04010A287201FFFF04010A287201B7
:10A95000FFFF04010A287201FFFF04010A287201A7
:10A96000FFFF04010A287201FFFF04010A28720197
:10A97000FFFF04010A287201FFFF04010A28720187
:10A98000FFFF0401AA287201FFFF0401AA28720137
:10A99000FFFF0401AA287201FFFF0401AA28720127
:10A9A000FFFF04010A247201FFFF0401BBF2100142
:10A9B000FFFF0401BBF21901FFFF0401BBF210010C
:10A9C000FFFF04010A287201FFFF04010A28720137
:10A9D000FFFF04010A287201FFFF04010A28720127
:10A9E000FFFF04010A287201FFFF04010A28720117
:10A9F000FFFF04010A287201FFFF04010A28720107
:10AA0000FFFF0401AA287201FFFF0401AA287201B6
:10AA1000FFFF0401AA287201FFFF0401AA287201A6
:10AA2000FFFF0401FE00FF01FFFF0401BBF2100164
:10AA3000FFFF0401BBF21901FFFF0401BBF210018B
:10AA4000FFFF04010A287201FFFF04010A287201B6
:10AA5000FFFF04010A287201FFFF04010A287201A6
:10AA6000FFFF04010A287201FFFF04010A28720196
:10AA7000FFFF04010A287201FFFF04010A28720186
:10AA8000FFFF0401AA287201FFFF0401AA28720136
:10AA9000FFFF0401AA287201FFFF0401AA28720126
:10AAA000FFFF0401FE00FF01FFFF0401BBF21001E4
:10AAB000FFFF0401BBF21901FFFF0401BBF210010B
:10AAC000FFFF04010A287201FFFF04010A28720136
:10AAD000FFFF04010A287201FFFF04010A28720126
:10AAE000FFFF04010A287201FFFF04010A28720116
:10AAF000FFFF04010A287201FFFF04010A28720106
:10AB0000FFFF0401AA287201FFFF0401AA287201B5
:10AB1000FFFF0401AA287201FFFF0401AA287201A5
:10AB2000FFFF04010A247201FFFF0401BBF21001C0
:10AB3000FFFF0401BBF21901FFFF0401BBF210018A
:10AB4000FFFF04010A287201FFFF04010A287201B5
:10AB5000FFFF04010A287201FFFF04010A287201A5
:10AB6000FFFF04010A287201FFFF04010A28720195
:10AB7000FFFF04010A287201FFFF04010A28720185
:10AB8000FFFF0401AA287201FFFF0401AA28720135
:10AB9000FFFF0401AA287201FFFF0401AA28720125
:10ABA000FFFF04010A247201FFFF0401BBF2100140
:10ABB000FFFF0401BBF21901FFFF0401BBF210010A
:10ABC000FFFF04010A287201FFFF04010A28720135
:10ABD000FFFF04010A287201FFFF04010A28720125
:10ABE000FFFF04010A287201FFFF04010A28720115
:10ABF000FFFF04010A287201FFFF04010A28720105
:10AC0000FFFF0401AA287201FFFF0401AA287201B4
:10AC1000FFFF0401AA287201FFFF0401AA287201A4
:10AC2000FFFF0401FE00FF01FFFF0401BBF2100162
:10AC3000FFFF0401BBF21901FFFF0401BBF2100189
:10AC4000FFFF04010A287201FFFF04010A287201B4
:10AC5000FFFF04010A287201FFFF04010A287201A4
:10AC6000FFFF04010A287201FFFF04010A28720194
:10AC7000FFFF04010A287201FFFF04010A28720184
:10AC8000FFFF0401AA287201FFFF0401AA28720134
:10AC9000FFFF0401AA287201FFFF0401AA28720124
:10ACA000FFFF0401FE00FF01FFFF0401BBF21001E2
:10ACB000FFFF0401BBF21901FFFF0401BBF2100109
:10ACC000FFFF04010A287201FFFF04010A28720134
:10ACD000FFFF04010A287201FFFF04010A28720124
:10ACE000FFFF04010A287201FFFF04010A28720114
:10ACF000FFFF04010A287201FFFF04010A28720104
:10AD0000FFFF0401AA287201FFFF0401AA287201B3
:10AD1000FFFF0401AA287201FFFF0401AA287201A3
:10AD2000FFFF04010A247201FFFF0401BBF21001BE
:10AD3000FFFF0401BBF21901FFFF0401BBF2100188
:10AD4000FFFF04010A287201FFFF04010A287201B3
:10AD5000FFFF04010A287201FFFF04010A287201A3
:10AD6000FFFF04010A287201FFFF04010A28720193
:10AD7000FFFF04010A287201FFFF04010A28720183
:10AD8000FFFF0401AA287201FFFF0401AA28720133
:10AD9000FFFF0401AA287201FFFF0401AA28720123
:10ADA000FFFF04010A247201FFFF0401BBF210013E
:10ADB000FFFF0401BBF21901FFFF0401BBF2100108
:10ADC000FFFF04010A287201FFFF04010A28720133
:10ADD000FFFF04010A287201FFFF04010A28720123
:10ADE000FFFF04010A287201FFFF04010A28720113
:10ADF000FFFF04010A287201FFFF04010A28720103
:10AE0000FFFF0401AA287201FFFF0401AA287201B2
:10AE1000FFFF0401AA287201FFFF0401AA287201A2
:10AE2000FFFF0401FE00FF01FFFF0401BBF2100160
:10AE3000FFFF0401BBF21901FFFF0401BBF2100187
:10AE4000FFFF04010A287201FFFF04010A287201B2
:10AE5000FFFF04010A287201FFFF04010A287201A2
:10AE6000FFFF04010A287201FFFF04010A28720192
:10AE7000FFFF04010A287201FFFF04010A28720182
:10AE8000FFFF0401AA287201FFFF0401AA28720132
:10AE9000FFFF0401AA287201FFFF0401AA28720122
:10AEA000FFFF0401FE00FF01FFFF0401BBF21001E0
:10AEB000FFFF0401BBF21901FFFF0401BBF2100107
:10AEC000FFFF04010A287201FFFF04010A28720132
:10AED000FFFF04010A287201FFFF04010A28720122
:10AEE000FFFF04010A287201FFFF04010A28720112
:10AEF000FFFF04010A287201FFFF04010A28720102
:10AF0000FFFF0401AA287201FFFF0401AA287201B1
:10AF1000FFFF0401AA287201FFFF0401AA287201A1
:10AF2000FFFF04010A247201FFFF0401BBF21001BC
:10AF3000FFFF0401BBF21901FFFF0401BBF2100186
:10AF4000FFFF04010A287201FFFF04010A287201B1
:10AF5000FFFF04010A287201FFFF04010A287201A1
:10AF6000FFFF04010A287201FFFF04010A28720191
:10AF7000FFFF04010A287201FFFF04010A28720181
:10AF8000FFFF0401AA287201FFFF0401AA28720131
:10AF9000FFFF0401AA287201FFFF0401AA28720121
:10AFA000FFFF04010A247201FFFF0401BBF210013C
:10AFB000FFFF0401BBF21901FFFF0401BBF2100106
:10AFC000FFFF04010A287201FFFF04010A28720131
:10AFD000FFFF04010A287201FFFF04010A28720121
:10AFE000FFFF04010A287201FFFF04010A28720111
:10AFF000FFFF04010A287201FFFF04010A28720101
:10B00000FFFF0401AA287201FFFF0401AA287201B0
:10B01000FFFF0401AA287201FFFF0401AA287201A0
:10B02000FFFF0401FE00FF01FFFF0401BBF210015E
:10B03000FFFF0401BBF21901FFFF0401BBF2100185
:10B04000FFFF04010A287201FFFF04010A287201B0
:10B05000FFFF04010A287201FFFF04010A287201A0
:10B06000FFFF04010A287201FFFF04010A28720190
:10B07000FFFF04010A287201FFFF04010A28720180
:10B08000FFFF0401AA287201FFFF0401AA28720130
:10B09000FFFF0401AA287201FFFF0401AA28720120
:10B0A000FFFF0401FE00FF01FFFF0401BBF21001DE
:10B0B000FFFF0401BBF21901FFFF0401BBF2100105
:10B0C000FFFF04010A287201FFFF04010A28720130
:10B0D000FFFF04010A287201FFFF04010A28720120
:10B0E000FFFF04010A287201FFFF04010A28720110
:10B0F000FFFF04010A287201FFFF04010A28720100
:10B10000FFFF0401AA287201FFFF0401AA287201AF
:10B11000FFFF0401AA287201FFFF0401AA2872019F
:10B12000FFFF04010A247201FFFF0401BBF21001BA
:10B13000FFFF0401BBF21901FFFF0401BBF2100184
:10B14000FFFF04010A287201FFFF04010A287201AF
:10B15000FFFF04010A287201FFFF04010A2872019F
:10B16000FFFF04010A287201FFFF04010A2872018F
:10B17000FFFF04010A287201FFFF04010A2872017F
:10B18000FFFF0401AA287201FFFF0401AA2872012F
:10B19000FFFF0401AA287201FFFF0401AA2872011F
:10B1A000FFFF04010A247201FFFF0401BBF210013A
:10B1B000FFFF0401BBF21901FFFF0401BBF2100104
:10B1C000FFFF04010A287201FFFF04010A2872012F
:10B1D000FFFF04010A287201FFFF04010A2872011F
:10B1E000FFFF04010A287201FFFF04010A2872010F
:10B1F000FFFF04010A287201FFFF04010A287201FF
:10B20000FFFF0401AA287201FFFF0401AA287201AE
:10B21000FFFF0401AA287201FFFF0401AA2872019E
:10B22000FFFF0401FE00FF01FFFF0401BBF210015C
:10B23000FFFF0401BBF21901FFFF0401BBF2100183
:10B24000FFFF04010A287201FFFF04010A287201AE
:10B25000FFFF04010A287201FFFF04010A2872019E
:10B26000FFFF04010A287201FFFF04010A2872018E
:10B27000FFFF04010A287201FFFF04010A2872017E
:10B28000FFFF0401AA287201FFFF0401AA2872012E
:10B29000FFFF0401AA287201FFFF0401AA2872011E
:10B2A000FFFF0401FE00FF01FFFF0401BBF21001DC
:10B2B000FFFF0401BBF21901FFFF0401BBF2100103
:10B2C000FFFF04010A287201FFFF04010A2872012E
:10B2D000FFFF04010A287201FFFF04010A2872011E
:10B2E000FFFF04010A287201FFFF04010A2872010E
:10B2F000FFFF04010A287201FFFF04010A287201FE
:10B30000FFFF0401AA287201FFFF0401AA287201AD
:10B31000FFFF0401AA287201FFFF0401AA2872019D
:10B32000FFFF04010A247201FFFF0401BBF21001B8
:10B33000FFFF0401BBF21901FFFF0401BBF2100182
:10B34000FFFF04010A287201FFFF04010A287201AD
:10B35000FFFF04010A287201FFFF04010A2872019D
:10B36000FFFF04010A287201FFFF04010A2872018D
:10B37000FFFF04010A287201FFFF04010A2872017D
:10B38000FFFF0401AA287201FFFF0401AA2872012D
:10B39000FFFF0401AA287201FFFF0401AA2872011D
:10B3A000FFFF04010A247201FFFF0401BBF2100138
:10B3B000FFFF0401BBF21901FFFF0401BBF2100102
:10B3C000FFFF04010A287201FFFF04010A2872012D
:10B3D000FFFF04010A287201FFFF04010A2872011D
:10B3E000FFFF04010A287201FFFF04010A2872010D
:10B3F000FFFF04010A287201FFFF04010A287201FD
:10B40000FFFF0401AA287201FFFF0401AA287201AC
:10B41000FFFF0401AA287201FFFF0401AA2872019C
:10B42000FFFF0401FE00FF01FFFF0401BBF210015A
:10B43000FFFF0401BBF21901FFFF0401BBF2100181
:10B44000FFFF04010A287201FFFF04010A287201AC
:10B45000FFFF04010A287201FFFF04010A2872019C
:10B46000FFFF04010A287201FFFF04010A2872018C
:10B47000FFFF04010A287201FFFF04010A2872017C
:10B48000FFFF0401AA287201FFFF0401AA2872012C
:10B49000FFFF0401AA287201FFFF0401AA2872011C
:10B4A000FFFF0401FE00FF01FFFF0401BBF21001DA
:10B4B000FFFF0401BBF21901FFFF0401BBF2100101
:10B4C000FFFF04010A287201FFFF04010A2872012C
:10B4D000FFFF04010A287201FFFF04010A2872011C
:10B4E000FFFF04010A287201FFFF04010A2872010C
:10B4F000FFFF04010A287201FFFF04010A287201FC
:10B50000FFFF0401AA287201FFFF0401AA287201AB
:10B51000FFFF0401AA287201FFFF0401AA2872019B
:10B52000FFFF04010A247201FFFF0401BBF21001B6
:10B53000FFFF0401BBF21901FFFF0401BBF2100180
:10B54000FFFF04010A287201FFFF04010A287201AB
:10B55000FFFF04010A287201FFFF04010A2872019B
:10B56000FFFF04010A287201FFFF04010A2872018B
:10B57000FFFF04010A287201FFFF04010A2872017B
:10B58000FFFF0401AA287201FFFF0401AA2872012B
:10B59000FFFF0401AA287201FFFF0401AA2872011B
:10B5A000FFFF04010A247201FFFF0401BBF2100136
:10B5B000FFFF0401BBF21901FFFF0401BBF2100100
:10B5C000FFFF04010A287201FFFF04010A2872012B
:10B5D000FFFF04010A287201FFFF04010A2872011B
:10B5E000FFFF04010A287201FFFF04010A2872010B
:10B5F000FFFF04010A287201FFFF04010A287201FB
:10B60000FFFF0401AA287201FFFF0401AA287201AA
:10B61000FFFF0401AA287201FFFF0401AA2872019A
:10B62000FFFF0401FE00FF01FFFF0401BBF2100158
:10B63000FFFF0401BBF21901FFFF0401BBF210017F
:10B64000FFFF04010A287201FFFF04010A287201AA
:10B65000FFFF04010A287201FFFF04010A2872019A
:10B66000FFFF04010A287201FFFF04010A2872018A
:10B67000FFFF04010A287201FFFF04010A2872017A
:10B68000FFFF0401AA287201FFFF0401AA2872012A
:10B69000FFFF0401AA287201FFFF0401AA2872011A
:10B6A000FFFF0401FE00FF01FFFF0401BBF21001D8
:10B6B000FFFF0401BBF21901FFFF0401BBF21001FF
:10B6C000FFFF04010A287201FFFF04010A2872012A
:10B6D000FFFF04010A287201FFFF04010A2872011A
:10B6E000FFFF04010A287201FFFF04010A2872010A
:10B6F000FFFF04010A287201FFFF04010A287201FA
:10B70000FFFF0401AA287201FFFF0401AA287201A9
:10B71000FFFF0401AA287201FFFF0401AA28720199
:10B72000FFFF04010A247201FFFF0401BBF21001B4
:10B73000FFFF0401BBF21901FFFF0401BBF210017E
:10B74000FFFF04010A287201FFFF04010A287201A9
:10B75000FFFF04010A287201FFFF04010A28720199
:10B76000FFFF04010A287201FFFF04010A28720189
:10B77000FFFF04010A287201FFFF04010A28720179
:10B78000FFFF0401AA287201FFFF0401AA28720129
:10B79000FFFF0401AA287201FFFF0401AA28720119
:10B7A000FFFF04010A247201FFFF0401BBF2100134
:10B7B000FFFF0401BBF21901FFFF0401BBF21001FE
:10B7C000FFFF04010A287201FFFF04010A28720129
:10B7D000FFFF04010A287201FFFF04010A28720119
:10B7E000FFFF04010A287201FFFF04010A28720109
:10B7F000FFFF04010A287201FFFF04010A287201F9
:10B80000FFFF0401AA287201FFFF0401AA287201A8
:10B81000FFFF0401AA287201FFFF0401AA28720198
:10B82000FFFF0401FE00FF01FFFF0401BBF2100156
:10B83000FFFF0401BBF21901FFFF0401BBF210017D
:10B84000FFFF04010A287201FFFF04010A287201A8
:10B85000FFFF04010A287201FFFF04010A28720198
:10B86000FFFF04010A287201FFFF04010A28720188
:10B87000FFFF04010A287201FFFF04010A28720178
:10B88000FFFF0401AA287201FFFF0401AA28720128
:10B89000FFFF0401AA287201FFFF0401AA28720118
:10B8A000FFFF0401FE00FF01FFFF0401BBF21001D6
:10B8B000FFFF0401BBF21901FFFF0401BBF21001FD
:10B8C000FFFF04010A287201FFFF04010A28720128
:10B8D000FFFF04010A287201FFFF04010A28720118
:10B8E000FFFF04010A287201FFFF04010A28720108
:10B8F000FFFF04010A287201FFFF04010A287201F8
:10B90000FFFF0401AA287201FFFF0401AA287201A7
:10B91000FFFF0401AA287201FFFF0401AA28720197
:10B92000FFFF04010A247201FFFF0401BBF21001B2
:10B93000FFFF0401BBF21901FFFF0401BBF210017C
:10B94000FFFF04010A287201FFFF04010A287201A7
:10B95000FFFF04010A287201FFFF04010A28720197
:10B96000FFFF04010A287201FFFF04010A28720187
:10B97000FFFF04010A287201FFFF04010A28720177
:10B98000FFFF0401AA287201FFFF0401AA28720127
:10B99000FFFF0401AA287201FFFF0401AA28720117
:10B9A000FFFF04010A247201FFFF0401BBF2100132
:10B9B000FFFF0401BBF21901FFFF0401BBF21001FC
:10B9C000FFFF04010A287201FFFF04010A28720127
:10B9D000FFFF04010A287201FFFF04010A28720117
:10B9E000FFFF04010A287201FFFF04010A28720107
:10B9F000FFFF04010A287201FFFF04010A287201F7
:10BA0000FFFF0401AA287201FFFF0401AA287201A6
:10BA1000FFFF0401AA287201FFFF0401AA28720196
:10BA2000FFFF0401FE00FF01FFFF0401BBF2100154
:10BA3000FFFF0401BBF21901FFFF0401BBF210017B
:10BA4000FFFF04010A287201FFFF04010A287201A6
:10BA5000FFFF04010A287201FFFF04010A28720196
:10BA6000FFFF04010A287201FFFF04010A28720186
:10BA7000FFFF04010A287201FFFF04010A28720176
:10BA8000FFFF0401AA287201FFFF0401AA28720126
:10BA9000FFFF0401AA287201FFFF0401AA28720116
:10BAA000FFFF0401FE00FF01FFFF0401BBF21001D4
:10BAB000FFFF0401BBF21901FFFF0401BBF21001FB
:10BAC000FFFF04010A287201FFFF04010A28720126
:10BAD000FFFF04010A287201FFFF04010A28720116
:10BAE000FFFF04010A287201FFFF04010A28720106
:10BAF000FFFF04010A287201FFFF04010A287201F6
:10BB0000FFFF0401AA287201FFFF0401AA287201A5
:10BB1000FFFF0401AA287201FFFF0401AA28720195
:10BB2000FFFF04010A247201FFFF0401BBF21001B0
:10BB3000FFFF0401BBF21901FFFF0401BBF210017A
:10BB4000FFFF04010A287201FFFF04010A287201A5
:10BB5000FFFF04010A287201FFFF04010A28720195
:10BB6000FFFF04010A287201FFFF04010A28720185
:10BB7000FFFF04010A287201FFFF04010A28720175
:10BB8000FFFF0401AA287201FFFF0401AA28720125
:10BB9000FFFF0401AA287201FFFF0401AA28720115
:10BBA000FFFF04010A247201FFFF0401BBF2100130
:10BBB000FFFF0401BBF21901FFFF0401BBF21001FA
:10BBC000FFFF04010A287201FFFF04010A28720125
:10BBD000FFFF04010A287201FFFF04010A28720115
:10BBE000FFFF04010A287201FFFF04010A28720105
:10BBF000FFFF04010A287201FFFF04010A287201F5
:10BC0000FFFF0401AA287201FFFF0401AA287201A4
:10BC1000FFFF0401AA287201FFFF0401AA28720194
:10BC2000FFFF0401FE00FF01FFFF0401BBF2100152
:10BC3000FFFF0401BBF21901FFFF0401BBF2100179
:10BC4000FFFF04010A287201FFFF04010A287201A4
:10BC5000FFFF04010A287201FFFF04010A28720194
:10BC6000FFFF04010A287201FFFF04010A28720184
:10BC7000FFFF04010A287201FFFF04010A28720174
:10BC8000FFFF0401AA287201FFFF0401AA28720124
:10BC9000FFFF0401AA287201FFFF0401AA28720114
:10BCA000FFFF0401FE00FF01FFFF0401BBF21001D2
:10BCB000FFFF0401BBF21901FFFF0401BBF21001F9
:10BCC000FFFF04010A287201FFFF04010A28720124
:10BCD000FFFF04010A287201FFFF04010A28720114
:10BCE000FFFF04010A287201FFFF04010A28720104
:10BCF000FFFF04010A287201FFFF04010A287201F4
:10BD0000FFFF0401AA287201FFFF0401AA287201A3
:10BD1000FFFF0401AA287201FFFF0401AA28720193
:10BD2000FFFF04010A247201FFFF0401BBF21001AE
:10BD3000FFFF0401BBF21901FFFF0401BBF2100178
:10BD4000FFFF04010A287201FFFF04010A287201A3
:10BD5000FFFF04010A287201FFFF04010A28720193
:10BD6000FFFF04010A287201FFFF04010A28720183
:10BD7000FFFF04010A287201FFFF04010A28720173
:10BD8000FFFF0401AA287201FFFF0401AA28720123
:10BD9000FFFF0401AA287201FFFF0401AA28720113
:10BDA000FFFF04010A247201FFFF0401BBF210012E
:10BDB000FFFF0401BBF21901FFFF0401BBF21001F8
:10BDC000FFFF04010A287201FFFF04010A28720123
:10BDD000FFFF04010A287201FFFF04010A28720113
:10BDE000FFFF04010A287201FFFF04010A28720103
:10BDF000FFFF04010A287201FFFF04010A287201F3
:10BE0000FFFF0401AA287201FFFF0401AA287201A2
:10BE1000FFFF0401AA287201FFFF0401AA28720192
:10BE2000FFFF0401FE00FF01FFFF0401BBF2100150
:10BE3000FFFF0401BBF21901FFFF0401BBF2100177
:10BE4000FFFF04010A287201FFFF04010A287201A2
:10BE5000FFFF04010A287201FFFF04010A28720192
:10BE6000FFFF04010A287201FFFF04010A28720182
:10BE7000FFFF04010A287201FFFF04010A28720172
:10BE8000FFFF0401AA287201FFFF0401AA28720122
:10BE9000FFFF0401AA287201FFFF0401AA28720112
:10BEA000FFFF0401FE00FF01FFFF0401BBF21001D0
:10BEB000FFFF0401BBF21901FFFF0401BBF21001F7
:10BEC000FFFF04010A287201FFFF04010A28720122
:10BED000FFFF04010A287201FFFF04010A28720112
:10BEE000FFFF04010A287201FFFF04010A28720102
:10BEF000FFFF04010A287201FFFF04010A287201F2
:10BF0000FFFF0401AA287201FFFF0401AA287201A1
:10BF1000FFFF0401AA287201FFFF0401AA28720191
:10BF2000FFFF04010A247201FFFF0401BBF21001AC
:10BF3000FFFF0401BBF21901FFFF0401BBF2100176
:10BF4000FFFF04010A287201FFFF04010A287201A1
:10BF5000FFFF04010A287201FFFF04010A28720191
:10BF6000FFFF04010A287201FFFF04010A28720181
:10BF7000FFFF04010A287201FFFF04010A28720171
:10BF8000FFFF0401AA287201FFFF0401AA28720121
:10BF9000FFFF0401AA287201FFFF0401AA28720111
:10BFA000FFFF04010A247201FFFF0401BBF210012C
:10BFB000FFFF0401BBF21901FFFF0401BBF21001F6
:10BFC000FFFF04010A287201FFFF04010A28720121
:10BFD000FFFF04010A287201FFFF04010A28720111
:10BFE000FFFF04010A287201FFFF04010A28720101
:10BFF000FFFF04010A287201FFFF04010A287201F1
:10C00000FFFF0401AA287201FFFF0401AA287201A0
:10C01000FFFF0401AA287201FFFF0401AA28720190
:10C02000FFFF0401FE00FF01FFFF0401BBF210014E
:10C03000FFFF0401BBF21901FFFF0401BBF2100175
:10C04000FFFF04010A287201FFFF04010A287201A0
:10C05000FFFF04010A287201FFFF04010A28720190
:10C06000FFFF04010A287201FFFF04010A28720180
:10C07000FFFF04010A287201FFFF04010A28720170
:10C08000FFFF0401AA287201FFFF0401AA28720120
:10C09000FFFF0401AA287201FFFF0401AA28720110
:10C0A000FFFF0401FE00FF01FFFF0401BBF21001CE
:10C0B000FFFF0401BBF21901FFFF0401BBF21001F5
:10C0C000FFFF04010A287201FFFF04010A28720120
:10C0D000FFFF04010A287201FFFF04010A28720110
:10C0E000FFFF04010A287201FFFF04010A28720100
:10C0F000FFFF04010A287201FFFF04010A287201F0
:10C10000FFFF0401AA287201FFFF0401AA2872019F
:10C11000FFFF0401AA287201FFFF0401AA2872018F
:10C12000FFFF04010A247201FFFF0401BBF21001AA
:10C13000FFFF0401BBF21901FFFF0401BBF2100174
:10C14000FFFF04010A287201FFFF04010A2872019F
:10C15000FFFF04010A287201FFFF04010A2872018F
:10C16000FFFF04010A287201FFFF04010A2872017F
:10C17000FFFF04010A287201FFFF04010A2872016F
:10C18000FFFF0401AA287201FFFF0401AA2872011F
:10C19000FFFF0401AA287201FFFF0401AA2872010F
:10C1A000FFFF04010A247201FFFF0401BBF210012A
:10C1B000FFFF0401BBF21901FFFF0401BBF21001F4
:10C1C000FFFF04010A287201FFFF04010A2872011F
:10C1D000FFFF04010A287201FFFF04010A2872010F
:10C1E000FFFF04010A287201FFFF04010A287201FF
:10C1F000FFFF04010A287201FFFF04010A287201EF
:10C20000FFFF0401AA287201FFFF0401AA2872019E
:10C21000FFFF0401AA287201FFFF0401AA2872018E
:10C22000FFFF0401FE00FF01FFFF0401BBF210014C
:10C23000FFFF0401BBF21901FFFF0401BBF2100173
:10C24000FFFF04010A287201FFFF04010A2872019E
:10C25000FFFF04010A287201FFFF04010A2872018E
:10C26000FFFF04010A287201FFFF04010A2872017E
:10C27000FFFF04010A287201FFFF04010A2872016E
:10C28000FFFF0401AA287201FFFF0401AA2872011E
:10C29000FFFF0401AA287201FFFF0401AA2872010E
:10C2A000FFFF0401FE00FF01FFFF0401BBF21001CC
:10C2B000FFFF0401BBF21901FFFF0401BBF21001F3
:10C2C000FFFF04010A287201FFFF04010A2872011E
:10C2D000FFFF04010A287201FFFF04010A2872010E
:10C2E000FFFF04010A287201FFFF04010A287201FE
:10C2F000FFFF04010A287201FFFF04010A287201EE
:10C30000FFFF0401AA287201FFFF0401AA2872019D
:10C31000FFFF0401AA287201FFFF0401AA2872018D
:10C32000FFFF04010A247201FFFF0401BBF21001A8
:10C33000FFFF0401BBF21901FFFF0401BBF2100172
:10C34000FFFF04010A287201FFFF04010A2872019D
:10C35000FFFF04010A287201FFFF04010A2872018D
:10C36000FFFF04010A287201FFFF04010A2872017D
:10C37000FFFF04010A287201FFFF04010A2872016D
:10C38000FFFF0401AA287201FFFF0401AA2872011D
:10C39000FFFF0401AA287201FFFF0401AA2872010D
:10C3A000FFFF04010A247201FFFF0401BBF2100128
:10C3B000FFFF0401BBF21901FFFF0401BBF21001F2
:10C3C000FFFF04010A287201FFFF04010A2872011D
:10C3D000FFFF04010A287201FFFF04010A2872010D
:10C3E000FFFF04010A287201FFFF04010A287201FD
:10C3F000FFFF04010A287201FFFF04010A287201ED
:10C40000FFFF0401AA287201FFFF0401AA2872019C
:10C41000FFFF0401AA287201FFFF0401AA2872018C
:10C42000FFFF0401FE00FF01FFFF0401BBF210014A
:10C43000FFFF0401BBF21901FFFF0401BBF2100171
:10C44000FFFF04010A287201FFFF04010A2872019C
:10C45000FFFF04010A287201FFFF04010A2872018C
:10C46000FFFF04010A287201FFFF04010A2872017C
:10C47000FFFF04010A287201FFFF04010A2872016C
:10C48000FFFF0401AA287201FFFF0401AA2872011C
:10C49000FFFF0401AA287201FFFF0401AA2872010C
:10C4A000FFFF0401FE00FF01FFFF0401BBF21001CA
:10C4B000FFFF0401BBF21901FFFF0401BBF21001F1
:10C4C000FFFF04010A287201FFFF04010A2872011C
:10C4D000FFFF04010A287201FFFF04010A2872010C
:10C4E000FFFF04010A287201FFFF04010A287201FC
:10C4F000FFFF04010A287201FFFF04010A287201EC
:10C50000FFFF0401AA287201FFFF0401AA2872019B
:10C51000FFFF0401AA287201FFFF0401AA2872018B
:10C52000FFFF04010A247201FFFF0401BBF21001A6
:10C53000FFFF0401BBF21901FFFF0401BBF2100170
:10C54000FFFF04010A287201FFFF04010A2872019B
:10C55000FFFF04010A287201FFFF04010A2872018B
:10C56000FFFF04010A287201FFFF04010A2872017B
:10C57000FFFF04010A287201FFFF04010A2872016B
:10C58000FFFF0401AA287201FFFF0401AA2872011B
:10C59000FFFF0401AA287201FFFF0401AA2872010B
:10C5A000FFFF04010A247201FFFF0401BBF2100126
:10C5B000FFFF0401BBF21901FFFF0401BBF21001F0
:10C5C000FFFF04010A287201FFFF04010A2872011B
:10C5D000FFFF04010A287201FFFF04010A2872010B
:10C5E000FFFF04010A287201FFFF04010A287201FB
:10C5F000FFFF04010A287201FFFF04010A287201EB
:10C60000FFFF0401AA287201FFFF0401AA2872019A
:10C61000FFFF0401AA287201FFFF0401AA2872018A
:10C62000FFFF0401FE00FF01FFFF0401BBF2100148
:10C63000FFFF0401BBF21901FFFF0401BBF210016F
:10C64000FFFF04010A287201FFFF04010A2872019A
:10C65000FFFF04010A287201FFFF04010A2872018A
:10C66000FFFF04010A287201FFFF04010A2872017A
:10C67000FFFF04010A287201FFFF04010A2872016A
:10C68000FFFF0401AA287201FFFF0401AA2872011A
:10C69000FFFF0401AA287201FFFF0401AA2872010A
:10C6A000FFFF0401FE00FF01FFFF0401BBF21001C8
:10C6B000FFFF0401BBF21901FFFF0401BBF21001EF
:10C6C000FFFF04010A287201FFFF04010A2872011A
:10C6D000FFFF04010A287201FFFF04010A2872010A
:10C6E000FFFF04010A287201FFFF04010A287201FA
:10C6F000FFFF04010A287201FFFF04010A287201EA
:10C70000FFFF0401AA287201FFFF0401AA28720199
:10C71000FFFF0401AA287201FFFF0401AA28720189
:10C72000FFFF04010A247201FFFF0401BBF21001A4
:10C73000FFFF0401BBF21901FFFF0401BBF210016E
:10C74000FFFF04010A287201FFFF04010A28720199
:10C75000FFFF04010A287201FFFF04010A28720189
:10C76000FFFF04010A287201FFFF04010A28720179
:10C77000FFFF04010A287201FFFF04010A28720169
:10C78000FFFF0401AA287201FFFF0401AA28720119
:10C79000FFFF0401AA287201FFFF0401AA28720109
:10C7A000FFFF04010A247201FFFF0401BBF2100124
:10C7B000FFFF0401BBF21901FFFF0401BBF21001EE
:10C7C000FFFF04010A287201FFFF04010A28720119
:10C7D000FFFF04010A287201FFFF04010A28720109
:10C7E000FFFF04010A287201FFFF04010A287201F9
:10C7F000FFFF04010A287201FFFF04010A287201E9
:10C80000FFFF0401AA287201FFFF0401AA28720198
:10C81000FFFF0401AA287201FFFF0401AA28720188
:10C82000FFFF0401FE00FF01FFFF0401BBF2100146
:10C83000FFFF0401BBF21901FFFF0401BBF210016D
:10C84000FFFF04010A287201FFFF04010A28720198
:10C85000FFFF04010A287201FFFF04010A28720188
:10C86000FFFF04010A287201FFFF04010A28720178
:10C87000FFFF04010A287201FFFF04010A28720168
:10C88000FFFF0401AA287201FFFF0401AA28720118
:10C89000FFFF0401AA287201FFFF0401AA28720108
:10C8A000FFFF0401FE00FF01FFFF0401BBF21001C6
:10C8B000FFFF0401BBF21901FFFF0401BBF21001ED
:10C8C000FFFF04010A287201FFFF04010A28720118
:10C8D000FFFF04010A287201FFFF04010A28720108
:10C8E000FFFF04010A287201FFFF04010A287201F8
:10C8F000FFFF04010A287201FFFF04010A287201E8
:10C90000FFFF0401AA287201FFFF0401AA28720197
:10C91000FFFF0401AA287201FFFF0401AA28720187
:10C92000FFFF04010A247201FFFF0401BBF21001A2
:10C93000FFFF0401BBF21901FFFF0401BBF210016C
:10C94000FFFF04010A287201FFFF04010A28720197
:10C95000FFFF04010A287201FFFF04010A28720187
:10C96000FFFF04010A287201FFFF04010A28720177
:10C97000FFFF04010A287201FFFF04010A28720167
:10C98000FFFF0401AA287201FFFF0401AA28720117
:10C99000FFFF0401AA287201FFFF0401AA28720107
:10C9A000FFFF04010A247201FFFF0401BBF2100122
:10C9B000FFFF0401BBF21901FFFF0401BBF21001EC
:10C9C000FFFF04010A287201FFFF04010A28720117
:10C9D000FFFF04010A287201FFFF04010A28720107
:10C9E000FFFF04010A287201FFFF04010A287201F7
:10C9F000FFFF04010A287201FFFF04010A287201E7
:10CA0000FFFF0401AA287201FFFF0401AA28720196
:10CA1000FFFF0401AA287201FFFF0401AA28720186
:10CA2000FFFF0401FE00FF01FFFF0401BBF2100144
:10CA3000FFFF0401BBF21901FFFF0401BBF210016B
:10CA4000FFFF04010A287201FFFF04010A28720196
:10CA5000FFFF04010A287201FFFF04010A28720186
:10CA6000FFFF04010A287201FFFF04010A28720176
:10CA7000FFFF04010A287201FFFF04010A28720166
:10CA8000FFFF0401AA287201FFFF0401AA28720116
:10CA9000FFFF0401AA287201FFFF0401AA28720106
:10CAA000FFFF0401FE00FF01FFFF0401BBF21001C4
:10CAB000FFFF0401BBF21901FFFF0401BBF21001EB
:10CAC000FFFF04010A287201FFFF04010A28720116
:10CAD000FFFF04010A287201FFFF04010A28720106
:10CAE000FFFF04010A287201FFFF04010A287201F6
:10CAF000FFFF04010A287201FFFF04010A287201E6
:10CB0000FFFF0401AA287201FFFF0401AA28720195
:10CB1000FFFF0401AA287201FFFF0401AA28720185
:10CB2000FFFF04010A247201FFFF0401BBF21001A0
:10CB3000FFFF0401BBF21901FFFF0401BBF210016A
:10CB4000FFFF04010A287201FFFF04010A28720195
:10CB5000FFFF04010A287201FFFF04010A28720185
:10CB6000FFFF04010A287201FFFF04010A28720175
:10CB7000FFFF04010A287201FFFF04010A28720165
:10CB8000FFFF0401AA287201FFFF0401AA28720115
:10CB9000FFFF0401AA287201FFFF0401AA28720105
:10CBA000FFFF04010A247201FFFF0401BBF2100120
:10CBB000FFFF0401BBF21901FFFF0401BBF21001EA
:10CBC000FFFF04010A287201FFFF04010A28720115
:10CBD000FFFF04010A287201FFFF04010A28720105
:10CBE000FFFF04010A287201FFFF04010A287201F5
:10CBF000FFFF04010A287201FFFF04010A287201E5
:10CC0000FFFF0401AA287201FFFF0401AA28720194
:10CC1000FFFF0401AA287201FFFF0401AA28720184
:10CC2000FFFF0401FE00FF01FFFF0401BBF2100142
:10CC3000FFFF0401BBF21901FFFF0401BBF2100169
:10CC4000FFFF04010A287201FFFF04010A28720194
:10CC5000FFFF04010A287201FFFF04010A28720184
:10CC6000FFFF04010A287201FFFF04010A28720174
:10CC7000FFFF04010A287201FFFF04010A28720164
:10CC8000FFFF0401AA287201FFFF0401AA28720114
:10CC9000FFFF0401AA287201FFFF0401AA28720104
:10CCA000FFFF0401FE00FF01FFFF0401BBF21001C2
:10CCB000FFFF0401BBF21901FFFF0401BBF21001E9
:10CCC000FFFF04010A287201FFFF04010A28720114
:10CCD000FFFF04010A287201FFFF04010A28720104
:10CCE000FFFF04010A287201FFFF04010A287201F4
:10CCF000FFFF04010A287201FFFF04010A287201E4
:10CD0000FFFF0401AA287201FFFF0401AA28720193
:10CD1000FFFF0401AA287201FFFF0401AA28720183
:10CD2000FFFF04010A247201FFFF0401BBF210019E
:10CD3000FFFF0401BBF21901FFFF0401BBF2100168
:10CD4000FFFF04010A287201FFFF04010A28720193
:10CD5000FFFF04010A287201FFFF04010A28720183
:10CD6000FFFF04010A287201FFFF04010A28720173
:10CD7000FFFF04010A287201FFFF04010A28720163
:10CD8000FFFF0401AA287201FFFF0401AA28720113
:10CD9000FFFF0401AA287201FFFF0401AA28720103
:10CDA000FFFF04010A247201FFFF0401BBF210011E
:10CDB000FFFF0401BBF21901FFFF0401BBF21001E8
:10CDC000FFFF04010A287201FFFF04010A28720113
:10CDD000FFFF04010A287201FFFF04010A28720103
:10CDE000FFFF04010A287201FFFF04010A287201F3
:10CDF000FFFF04010A287201FFFF04010A287201E3
:10CE0000FFFF0401AA287201FFFF0401AA28720192
:10CE1000FFFF0401AA287201FFFF0401AA28720182
:10CE2000FFFF0401FE00FF01FFFF0401BBF2100140
:10CE3000FFFF0401BBF21901FFFF0401BBF2100167
:10CE4000FFFF04010A287201FFFF04010A28720192
:10CE5000FFFF04010A287201FFFF04010A28720182
:10CE6000FFFF04010A287201FFFF04010A28720172
:10CE7000FFFF04010A287201FFFF04010A28720162
:10CE8000FFFF0401AA287201FFFF0401AA28720112
:10CE9000FFFF0401AA287201FFFF0401AA28720102
:10CEA000FFFF0401FE00FF01FFFF0401BBF21001C0
:10CEB000FFFF0401BBF21901FFFF0401BBF21001E7
:10CEC000FFFF04010A287201FFFF04010A28720112
:10CED000FFFF04010A287201FFFF04010A28720102
:10CEE000FFFF04010A287201FFFF04010A287201F2
:10CEF000FFFF04010A287201FFFF04010A287201E2
:10CF0000FFFF0401AA287201FFFF0401AA28720191
:10CF1000FFFF0401AA287201FFFF0401AA28720181
:10CF2000FFFF04010A247201FFFF0401BBF210019C
:10CF3000FFFF0401BBF21901FFFF0401BBF2100166
:10CF4000FFFF04010A287201FFFF04010A28720191
:10CF5000FFFF04010A287201FFFF04010A28720181
:10CF6000FFFF04010A287201FFFF04010A28720171
:10CF7000FFFF04010A287201FFFF04010A28720161
:10CF8000FFFF0401AA287201FFFF0401AA28720111
:10CF9000FFFF0401AA287201FFFF0401AA28720101
:10CFA000FFFF04010A247201FFFF0401BBF210011C
:10CFB000FFFF0401BBF21901FFFF0401BBF21001E6
:10CFC000FFFF04010A287201FFFF04010A28720111
:10CFD000FFFF04010A287201FFFF04010A28720101
:10CFE000FFFF04010A287201FFFF04010A287201F1
:10CFF000FFFF04010A287201FFFF04010A287201E1
:10D00000FFFF0401AA287201FFFF0401AA28720190
:10D01000FFFF0401AA287201FFFF0401AA28720180
:10D02000FFFF0401FE00FF01FFFF0401BBF210013E
:10D03000FFFF0401BBF21901FFFF0401BBF2100165
:10D04000FFFF04010A287201FFFF04010A28720190
:10D05000FFFF04010A287201FFFF04010A28720180
:10D06000FFFF04010A287201FFFF04010A28720170
:10D07000FFFF04010A287201FFFF04010A28720160
:10D08000FFFF0401AA287201FFFF0401AA28720110
:10D09000FFFF0401AA287201FFFF0401AA28720100
:10D0A000FFFF0401FE00FF01FFFF0401BBF21001BE
:10D0B000FFFF0401BBF21901FFFF0401BBF21001E5
:10D0C000FFFF04010A287201FFFF04010A28720110
:10D0D000FFFF04010A287201FFFF04010A28720100
:10D0E000FFFF04010A287201FFFF04010A287201F0
:10D0F000FFFF04010A287201FFFF04010A287201E0
:10D10000FFFF0401AA287201FFFF0401AA2872018F
:10D11000FFFF0401AA287201FFFF0401AA2872017F
:10D12000FFFF04010A247201FFFF0401BBF210019A
:10D13000FFFF0401BBF21901FFFF0401BBF2100164
:10D14000FFFF04010A287201FFFF04010A2872018F
:10D15000FFFF04010A287201FFFF04010A2872017F
:10D16000FFFF04010A287201FFFF04010A2872016F
:10D17000FFFF04010A287201FFFF04010A2872015F
:10D18000FFFF0401AA287201FFFF0401AA2872010F
:10D19000FFFF0401AA287201FFFF0401AA287201FF
:10D1A000FFFF04010A247201FFFF0401BBF210011A
:10D1B000FFFF0401BBF21901FFFF0401BBF21001E4
:10D1C000FFFF04010A287201FFFF04010A2872010F
:10D1D000FFFF04010A287201FFFF04010A287201FF
:10D1E000FFFF04010A287201FFFF04010A287201EF
:10D1F000FFFF04010A287201FFFF04010A287201DF
:10D20000FFFF0401AA287201FFFF0401AA2872018E
:10D21000FFFF0401AA287201FFFF0401AA2872017E
:10D22000FFFF0401FE00FF01FFFF0401BBF210013C
:10D23000FFFF0401BBF21901FFFF0401BBF2100163
:10D24000FFFF04010A287201FFFF04010A2872018E
:10D25000FFFF04010A287201FFFF04010A2872017E
:10D26000FFFF04010A287201FFFF04010A2872016E
:10D27000FFFF04010A287201FFFF04010A2872015E
:10D28000FFFF0401AA287201FFFF0401AA2872010E
:10D29000FFFF0401AA287201FFFF0401AA287201FE
:10D2A000FFFF0401FE00FF01FFFF0401BBF21001BC
:10D2B000FFFF0401BBF21901FFFF0401BBF21001E3
:10D2C000FFFF04010A287201FFFF04010A2872010E
:10D2D000FFFF04010A287201FFFF04010A287201FE
:10D2E000FFFF04010A287201FFFF04010A287201EE
:10D2F000FFFF04010A287201FFFF04010A287201DE
:10D30000FFFF0401AA287201FFFF0401AA2872018D
:10D31000FFFF0401AA287201FFFF0401AA2872017D
:10D32000FFFF04010A247201FFFF0401BBF2100198
:10D33000FFFF0401BBF21901FFFF0401BBF2100162
:10D34000FFFF04010A287201FFFF04010A2872018D
:10D35000FFFF04010A287201FFFF04010A2872017D
:10D36000FFFF04010A287201FFFF04010A2872016D
:10D37000FFFF04010A287201FFFF04010A2872015D
:10D38000FFFF0401AA287201FFFF0401AA2872010D
:10D39000FFFF0401AA287201FFFF0401AA287201FD
:10D3A000FFFF04010A247201FFFF0401BBF2100118
:10D3B000FFFF0401BBF21901FFFF0401BBF21001E2
:10D3C000FFFF04010A287201FFFF04010A2872010D
:10D3D000FFFF04010A287201FFFF04010A287201FD
:10D3E000FFFF04010A287201FFFF04010A287201ED
:10D3F000FFFF04010A287201FFFF04010A287201DD
:10D40000FFFF0401AA287201FFFF0401AA2872018C
:10D41000FFFF0401AA287201FFFF0401AA2872017C
:10D42000FFFF0401FE00FF01FFFF0401BBF210013A
:10D43000FFFF0401BBF21901FFFF0401BBF2100161
:10D44000FFFF04010A287201FFFF04010A2872018C
:10D45000FFFF04010A287201FFFF04010A2872017C
:10D46000FFFF04010A287201FFFF04010A2872016C
:10D47000FFFF04010A287201FFFF04010A2872015C
:10D48000FFFF0401AA287201FFFF0401AA2872010C
:10D49000FFFF0401AA287201FFFF0401AA287201FC
:10D4A000FFFF0401FE00FF01FFFF0401BBF21001BA
:10D4B000FFFF0401BBF21901FFFF0401BBF21001E1
:10D4C000FFFF04010A287201FFFF04010A2872010C
:10D4D000FFFF04010A287201FFFF04010A287201FC
:10D4E000FFFF04010A287201FFFF04010A287201EC
:10D4F000FFFF04010A287201FFFF04010A287201DC
:10D50000FFFF0401AA287201FFFF0401AA2872018B
:10D51000FFFF0401AA287201FFFF0401AA2872017B
:10D52000FFFF04010A247201FFFF0401BBF2100196
:10D53000FFFF0401BBF21901FFFF0401BBF2100160
:10D54000FFFF04010A287201FFFF04010A2872018B
:10D55000FFFF04010A287201FFFF04010A2872017B
:10D56000FFFF04010A287201FFFF04010A2872016B
:10D57000FFFF04010A287201FFFF04010A2872015B
:10D58000FFFF0401AA287201FFFF0401AA2872010B
:10D59000FFFF0401AA287201FFFF0401AA287201FB
:10D5A000FFFF04010A247201FFFF0401BBF2100116
:10D5B000FFFF0401BBF21901FFFF0401BBF21001E0
:10D5C000FFFF04010A287201FFFF04010A2872010B
:10D5D000FFFF04010A287201FFFF04010A287201FB
:10D5E000FFFF04010A287201FFFF04010A287201EB
:10D5F000FFFF04010A287201FFFF04010A287201DB
:10D60000FFFF0401AA287201FFFF0401AA2872018A
:10D61000FFFF0401AA287201FFFF0401AA2872017A
:10D62000FFFF0401FE00FF01FFFF0401BBF2100138
:10D63000FFFF0401BBF21901FFFF0401BBF210015F
:10D64000FFFF04010A287201FFFF04010A2872018A
:10D65000FFFF04010A287201FFFF04010A2872017A
:10D66000FFFF04010A287201FFFF04010A2872016A
:10D67000FFFF04010A287201FFFF04010A2872015A
:10D68000FFFF0401AA287201FFFF0401AA2872010A
:10D69000FFFF0401AA287201FFFF0401AA287201FA
:10D6A000FFFF0401FE00FF01FFFF0401BBF21001B8
:10D6B000FFFF0401BBF21901FFFF0401BBF21001DF
:10D6C000FFFF04010A287201FFFF04010A2872010A
:10D6D000FFFF04010A287201FFFF04010A287201FA
:10D6E000FFFF04010A287201FFFF04010A287201EA
:10D6F000FFFF04010A287201FFFF04010A287201DA
:10D70000FFFF0401AA287201FFFF0401AA28720189
:10D71000FFFF0401AA287201FFFF0401AA28720179
:10D72000FFFF04010A247201FFFF0401BBF2100194
:10D73000FFFF0401BBF21901FFFF0401BBF210015E
:10D74000FFFF04010A287201FFFF04010A28720189
:10D75000FFFF04010A287201FFFF04010A28720179
:10D76000FFFF04010A287201FFFF04010A28720169
:10D77000FFFF04010A287201FFFF04010A28720159
:10D78000FFFF0401AA287201FFFF0401AA28720109
:10D79000FFFF0401AA287201FFFF0401AA287201F9
:10D7A000FFFF04010A247201FFFF0401BBF2100114
:10D7B000FFFF0401BBF21901FFFF0401BBF21001DE
:10D7C000FFFF04010A287201FFFF04010A28720109
:10D7D000FFFF04010A287201FFFF04010A287201F9
:10D7E000FFFF04010A287201FFFF04010A287201E9
:10D7F000FFFF04010A287201FFFF04010A287201D9
:10D80000FFFF0401AA287201FFFF0401AA28720188
:10D81000FFFF0401AA287201FFFF0401AA28720178
:10D82000FFFF0401FE00FF01FFFF0401BBF2100136
:10D83000FFFF0401BBF21901FFFF0401BBF210015D
:10D84000FFFF04010A287201FFFF04010A28720188
:10D85000FFFF04010A287201FFFF04010A28720178
:10D86000FFFF04010A287201FFFF04010A28720168
:10D87000FFFF04010A287201FFFF04010A28720158
:10D88000FFFF0401AA287201FFFF0401AA28720108
:10D89000FFFF0401AA287201FFFF0401AA287201F8
:10D8A000FFFF0401FE00FF01FFFF0401BBF21001B6
:10D8B000FFFF0401BBF21901FFFF0401BBF21001DD
:10D8C000FFFF04010A287201FFFF04010A28720108
:10D8D000FFFF04010A287201FFFF04010A287201F8
:10D8E000FFFF04010A287201FFFF04010A287201E8
:10D8F000FFFF04010A287201FFFF04010A287201D8
:10D90000FFFF0401AA287201FFFF0401AA28720187
:10D91000FFFF0401AA287201FFFF0401AA28720177
:10D92000FFFF04010A247201FFFF0401BBF2100192
:10D93000FFFF0401BBF21901FFFF0401BBF210015C
:10D94000FFFF04010A287201FFFF04010A28720187
:10D95000FFFF04010A287201FFFF04010A28720177
:10D96000FFFF04010A287201FFFF04010A28720167
:10D97000FFFF04010A287201FFFF04010A28720157
:10D98000FFFF0401AA287201FFFF0401AA28720107
:10D99000FFFF0401AA287201FFFF0401AA287201F7
:10D9A000FFFF04010A247201FFFF0401BBF2100112
:10D9B000FFFF0401BBF21901FFFF0401BBF21001DC
:10D9C000FFFF04010A287201FFFF04010A28720107
:10D9D000FFFF04010A287201FFFF04010A287201F7
:10D9E000FFFF04010A287201FFFF04010A287201E7
:10D9F000FFFF04010A287201FFFF04010A287201D7
:10DA0000FFFF0401AA287201FFFF0401AA28720186
:10DA1000FFFF0401AA287201FFFF0401AA28720176
:10DA2000FFFF0401FE00FF01FFFF0401BBF2100134
:10DA3000FFFF0401BBF21901FFFF0401BBF210015B
:10DA4000FFFF04010A287201FFFF04010A28720186
:10DA5000FFFF04010A287201FFFF04010A28720176
:10DA6000FFFF04010A287201FFFF04010A28720166
:10DA7000FFFF04010A287201FFFF04010A28720156
:10DA8000FFFF0401AA287201FFFF0401AA28720106
:10DA9000FFFF0401AA287201FFFF0401AA287201F6
:10DAA000FFFF0401FE00FF01FFFF0401BBF21001B4
:10DAB000FFFF0401BBF21901FFFF0401BBF21001DB
:10DAC000FFFF04010A287201FFFF04010A28720106
:10DAD000FFFF04010A287201FFFF04010A287201F6
:10DAE000FFFF04010A287201FFFF04010A287201E6
:10DAF000FFFF04010A287201FFFF04010A287201D6
:10DB0000FFFF0401AA287201FFFF0401AA28720185
:10DB1000FFFF0401AA287201FFFF0401AA28720175
:10DB2000FFFF04010A247201FFFF0401BBF2100190
:10DB3000FFFF0401BBF21901FFFF0401BBF210015A
:10DB4000FFFF04010A287201FFFF04010A28720185
:10DB5000FFFF04010A287201FFFF04010A28720175
:10DB6000FFFF04010A287201FFFF04010A28720165
:10DB7000FFFF04010A287201FFFF04010A28720155
:10DB8000FFFF0401AA287201FFFF0401AA28720105
:10DB9000FFFF0401AA287201FFFF0401AA287201F5
:10DBA000FFFF04010A247201FFFF0401BBF2100110
:10DBB000FFFF0401BBF21901FFFF0401BBF21001DA
:10DBC000FFFF04010A287201FFFF04010A28720105
:10DBD000FFFF04010A287201FFFF04010A287201F5
:10DBE000FFFF04010A287201FFFF04010A287201E5
:10DBF000FFFF04010A287201FFFF04010A287201D5
:10DC0000FFFF0401AA287201FFFF0401AA28720184
:10DC1000FFFF0401AA287201FFFF0401AA28720174
:10DC2000FFFF0401FE00FF01FFFF0401BBF2100132
:10DC3000FFFF0401BBF21901FFFF0401BBF2100159
:10DC4000FFFF04010A287201FFFF04010A28720184
:10DC5000FFFF04010A287201FFFF04010A28720174
:10DC6000FFFF04010A287201FFFF04010A28720164
:10DC7000FFFF04010A287201FFFF04010A28720154
:10DC8000FFFF0401AA287201FFFF0401AA28720104
:10DC9000FFFF0401AA287201FFFF0401AA287201F4
:10DCA000FFFF0401FE00FF01FFFF0401BBF21001B2
:10DCB000FFFF0401BBF21901FFFF0401BBF21001D9
:10DCC000FFFF04010A287201FFFF04010A28720104
:10DCD000FFFF04010A287201FFFF04010A287201F4
:10DCE000FFFF04010A287201FFFF04010A287201E4
:10DCF000FFFF04010A287201FFFF04010A287201D4
:10DD0000FFFF0401AA287201FFFF0401AA28720183
:10DD1000FFFF0401AA287201FFFF0401AA28720173
:10DD2000FFFF04010A247201FFFF0401BBF210018E
:10DD3000FFFF0401BBF21901FFFF0401BBF2100158
:10DD4000FFFF04010A287201FFFF04010A28720183
:10DD5000FFFF04010A287201FFFF04010A28720173
:10DD6000FFFF04010A287201FFFF04010A28720163
:10DD7000FFFF04010A287201FFFF04010A28720153
:10DD8000FFFF0401AA287201FFFF0401AA28720103
:10DD9000FFFF0401AA287201FFFF0401AA287201F3
:10DDA000FFFF04010A247201FFFF0401BBF210010E
:10DDB000FFFF0401BBF21901FFFF0401BBF21001D8
:10DDC000FFFF04010A287201FFFF04010A28720103
:10DDD000FFFF04010A287201FFFF04010A287201F3
:10DDE000FFFF04010A287201FFFF04010A287201E3
:10DDF000FFFF04010A287201FFFF04010A287201D3
:10DE0000FFFF0401AA287201FFFF0401AA28720182
:10DE1000FFFF0401AA287201FFFF0401AA28720172
:10DE2000FFFF0401FE00FF01FFFF0401BBF2100130
:10DE3000FFFF0401BBF21901FFFF0401BBF2100157
:10DE4000FFFF04010A287201FFFF04010A28720182
:10DE5000FFFF04010A287201FFFF04010A28720172
:10DE6000FFFF04010A287201FFFF04010A28720162
:10DE7000FFFF04010A287201FFFF04010A28720152
:10DE8000FFFF0401AA287201FFFF0401AA28720102
:10DE9000FFFF0401AA287201FFFF0401AA287201F2
:10DEA000FFFF0401FE00FF01FFFF0401BBF21001B0
:10DEB000FFFF0401BBF21901FFFF0401BBF21001D7
:10DEC000FFFF04010A287201FFFF04010A28720102
:10DED000FFFF04010A287201FFFF04010A287201F2
:10DEE000FFFF04010A287201FFFF04010A287201E2
:10DEF000FFFF04010A287201FFFF04010A287201D2
:10DF0000FFFF0401AA287201FFFF0401AA28720181
:10DF1000FFFF0401AA287201FFFF0401AA28720171
:10DF2000FFFF04010A247201FFFF0401BBF210018C
:10DF3000FFFF0401BBF21901FFFF0401BBF2100156
:10DF4000FFFF04010A287201FFFF04010A28720181
:10DF5000FFFF04010A287201FFFF04010A28720171
:10DF6000FFFF04010A287201FFFF04010A28720161
:10DF7000FFFF04010A287201FFFF04010A28720151
:10DF8000FFFF0401AA287201FFFF0401AA28720101
:10DF9000FFFF0401AA287201FFFF0401AA287201F1
:10DFA000FFFF04010A247201FFFF0401BBF210010C
:10DFB000FFFF0401BBF21901FFFF0401BBF21001D6
:10DFC000FFFF04010A287201FFFF04010A28720101
:10DFD000FFFF04010A287201FFFF04010A287201F1
:10DFE000FFFF04010A287201FFFF04010A287201E1
:10DFF000FFFF04010A287201FFFF04010A287201D1
:10E00000FFFF0401AA287201FFFF0401AA28720180
:10E01000FFFF0401AA287201FFFF0401AA28720170
:10E02000FFFF0401FE00FF01FFFF0401BBF210012E
:10E03000FFFF0401BBF21901FFFF0401BBF2100155
:10E04000FFFF04010A287201FFFF04010A28720180
:10E05000FFFF04010A287201FFFF04010A28720170
:10E06000FFFF04010A287201FFFF04010A28720160
:10E07000FFFF04010A287201FFFF04010A28720150
:10E08000FFFF0401AA287201FFFF0401AA28720100
:10E09000FFFF0401AA287201FFFF0401AA287201F0
:10E0A000FFFF0401FE00FF01FFFF0401BBF21001AE
:10E0B000FFFF0401BBF21901FFFF0401BBF21001D5
:10E0C000FFFF04010A287201FFFF04010A28720100
:10E0D000FFFF04010A287201FFFF04010A287201F0
:10E0E000FFFF04010A287201FFFF04010A287201E0
:10E0F000FFFF04010A287201FFFF04010A287201D0
:10E10000FFFF0401AA287201FFFF0401AA2872017F
:10E11000FFFF0401AA287201FFFF0401AA2872016F
:10E12000FFFF04010A247201FFFF0401BBF210018A
:10E13000FFFF0401BBF21901FFFF0401BBF2100154
:10E14000FFFF04010A287201FFFF04010A2872017F
:10E15000FFFF04010A287201FFFF04010A2872016F
:10E16000FFFF04010A287201FFFF04010A2872015F
:10E17000FFFF04010A287201FFFF04010A2872014F
:10E18000FFFF0401AA287201FFFF0401AA287201FF
:10E19000FFFF0401AA287201FFFF0401AA287201EF
:10E1A000FFFF04010A247201FFFF0401BBF210010A
:10E1B000FFFF0401BBF21901FFFF0401BBF21001D4
:10E1C000FFFF04010A287201FFFF04010A287201FF
:10E1D000FFFF04010A287201FFFF04010A287201EF
:10E1E000FFFF04010A287201FFFF04010A287201DF
:10E1F000FFFF04010A287201FFFF04010A287201CF
:10E20000FFFF0401AA287201FFFF0401AA2872017E
:10E21000FFFF0401AA287201FFFF0401AA2872016E
:10E22000FFFF0401FE00FF01FFFF0401BBF210012C
:10E23000FFFF0401BBF21901FFFF0401BBF2100153
:10E24000FFFF04010A287201FFFF04010A2872017E
:10E25000FFFF04010A287201FFFF04010A2872016E
:10E26000FFFF04010A287201FFFF04010A2872015E
:10E27000FFFF04010A287201FFFF04010A2872014E
:10E28000FFFF0401AA287201FFFF0401AA287201FE
:10E29000FFFF0401AA287201FFFF0401AA287201EE
:10E2A000FFFF0401FE00FF01FFFF0401BBF21001AC
:10E2B000FFFF0401BBF21901FFFF0401BBF21001D3
:10E2C000FFFF04010A287201FFFF04010A287201FE
:10E2D000FFFF04010A287201FFFF04010A287201EE
:10E2E000FFFF04010A287201FFFF04010A287201DE
:10E2F000FFFF04010A287201FFFF04010A287201CE
:10E30000FFFF0401AA287201FFFF0401AA2872017D
:10E31000FFFF0401AA287201FFFF0401AA2872016D
:10E32000FFFF04010A247201FFFF0401BBF2100188
:10E33000FFFF0401BBF21901FFFF0401BBF2100152
:10E34000FFFF04010A287201FFFF04010A2872017D
:10E35000FFFF04010A287201FFFF04010A2872016D
:10E36000FFFF04010A287201FFFF04010A2872015D
:10E37000FFFF04010A287201FFFF04010A2872014D
:10E38000FFFF0401AA287201FFFF0401AA287201FD
:10E39000FFFF0401AA287201FFFF0401AA287201ED
:10E3A000FFFF04010A247201FFFF0401BBF2100108
:10E3B000FFFF0401BBF21901FFFF0401BBF21001D2
:10E3C000FFFF04010A287201FFFF04010A287201FD
:10E3D000FFFF04010A287201FFFF04010A287201ED
:10E3E000FFFF04010A287201FFFF04010A287201DD
:10E3F000FFFF04010A287201FFFF04010A287201CD
:10E40000FFFF0401AA287201FFFF0401AA2872017C
:10E41000FFFF0401AA287201FFFF0401AA2872016C
:10E42000FFFF0401FE00FF01FFFF0401BBF210012A
:10E43000FFFF0401BBF21901FFFF0401BBF2100151
:10E44000FFFF04010A287201FFFF04010A2872017C
:10E45000FFFF04010A287201FFFF04010A2872016C
:10E46000FFFF04010A287201FFFF04010A2872015C
:10E47000FFFF04010A287201FFFF04010A2872014C
:10E48000FFFF0401AA287201FFFF0401AA287201FC
:10E49000FFFF0401AA287201FFFF0401AA287201EC
:10E4A000FFFF0401FE00FF01FFFF0401BBF21001AA
:10E4B000FFFF0401BBF21901FFFF0401BBF21001D1
:10E4C000FFFF04010A287201FFFF04010A287201FC
:10E4D000FFFF04010A287201FFFF04010A287201EC
:10E4E000FFFF04010A287201FFFF04010A287201DC
:10E4F000FFFF04010A287201FFFF04010A287201CC
:10E50000FFFF0401AA287201FFFF0401AA2872017B
:10E51000FFFF0401AA287201FFFF0401AA2872016B
:10E52000FFFF04010A247201FFFF0401BBF2100186
:10E53000FFFF0401BBF21901FFFF0401BBF2100150
:10E54000FFFF04010A287201FFFF04010A2872017B
:10E55000FFFF04010A287201FFFF04010A2872016B
:10E56000FFFF04010A287201FFFF04010A2872015B
:10E57000FFFF04010A287201FFFF04010A2872014B
:10E58000FFFF0401AA287201FFFF0401AA287201FB
:10E59000FFFF0401AA287201FFFF0401AA287201EB
:10E5A000FFFF04010A247201FFFF0401BBF2100106
:10E5B000FFFF0401BBF21901FFFF0401BBF21001D0
:10E5C000FFFF04010A287201FFFF04010A287201FB
:10E5D000FFFF04010A287201FFFF04010A287201EB
:10E5E000FFFF04010A287201FFFF04010A287201DB
:10E5F000FFFF04010A287201FFFF04010A287201CB
:10E60000FFFF0401AA287201FFFF0401AA2872017A
:10E61000FFFF0401AA287201FFFF0401AA2872016A
:10E62000FFFF0401FE00FF01FFFF0401BBF2100128
:10E63000FFFF0401BBF21901FFFF0401BBF210014F
:10E64000FFFF04010A287201FFFF04010A2872017A
:10E65000FFFF04010A287201FFFF04010A2872016A
:10E66000FFFF04010A287201FFFF04010A2872015A
:10E67000FFFF04010A287201FFFF04010A2872014A
:10E68000FFFF0401AA287201FFFF0401AA287201FA
:10E69000FFFF0401AA287201FFFF0401AA287201EA
:10E6A000FFFF0401FE00FF01FFFF0401BBF21001A8
:10E6B000FFFF0401BBF21901FFFF0401BBF21001CF
:10E6C000FFFF04010A287201FFFF04010A287201FA
:10E6D000FFFF04010A287201FFFF04010A287201EA
:10E6E000FFFF04010A287201FFFF04010A287201DA
:10E6F000FFFF04010A287201FFFF04010A287201CA
:10E70000FFFF0401AA287201FFFF0401AA28720179
:10E71000FFFF0401AA287201FFFF0401AA28720169
:10E72000FFFF04010A247201FFFF0401BBF2100184
:10E73000FFFF0401BBF21901FFFF0401BBF210014E
:10E74000FFFF04010A287201FFFF04010A28720179
:10E75000FFFF04010A287201FFFF04010A28720169
:10E76000FFFF04010A287201FFFF04010A28720159
:10E77000FFFF04010A287201FFFF04010A28720149
:10E78000FFFF0401AA287201FFFF0401AA287201F9
:10E79000FFFF0401AA287201FFFF0401AA287201E9
:10E7A000FFFF04010A247201FFFF0401BBF2100104
:10E7B000FFFF0401BBF21901FFFF0401BBF21001CE
:10E7C000FFFF04010A287201FFFF04010A287201F9
:10E7D000FFFF04010A287201FFFF04010A287201E9
:10E7E000FFFF04010A287201FFFF04010A287201D9
:10E7F000FFFF04010A287201FFFF04010A287201C9
:10E80000FFFF0401AA287201FFFF0401AA28720178
:10E81000FFFF0401AA287201FFFF0401AA28720168
:10E82000FFFF0401FE00FF01FFFF0401BBF2100126
:10E83000FFFF0401BBF21901FFFF0401BBF210014D
:10E84000FFFF04010A287201FFFF04010A28720178
:10E85000FFFF04010A287201FFFF04010A28720168
:10E86000FFFF04010A287201FFFF04010A28720158
:10E87000FFFF04010A287201FFFF04010A28720148
:10E88000FFFF0401AA287201FFFF0401AA287201F8
:10E89000FFFF0401AA287201FFFF0401AA287201E8
:10E8A000FFFF0401FE00FF01FFFF0401BBF21001A6
:10E8B000FFFF0401BBF21901FFFF0401BBF21001CD
:10E8C000FFFF04010A287201FFFF04010A287201F8
:10E8D000FFFF04010A287201FFFF04010A287201E8
:10E8E000FFFF04010A287201FFFF04010A287201D8
:10E8F000FFFF04010A287201FFFF04010A287201C8
:10E90000FFFF0401AA287201FFFF0401AA28720177
:10E91000FFFF0401AA287201FFFF0401AA28720167
:10E92000FFFF04010A247201FFFF0401BBF2100182
:10E93000FFFF0401BBF21901FFFF0401BBF210014C
:10E94000FFFF04010A287201FFFF04010A28720177
:10E95000FFFF04010A287201FFFF04010A28720167
:10E96000FFFF04010A287201FFFF04010A28720157
:10E97000FFFF04010A287201FFFF04010A28720147
:10E98000FFFF0401AA287201FFFF0401AA287201F7
:10E99000FFFF0401AA287201FFFF0401AA287201E7
:10E9A000FFFF04010A247201FFFF0401BBF2100102
:10E9B000FFFF0401BBF21901FFFF0401BBF21001CC
:10E9C000FFFF04010A287201FFFF04010A287201F7
:10E9D000FFFF04010A287201FFFF04010A287201E7
:10E9E000FFFF04010A287201FFFF04010A287201D7
:10E9F000FFFF04010A287201FFFF04010A287201C7
:10EA0000FFFF0401AA287201FFFF0401AA28720176
:10EA1000FFFF0401AA287201FFFF0401AA28720166
:10EA2000FFFF0401FE00FF01FFFF0401BBF2100124
:10EA3000FFFF0401BBF21901FFFF0401BBF210014B
:10EA4000FFFF04010A287201FFFF04010A28720176
:10EA5000FFFF04010A287201FFFF04010A28720166
:10EA6000FFFF04010A287201FFFF04010A28720156
:10EA7000FFFF04010A287201FFFF04010A28720146
:10EA8000FFFF0401AA287201FFFF0401AA287201F6
:10EA9000FFFF0401AA287201FFFF0401AA287201E6
:10EAA000FFFF0401FE00FF01FFFF0401BBF21001A4
:10EAB000FFFF0401BBF21901FFFF0401BBF21001CB
:10EAC000FFFF04010A287201FFFF04010A287201F6
:10EAD000FFFF04010A287201FFFF04010A287201E6
:10EAE000FFFF04010A287201FFFF04010A287201D6
:10EAF000FFFF04010A287201FFFF04010A287201C6
:10EB0000FFFF0401AA287201FFFF0401AA28720175
:10EB1000FFFF0401AA287201FFFF0401AA28720165
:10EB2000FFFF04010A247201FFFF0401BBF2100180
:10EB3000FFFF0401BBF21901FFFF0401BBF210014A
:10EB4000FFFF04010A287201FFFF04010A28720175
:10EB5000FFFF04010A287201FFFF04010A28720165
:10EB6000FFFF04010A287201FFFF04010A28720155
:10EB7000FFFF04010A287201FFFF04010A28720145
:10EB8000FFFF0401AA287201FFFF0401AA287201F5
:10EB9000FFFF0401AA287201FFFF0401AA287201E5
:10EBA000FFFF04010A247201FFFF0401BBF2100100
:10EBB000FFFF0401BBF21901FFFF0401BBF21001CA
:10EBC000FFFF04010A287201FFFF04010A287201F5
:10EBD000FFFF04010A287201FFFF04010A287201E5
:10EBE000FFFF04010A287201FFFF04010A287201D5
:10EBF000FFFF04010A287201FFFF04010A287201C5
:10EC0000FFFF0401AA287201FFFF0401AA28720174
:10EC1000FFFF0401AA287201FFFF0401AA28720164
:10EC2000FFFF0401FE00FF01FFFF0401BBF2100122
:10EC3000FFFF0401BBF21901FFFF0401BBF2100149
:10EC4000FFFF04010A287201FFFF04010A28720174
:10EC5000FFFF04010A287201FFFF04010A28720164
:10EC6000FFFF04010A287201FFFF04010A28720154
:10EC7000FFFF04010A287201FFFF04010A28720144
:10EC8000FFFF0401AA287201FFFF0401AA287201F4
:10EC9000FFFF0401AA287201FFFF0401AA287201E4
:10ECA000FFFF0401FE00FF01FFFF0401BBF21001A2
:10ECB000FFFF0401BBF21901FFFF0401BBF21001C9
:10ECC000FFFF04010A287201FFFF04010A287201F4
:10ECD000FFFF04010A287201FFFF04010A287201E4
:10ECE000FFFF04010A287201FFFF04010A287201D4
:10ECF000FFFF04010A287201FFFF04010A287201C4
:10ED0000FFFF0401AA287201FFFF0401AA28720173
:10ED1000FFFF0401AA287201FFFF0401AA28720163
:10ED2000FFFF04010A247201FFFF0401BBF210017E
:10ED3000FFFF0401BBF21901FFFF0401BBF2100148
:10ED4000FFFF04010A287201FFFF04010A28720173
:10ED5000FFFF04010A287201FFFF04010A28720163
:10ED6000FFFF04010A287201FFFF04010A28720153
:10ED7000FFFF04010A287201FFFF04010A28720143
:10ED8000FFFF0401AA287201FFFF0401AA287201F3
:10ED9000FFFF0401AA287201FFFF0401AA287201E3
:10EDA000FFFF04010A247201FFFF0401BBF21001FE
:10EDB000FFFF0401BBF21901FFFF0401BBF21001C8
:10EDC000FFFF04010A287201FFFF04010A287201F3
:10EDD000FFFF04010A287201FFFF04010A287201E3
:10EDE000FFFF04010A287201FFFF04010A287201D3
:10EDF000FFFF04010A287201FFFF04010A287201C3
:10EE0000FFFF0401AA287201FFFF0401AA28720172
:10EE1000FFFF0401AA287201FFFF0401AA28720162
:10EE2000FFFF0401FE00FF01FFFF0401BBF2100120
:10EE3000FFFF0401BBF21901FFFF0401BBF2100147
:10EE4000FFFF04010A287201FFFF04010A28720172
:10EE5000FFFF04010A287201FFFF04010A28720162
:10EE6000FFFF04010A287201FFFF04010A28720152
:10EE7000FFFF04010A287201FFFF04010A28720142
:10EE8000FFFF0401AA287201FFFF0401AA287201F2
:10EE9000FFFF0401AA287201FFFF0401AA287201E2
:10EEA000FFFF0401FE00FF01FFFF0401BBF21001A0
:10EEB000FFFF0401BBF21901FFFF0401BBF21001C7
:10EEC000FFFF04010A287201FFFF04010A287201F2
:10EED000FFFF04010A287201FFFF04010A287201E2
:10EEE000FFFF04010A287201FFFF04010A287201D2
:10EEF000FFFF04010A287201FFFF04010A287201C2
:10EF0000FFFF0401AA287201FFFF0401AA28720171
:10EF1000FFFF0401AA287201FFFF0401AA28720161
:10EF2000FFFF04010A247201FFFF0401BBF210017C
:10EF3000FFFF0401BBF21901FFFF0401BBF2100146
:10EF4000FFFF04010A287201FFFF04010A28720171
:10EF5000FFFF04010A287201FFFF04010A28720161
:10EF6000FFFF04010A287201FFFF04010A28720151
:10EF7000FFFF04010A287201FFFF04010A28720141
:10EF8000FFFF0401AA287201FFFF0401AA287201F1
:10EF9000FFFF0401AA287201FFFF0401AA287201E1
:10EFA000FFFF04010A247201FFFF0401BBF21001FC
:10EFB000FFFF0401BBF21901FFFF0401BBF21001C6
:10EFC000FFFF04010A287201FFFF04010A287201F1
:10EFD000FFFF04010A287201FFFF04010A287201E1
:10EFE000FFFF04010A287201FFFF04010A287201D1
:10EFF000FFFF04010A287201FFFF04010A287201C1
:10F00000FFFF0401AA287201FFFF0401AA28720170
:10F01000FFFF0401AA287201FFFF0401AA28720160
:10F02000FFFF0401FE00FF01FFFF0401BBF210011E
:10F03000FFFF0401BBF21901FFFF0401BBF2100145
:10F04000FFFF04010A287201FFFF04010A28720170
:10F05000FFFF04010A287201FFFF04010A28720160
:10F06000FFFF04010A287201FFFF04010A28720150
:10F07000FFFF04010A287201FFFF04010A28720140
:10F08000FFFF0401AA287201FFFF0401AA287201F0
:10F09000FFFF0401AA287201FFFF0401AA287201E0
:10F0A000FFFF0401FE00FF01FFFF0401BBF210019E
:10F0B000FFFF0401BBF21901FFFF0401BBF21001C5
:10F0C000FFFF04010A287201FFFF04010A287201F0
:10F0D000FFFF04010A287201FFFF04010A287201E0
:10F0E000FFFF04010A287201FFFF04010A287201D0
:10F0F000FFFF04010A287201FFFF04010A287201C0
:10F10000FFFF0401AA287201FFFF0401AA2872016F
:10F11000FFFF0401AA287201FFFF0401AA2872015F
:10F12000FFFF04010A247201FFFF0401BBF210017A
:10F13000FFFF0401BBF21901FFFF0401BBF2100144
:10F14000FFFF04010A287201FFFF04010A2872016F
:10F15000FFFF04010A287201FFFF04010A2872015F
:10F16000FFFF04010A287201FFFF04010A2872014F
:10F17000FFFF04010A287201FFFF04010A2872013F
:10F18000FFFF0401AA287201FFFF0401AA287201EF
:10F19000FFFF0401AA287201FFFF0401AA287201DF
:10F1A000FFFF04010A247201FFFF0401BBF21001FA
:10F1B000FFFF0401BBF21901FFFF0401BBF21001C4
:10F1C000FFFF04010A287201FFFF04010A287201EF
:10F1D000FFFF04010A287201FFFF04010A287201DF
:10F1E000FFFF04010A287201FFFF04010A287201CF
:10F1F000FFFF04010A287201FFFF04010A287201BF
:10F20000FFFF0401AA287201FFFF0401AA2872016E
:10F21000FFFF0401AA287201FFFF0401AA2872015E
:10F22000FFFF0401FE00FF01FFFF0401BBF210011C
:10F23000FFFF0401BBF21901FFFF0401BBF2100143
:10F24000FFFF04010A287201FFFF04010A2872016E
:10F25000FFFF04010A287201FFFF04010A2872015E
:10F26000FFFF04010A287201FFFF04010A2872014E
:10F27000FFFF04010A287201FFFF04010A2872013E
:10F28000FFFF0401AA287201FFFF0401AA287201EE
:10F29000FFFF0401AA287201FFFF0401AA287201DE
:10F2A000FFFF0401FE00FF01FFFF0401BBF210019C
:10F2B000FFFF0401BBF21901FFFF0401BBF21001C3
:10F2C000FFFF04010A287201FFFF04010A287201EE
:10F2D000FFFF04010A287201FFFF04010A287201DE
:10F2E000FFFF04010A287201FFFF04010A287201CE
:10F2F000FFFF04010A287201FFFF04010A287201BE
:10F30000FFFF0401AA287201FFFF0401AA2872016D
:10F31000FFFF0401AA287201FFFF0401AA2872015D
:10F32000FFFF04010A247201FFFF0401BBF2100178
:10F33000FFFF0401BBF21901FFFF0401BBF2100142
:10F34000FFFF04010A287201FFFF04010A2872016D
:10F35000FFFF04010A287201FFFF04010A2872015D
:10F36000FFFF04010A287201FFFF04010A2872014D
:10F37000FFFF04010A287201FFFF04010A2872013D
:10F38000FFFF0401AA287201FFFF0401AA287201ED
:10F39000FFFF0401AA287201FFFF0401AA287201DD
:10F3A000FFFF04010A247201FFFF0401BBF21001F8
:10F3B000FFFF0401BBF21901FFFF0401BBF21001C2
:10F3C000FFFF04010A287201FFFF04010A287201ED
:10F3D000FFFF04010A287201FFFF04010A287201DD
:10F3E000FFFF04010A287201FFFF04010A287201CD
:10F3F000FFFF04010A287201FFFF04010A287201BD
:10F40000FFFF0401AA287201FFFF0401AA2872016C
:10F41000FFFF0401AA287201FFFF0401AA2872015C
:10F42000FFFF0401FE00FF01FFFF0401BBF210011A
:10F43000FFFF0401BBF21901FFFF0401BBF2100141
:10F44000FFFF04010A287201FFFF04010A2872016C
:10F45000FFFF04010A287201FFFF04010A2872015C
:10F46000FFFF04010A287201FFFF04010A2872014C
:10F47000FFFF04010A287201FFFF04010A2872013C
:10F48000FFFF0401AA287201FFFF0401AA287201EC
:10F49000FFFF0401AA287201FFFF0401AA287201DC
:10F4A000FFFF0401FE00FF01FFFF0401BBF210019A
:10F4B000FFFF0401BBF21901FFFF0401BBF21001C1
:10F4C000FFFF04010A287201FFFF04010A287201EC
:10F4D000FFFF04010A287201FFFF04010A287201DC
:10F4E000FFFF04010A287201FFFF04010A287201CC
:10F4F000FFFF04010A287201FFFF04010A287201BC
:10F50000FFFF0401AA287201FFFF0401AA2872016B
:10F51000FFFF0401AA287201FFFF0401AA2872015B
:10F52000FFFF04010A247201FFFF0401BBF2100176
:10F53000FFFF0401BBF21901FFFF0401BBF2100140
:10F54000FFFF04010A287201FFFF04010A2872016B
:10F55000FFFF04010A287201FFFF04010A2872015B
:10F56000FFFF04010A287201FFFF04010A2872014B
:10F57000FFFF04010A287201FFFF04010A2872013B
:10F58000FFFF0401AA287201FFFF0401AA287201EB
:10F59000FFFF0401AA287201FFFF0401AA287201DB
:10F5A000FFFF04010A247201FFFF0401BBF21001F6
:10F5B000FFFF0401BBF21901FFFF0401BBF21001C0
:10F5C000FFFF04010A287201FFFF04010A287201EB
:10F5D000FFFF04010A287201FFFF04010A287201DB
:10F5E000FFFF04010A287201FFFF04010A287201CB
:10F5F000FFFF04010A287201FFFF04010A287201BB
:10F60000FFFF0401AA287201FFFF0401AA2872016A
:10F61000FFFF0401AA287201FFFF0401AA2872015A
:10F62000FFFF0401FE00FF01FFFF0401BBF2100118
:10F63000FFFF0401BBF21901FFFF0401BBF210013F
:10F64000FFFF04010A287201FFFF04010A2872016A
:10F65000FFFF04010A287201FFFF04010A2872015A
:10F66000FFFF04010A287201FFFF04010A2872014A
:10F67000FFFF04010A287201FFFF04010A2872013A
:10F68000FFFF0401AA287201FFFF0401AA287201EA
:10F69000FFFF0401AA287201FFFF0401AA287201DA
:10F6A000FFFF0401FE00FF01FFFF0401BBF2100198
:10F6B000FFFF0401BBF21901FFFF0401BBF21001BF
:10F6C000FFFF04010A287201FFFF04010A287201EA
:10F6D000FFFF04010A287201FFFF04010A287201DA
:10F6E000FFFF04010A287201FFFF04010A287201CA
:10F6F000FFFF04010A287201FFFF04010A287201BA
:10F70000FFFF0401AA287201FFFF0401AA28720169
:10F71000FFFF0401AA287201FFFF0401AA28720159
:10F72000FFFF04010A247201FFFF0401BBF2100174
:10F73000FFFF0401BBF21901FFFF0401BBF210013E
:10F74000FFFF04010A287201FFFF04010A28720169
:10F75000FFFF04010A287201FFFF04010A28720159
:10F76000FFFF04010A287201FFFF04010A28720149
:10F77000FFFF04010A287201FFFF04010A28720139
:10F78000FFFF0401AA287201FFFF0401AA287201E9
:10F79000FFFF0401AA287201FFFF0401AA287201D9
:10F7A000FFFF04010A247201FFFF0401BBF21001F4
:10F7B000FFFF0401BBF21901FFFF0401BBF21001BE
:10F7C000FFFF04010A287201FFFF04010A287201E9
:10F7D000FFFF04010A287201FFFF04010A287201D9
:10F7E000FFFF04010A287201FFFF04010A287201C9
:10F7F000FFFF04010A287201FFFF04010A287201B9
:10F80000FFFF0401AA287201FFFF0401AA28720168
:10F81000FFFF0401AA287201FFFF0401AA28720158
:10F82000FFFF0401FE00FF01FFFF0401BBF2100116
:10F83000FFFF0401BBF21901FFFF0401BBF210013D
:10F84000FFFF04010A287201FFFF04010A28720168
:10F85000FFFF04010A287201FFFF04010A28720158
:10F86000FFFF04010A287201FFFF04010A28720148
:10F87000FFFF04010A287201FFFF04010A28720138
:10F88000FFFF0401AA287201FFFF0401AA287201E8
:10F89000FFFF0401AA287201FFFF0401AA287201D8
:10F8A000FFFF0401FE00FF01FFFF0401BBF2100196
:10F8B000FFFF0401BBF21901FFFF0401BBF21001BD
:10F8C000FFFF04010A287201FFFF04010A287201E8
:10F8D000FFFF04010A287201FFFF04010A287201D8
:10F8E000FFFF04010A287201FFFF04010A287201C8
:10F8F000FFFF04010A287201FFFF04010A287201B8
:10F90000FFFF0401AA287201FFFF0401AA28720167
:10F91000FFFF0401AA287201FFFF0401AA28720157
:10F92000FFFF04010A247201FFFF0401BBF2100172
:10F93000FFFF0401BBF21901FFFF0401BBF210013C
:10F94000FFFF04010A287201FFFF04010A28720167
:10F95000FFFF04010A287201FFFF04010A28720157
:10F96000FFFF04010A287201FFFF04010A28720147
:10F97000FFFF04010A287201FFFF04010A28720137
:10F98000FFFF0401AA287201FFFF0401AA287201E7
:10F99000FFFF0401AA287201FFFF0401AA287201D7
:10F9A000FFFF04010A247201FFFF0401BBF21001F2
:10F9B000FFFF0401BBF21901FFFF0401BBF21001BC
:10F9C000FFFF04010A287201FFFF04010A287201E7
:10F9D000FFFF04010A287201FFFF04010A287201D7
:10F9E000FFFF04010A287201FFFF04010A287201C7
:10F9F000FFFF04010A287201FFFF04010A287201B7
:10FA0000FFFF0401AA287201FFFF0401AA28720166
:10FA1000FFFF0401AA287201FFFF0401AA28720156
:10FA2000FFFF0401FE00FF01FFFF0401BBF2100114
:10FA3000FFFF0401BBF21901FFFF0401BBF210013B
:10FA4000FFFF04010A287201FFFF04010A28720166
:10FA5000FFFF04010A287201FFFF04010A28720156
:10FA6000FFFF04010A287201FFFF04010A28720146
:10FA7000FFFF04010A287201FFFF04010A28720136
:10FA8000FFFF0401AA287201FFFF0401AA287201E6
:10FA9000FFFF0401AA287201FFFF0401AA287201D6
:10FAA000FFFF0401FE00FF01FFFF0401BBF2100194
:10FAB000FFFF0401BBF21901FFFF0401BBF21001BB
:10FAC000FFFF04010A287201FFFF04010A287201E6
:10FAD000FFFF04010A287201FFFF04010A287201D6
:10FAE000FFFF04010A287201FFFF04010A287201C6
:10FAF000FFFF04010A287201FFFF04010A287201B6
:10FB0000FFFF0401AA287201FFFF0401AA28720165
:10FB1000FFFF0401AA287201FFFF0401AA28720155
:10FB2000FFFF04010A247201FFFF0401BBF2100170
:10FB3000FFFF0401BBF21901FFFF0401BBF210013A
:10FB4000FFFF04010A287201FFFF04010A28720165
:10FB5000FFFF04010A287201FFFF04010A28720155
:10FB6000FFFF04010A287201FFFF04010A28720145
:10FB7000FFFF04010A287201FFFF04010A28720135
:10FB8000FFFF0401AA287201FFFF0401AA287201E5
:10FB9000FFFF0401AA287201FFFF0401AA287201D5
:10FBA000FFFF04010A247201FFFF0401BBF21001F0
:10FBB000FFFF0401BBF21901FFFF0401BBF21001BA
:10FBC000FFFF04010A287201FFFF04010A287201E5
:10FBD000FFFF04010A287201FFFF04010A287201D5
:10FBE000FFFF04010A287201FFFF04010A287201C5
:10FBF000FFFF04010A287201FFFF04010A287201B5
:10FC0000FFFF0401AA287201FFFF0401AA28720164
:10FC1000FFFF0401AA287201FFFF0401AA28720154
:10FC2000FFFF0401FE00FF01FFFF0401BBF2100112
:10FC3000FFFF0401BBF21901FFFF0401BBF2100139
:10FC4000FFFF04010A287201FFFF04010A28720164
:10FC5000FFFF04010A287201FFFF04010A28720154
:10FC6000FFFF04010A287201FFFF04010A28720144
:10FC7000FFFF04010A287201FFFF04010A28720134
:10FC8000FFFF0401AA287201FFFF0401AA287201E4
:10FC9000FFFF0401AA287201FFFF0401AA287201D4
:10FCA000FFFF0401FE00FF01FFFF0401BBF2100192
:10FCB000FFFF0401BBF21901FFFF0401BBF21001B9
:10FCC000FFFF04010A287201FFFF04010A287201E4
:10FCD000FFFF04010A287201FFFF04010A287201D4
:10FCE000FFFF04010A287201FFFF04010A287201C4
:10FCF000FFFF04010A287201FFFF04010A287201B4
:10FD0000FFFF0401AA287201FFFF0401AA28720163
:10FD1000FFFF0401AA287201FFFF0401AA28720153
:10FD2000FFFF04010A247201FFFF0401BBF210016E
:10FD3000FFFF0401BBF21901FFFF0401BBF2100138
:10FD4000FFFF04010A287201FFFF04010A28720163
:10FD5000FFFF04010A287201FFFF04010A28720153
:10FD6000FFFF04010A287201FFFF04010A28720143
:10FD7000FFFF04010A287201FFFF04010A28720133
:10FD8000FFFF0401AA287201FFFF0401AA287201E3
:10FD9000FFFF0401AA287201FFFF0401AA287201D3
:10FDA000FFFF04010A247201FFFF0401BBF21001EE
:10FDB000FFFF0401BBF21901FFFF0401BBF21001B8
:10FDC000FFFF04010A287201FFFF04010A287201E3
:10FDD000FFFF04010A287201FFFF04010A287201D3
:10FDE000FFFF04010A287201FFFF04010A287201C3
:10FDF000FFFF04010A287201FFFF04010A287201B3
:10FE0000FFFF0401AA287201FFFF0401AA28720162
:10FE1000FFFF0401AA287201FFFF0401AA28720152
:10FE2000FFFF0401FE00FF01FFFF0401BBF2100110
:10FE3000FFFF0401BBF21901FFFF0401BBF2100137
:10FE4000FFFF04010A287201FFFF04010A28720162
:10FE5000FFFF04010A287201FFFF04010A28720152
:10FE6000FFFF04010A287201FFFF04010A28720142
:10FE7000FFFF04010A287201FFFF04010A28720132
:10FE8000FFFF0401AA287201FFFF0401AA287201E2
:10FE9000FFFF0401AA287201FFFF0401AA287201D2
:10FEA000FFFF0401FE00FF01FFFF0401BBF2100190
:10FEB000FFFF0401BBF21901FFFF0401BBF21001B7
:10FEC000FFFF04010A287201FFFF04010A287201E2
:10FED000FFFF04010A287201FFFF04010A287201D2
:10FEE000FFFF04010A287201FFFF04010A287201C2
:10FEF000FFFF04010A287201FFFF04010A287201B2
:10FF0000FFFF0401AA287201FFFF0401AA28720161
:10FF1000FFFF0401AA287201FFFF0401AA28720151
:10FF2000FFFF04010A247201FFFF0401BBF210016C
:10FF3000FFFF0401BBF21901FFFF0401BBF2100136
:10FF4000FFFF04010A287201FFFF04010A28720161
:10FF5000FFFF04010A287201FFFF04010A28720151
:10FF6000FFFF04010A287201FFFF04010A28720141
:10FF7000FFFF04010A287201FFFF04010A28720131
:10FF8000FFFF0401AA287201FFFF0401AA287201E1
:10FF9000FFFF0401AA287201FFFF0401AA287201D1
:10FFA000FFFF04010A247201FFFF0401BBF21001EC
:10FFB000FFFF0401BBF21901FFFF0401BBF21001B6
:10FFC000FFFF04010A287201FFFF04010A287201E1
:10FFD000FFFF04010A287201FFFF04010A287201D1
:10FFE000FFFF04010A287201FFFF04010A287201C1
:10FFF000FFFF04010A287201FFFF04010A287201B1
:020000040001F9
:10000000FFFF0401AA287201FFFF0401AA28720160
:10001000FFFF0401AA287201FFFF0401AA28720150
:10002000FFFF0401FE00FF01FFFF0401BBF210010E
:10003000FFFF0401BBF21901FFFF0401BBF2100135
:10004000FFFF04010A287201FFFF04010A28720160
:10005000FFFF04010A287201FFFF04010A28720150
:10006000FFFF04010A287201FFFF04010A28720140
:10007000FFFF04010A287201FFFF04010A28720130
:10008000FFFF0401AA287201FFFF0401AA287201E0
:10009000FFFF0401AA287201FFFF0401AA287201D0
:1000A000FFFF0401FE00FF01FFFF0401BBF210018E
:1000B000FFFF0401BBF21901FFFF0401BBF21001B5
:1000C000FFFF04010A287201FFFF04010A287201E0
:1000D000FFFF04010A287201FFFF04010A287201D0
:1000E000FFFF04010A287201FFFF04010A287201C0
:1000F000FFFF04010A287201FFFF04010A287201B0
:10010000FFFF0401AA287201FFFF0401AA2872015F
:10011000FFFF0401AA287201FFFF0401AA2872014F
:10012000FFFF0401094A1B01FFFF0401BBF210019C
:10013000FFFF0401BBF21901FFFF0401BBF2100134
:10014000FFFF04010A287201FFFF04010A2872015F
:10015000FFFF04010A287201FFFF04010A2872014F
:10016000FFFF04010A287201FFFF04010A2872013F
:10017000FFFF04010A287201FFFF04010A2872012F
:10018000FFFF0401AA287201FFFF0401AA287201DF
:10019000FFFF0401AA287201FFFF0401AA287201CF
:1001A000FFFF0401094A1B01FFFF0401BBF210011C
:1001B000FFFF0401BBF21901FFFF0401BBF21001B4
:1001C000FFFF04010A287201FFFF04010A287201DF
:1001D000FFFF04010A287201FFFF04010A287201CF
:1001E000FFFF04010A287201FFFF04010A287201BF
:1001F000FFFF04010A287201FFFF04010A287201AF
:10020000FFFF0401AA287201FFFF0401AA2872015E
:10021000FFFF0401AA287201FFFF0401AA2872014E
:10022000FFFF0401FE00FF01FFFF0401BBF210010C
:10023000FFFF0401BBF21901FFFF0401BBF2100133
:10024000FFFF04010A287201FFFF04010A2872015E
:10025000FFFF04010A287201FFFF04010A2872014E
:10026000FFFF04010A287201FFFF04010A2872013E
:10027000FFFF04010A287201FFFF04010A2872012E
:10028000FFFF0401AA287201FFFF0401AA287201DE
:10029000FFFF0401AA287201FFFF0401AA287201CE
:1002A000FFFF0401FE00FF01FFFF0401BBF210018C
:1002B000FFFF0401BBF21901FFFF0401BBF21001B3
:1002C000FFFF04010A287201FFFF04010A287201DE
:1002D000FFFF04010A287201FFFF04010A287201CE
:1002E000FFFF04010A287201FFFF04010A287201BE
:1002F000FFFF04010A287201FFFF04010A287201AE
:10030000FFFF0401AA287201FFFF0401AA2872015D
:10031000FFFF0401AA287201FFFF0401AA2872014D
:10032000FFFF0401094A1B01FFFF0401BBF210019A
:10033000FFFF0401BBF21901FFFF0401BBF2100132
:10034000FFFF04010A287201FFFF04010A2872015D
:10035000FFFF04010A287201FFFF04010A2872014D
:10036000FFFF04010A287201FFFF04010A2872013D
:10037000FFFF04010A287201FFFF04010A2872012D
:10038000FFFF0401AA287201FFFF0401AA287201DD
:10039000FFFF0401AA287201FFFF0401AA287201CD
:1003A000FFFF0401094A1B01FFFF0401BBF210011A
:1003B000FFFF0401BBF21901FFFF0401BBF21001B2
:1003C000FFFF04010A287201FFFF04010A287201DD
:1003D000FFFF04010A287201FFFF04010A287201CD
:1003E000FFFF04010A287201FFFF04010A287201BD
:1003F000FFFF04010A287201FFFF04010A287201AD
:10040000FFFF0401AA287201FFFF0401AA2872015C
:10041000FFFF0401AA287201FFFF0401AA2872014C
:10042000FFFF0401FE00FF01FFFF0401BBF210010A
:10043000FFFF0401BBF21901FFFF0401BBF2100131
:10044000FFFF04010A287201FFFF04010A2872015C
:10045000FFFF04010A287201FFFF04010A2872014C
:10046000FFFF04010A287201FFFF04010A2872013C
:10047000FFFF04010A287201FFFF04010A2872012C
:10048000FFFF0401AA287201FFFF0401AA287201DC
:10049000FFFF0401AA287201FFFF0401AA287201CC
:1004A000FFFF0401FE00FF01FFFF0401BBF210018A
:1004B000FFFF0401BBF21901FFFF0401BBF21001B1
:1004C000FFFF04010A287201FFFF04010A287201DC
:1004D000FFFF04010A287201FFFF04010A287201CC
:1004E000FFFF04010A287201FFFF04010A287201BC
:1004F000FFFF04010A287201FFFF04010A287201AC
:10050000FFFF0401AA287201FFFF0401AA2872015B
:10051000FFFF0401AA287201FFFF0401AA2872014B
:10052000FFFF0401094A1B01FFFF0401BBF2100198
:10053000FFFF0401BBF21901FFFF0401BBF2100130
:10054000FFFF04010A287201FFFF04010A2872015B
:10055000FFFF04010A287201FFFF04010A2872014B
:10056000FFFF04010A287201FFFF04010A2872013B
:10057000FFFF04010A287201FFFF04010A2872012B
:10058000FFFF0401AA287201FFFF0401AA287201DB
:10059000FFFF0401AA287201FFFF0401AA287201CB
:1005A000FFFF0401094A1B01FFFF0401BBF2100118
:1005B000FFFF0401BBF21901FFFF0401BBF21001B0
:1005C000FFFF04010A287201FFFF04010A287201DB
:1005D000FFFF04010A287201FFFF04010A287201CB
:1005E000FFFF04010A287201FFFF04010A287201BB
:1005F000FFFF04010A287201FFFF04010A287201AB
:10060000FFFF0401AA287201FFFF0401AA2872015A
:10061000FFFF0401AA287201FFFF0401AA2872014A
:10062000FFFF0401FE00FF01FFFF0401BBF2100108
:10063000FFFF0401BBF21901FFFF0401BBF210012F
:10064000FFFF04010A287201FFFF04010A2872015A
:10065000FFFF04010A287201FFFF04010A2872014A
:10066000FFFF04010A287201FFFF04010A2872013A
:10067000FFFF04010A287201FFFF04010A2872012A
:10068000FFFF0401AA287201FFFF0401AA287201DA
:10069000FFFF0401AA287201FFFF0401AA287201CA
:1006A000FFFF0401FE00FF01FFFF0401BBF2100188
:1006B000FFFF0401BBF21901FFFF0401BBF21001AF
:1006C000FFFF04010A287201FFFF04010A287201DA
:1006D000FFFF04010A287201FFFF04010A287201CA
:1006E000FFFF04010A287201FFFF04010A287201BA
:1006F000FFFF04010A287201FFFF04010A287201AA
:10070000FFFF0401AA287201FFFF0401AA28720159
:10071000FFFF0401AA287201FFFF0401AA28720149
:10072000FFFF0401094A1B01FFFF0401BBF2100196
:10073000FFFF0401BBF21901FFFF0401BBF210012E
:10074000FFFF04010A287201FFFF04010A28720159
:10075000FFFF04010A287201FFFF04010A28720149
:10076000FFFF04010A287201FFFF04010A28720139
:10077000FFFF04010A287201FFFF04010A28720129
:10078000FFFF0401AA287201FFFF0401AA287201D9
:10079000FFFF0401AA287201FFFF0401AA287201C9
:1007A000FFFF0401094A1B01FFFF0401BBF2100116
:1007B000FFFF0401BBF21901FFFF0401BBF21001AE
:1007C000FFFF04010A287201FFFF04010A287201D9
:1007D000FFFF04010A287201FFFF04010A287201C9
:1007E000FFFF04010A287201FFFF04010A287201B9
:1007F000FFFF04010A287201FFFF04010A287201A9
:10080000FFFF0401AA287201FFFF0401AA28720158
:10081000FFFF0401AA287201FFFF0401AA28720148
:10082000FFFF0401FE00FF01FFFF0401BBF2100106
:10083000FFFF0401BBF21901FFFF0401BBF210012D
:10084000FFFF04010A287201FFFF04010A28720158
:10085000FFFF04010A287201FFFF04010A28720148
:10086000FFFF04010A287201FFFF04010A28720138
:10087000FFFF04010A287201FFFF04010A28720128
:10088000FFFF0401AA287201FFFF0401AA287201D8
:10089000FFFF0401AA287201FFFF0401AA287201C8
:1008A000FFFF0401FE00FF01FFFF0401BBF2100186
:1008B000FFFF0401BBF21901FFFF0401BBF21001AD
:1008C000FFFF04010A287201FFFF04010A287201D8
:1008D000FFFF04010A287201FFFF04010A287201C8
:1008E000FFFF04010A287201FFFF04010A287201B8
:1008F000FFFF04010A287201FFFF04010A287201A8
:10090000FFFF0401AA287201FFFF0401AA28720157
:10091000FFFF0401AA287201FFFF0401AA28720147
:10092000FFFF0401094A1B01FFFF0401BBF2100194
:10093000FFFF0401BBF21901FFFF0401BBF210012C
:10094000FFFF04010A287201FFFF04010A28720157
:10095000FFFF04010A287201FFFF04010A28720147
:10096000FFFF04010A287201FFFF04010A28720137
:10097000FFFF04010A287201FFFF04010A28720127
:10098000FFFF0401AA287201FFFF0401AA287201D7
:10099000FFFF0401AA287201FFFF0401AA287201C7
:1009A000FFFF0401094A1B01FFFF0401BBF2100114
:1009B000FFFF0401BBF21901FFFF0401BBF21001AC
:1009C000FFFF04010A287201FFFF04010A287201D7
:1009D000FFFF04010A287201FFFF04010A287201C7
:1009E000FFFF04010A287201FFFF04010A287201B7
:1009F000FFFF04010A287201FFFF04010A287201A7
:100A0000FFFF0401AA287201FFFF0401AA28720156
:100A1000FFFF0401AA287201FFFF0401AA28720146
:100A2000FFFF0401FE00FF01FFFF0401BBF2100104
:100A3000FFFF0401BBF21901FFFF0401BBF210012B
:100A4000FFFF04010A287201FFFF04010A28720156
:100A5000FFFF04010A287201FFFF04010A28720146
:100A6000FFFF04010A287201FFFF04010A28720136
:100A7000FFFF04010A287201FFFF04010A28720126
:100A8000FFFF0401AA287201FFFF0401AA287201D6
:100A9000FFFF0401AA287201FFFF0401AA287201C6
:100AA000FFFF0401FE00FF01FFFF0401BBF2100184
:100AB000FFFF0401BBF21901FFFF0401BBF21001AB
:100AC000FFFF04010A287201FFFF04010A287201D6
:100AD000FFFF04010A287201FFFF04010A287201C6
:100AE000FFFF04010A287201FFFF04010A287201B6
:100AF000FFFF04010A287201FFFF04010A287201A6
:100B0000FFFF0401AA287201FFFF0401AA28720155
:100B1000FFFF0401AA287201FFFF0401AA28720145
:100B2000FFFF0401094A1B01FFFF0401BBF2100192
:100B3000FFFF0401BBF21901FFFF0401BBF210012A
:100B4000FFFF04010A287201FFFF04010A28720155
:100B5000FFFF04010A287201FFFF04010A28720145
:100B6000FFFF04010A287201FFFF04010A28720135
:100B7000FFFF04010A287201FFFF04010A28720125
:100B8000FFFF0401AA287201FFFF0401AA287201D5
:100B9000FFFF0401AA287201FFFF0401AA287201C5
:100BA000FFFF0401094A1B01FFFF0401BBF2100112
:100BB000FFFF0401BBF21901FFFF0401BBF21001AA
:100BC000FFFF04010A287201FFFF04010A287201D5
:100BD000FFFF04010A287201FFFF04010A287201C5
:100BE000FFFF04010A287201FFFF04010A287201B5
:100BF000FFFF04010A287201FFFF04010A287201A5
:100C0000FFFF0401AA287201FFFF0401AA28720154
:100C1000FFFF0401AA287201FFFF0401AA28720144
:100C2000FFFF0401FE00FF01FFFF0401BBF2100102
:100C3000FFFF0401BBF21901FFFF0401BBF2100129
:100C4000FFFF04010A287201FFFF04010A28720154
:100C5000FFFF04010A287201FFFF04010A28720144
:100C6000FFFF04010A287201FFFF04010A28720134
:100C7000FFFF04010A287201FFFF04010A28720124
:100C8000FFFF0401AA287201FFFF0401AA287201D4
:100C9000FFFF0401AA287201FFFF0401AA287201C4
:100CA000FFFF0401FE00FF01FFFF0401BBF2100182
:100CB000FFFF0401BBF21901FFFF0401BBF21001A9
:100CC000FFFF04010A287201FFFF04010A287201D4
:100CD000FFFF04010A287201FFFF04010A287201C4
:100CE000FFFF04010A287201FFFF04010A287201B4
:100CF000FFFF04010A287201FFFF04010A287201A4
:100D0000FFFF0401AA287201FFFF0401AA28720153
:100D1000FFFF0401AA287201FFFF0401AA28720143
:100D2000FFFF0401094A1B01FFFF0401BBF2100190
:100D3000FFFF0401BBF21901FFFF0401BBF2100128
:100D4000FFFF04010A287201FFFF04010A28720153
:100D5000FFFF04010A287201FFFF04010A28720143
:100D6000FFFF04010A287201FFFF04010A28720133
:100D7000FFFF04010A287201FFFF04010A28720123
:100D8000FFFF0401AA287201FFFF0401AA287201D3
:100D9000FFFF0401AA287201FFFF0401AA287201C3
:100DA000FFFF0401094A1B01FFFF0401BBF2100110
:100DB000FFFF0401BBF21901FFFF0401BBF21001A8
:100DC000FFFF04010A287201FFFF04010A287201D3
:100DD000FFFF04010A287201FFFF04010A287201C3
:100DE000FFFF04010A287201FFFF04010A287201B3
:100DF000FFFF04010A287201FFFF04010A287201A3
:100E0000FFFF0401AA287201FFFF0401AA28720152
:100E1000FFFF0401AA287201FFFF0401AA28720142
:100E2000FFFF0401FE00FF01FFFF0401BBF2100100
:100E3000FFFF0401BBF21901FFFF0401BBF2100127
:100E4000FFFF04010A287201FFFF04010A28720152
:100E5000FFFF04010A287201FFFF04010A28720142
:100E6000FFFF04010A287201FFFF04010A28720132
:100E7000FFFF04010A287201FFFF04010A28720122
:100E8000FFFF0401AA287201FFFF0401AA287201D2
:100E9000FFFF0401AA287201FFFF0401AA287201C2
:100EA000FFFF0401FE00FF01FFFF0401BBF2100180
:100EB000FFFF0401BBF21901FFFF0401BBF21001A7
:100EC000FFFF04010A287201FFFF04010A287201D2
:100ED000FFFF04010A287201FFFF04010A287201C2
:100EE000FFFF04010A287201FFFF04010A287201B2
:100EF000FFFF04010A287201FFFF04010A287201A2
:100F0000FFFF0401AA287201FFFF0401AA28720151
:100F1000FFFF0401AA287201FFFF0401AA28720141
:100F2000FFFF0401094A1B01FFFF0401BBF210018E
:100F3000FFFF0401BBF21901FFFF0401BBF2100126
:100F4000FFFF04010A287201FFFF04010A28720151
:100F5000FFFF04010A287201FFFF04010A28720141
:100F6000FFFF04010A287201FFFF04010A28720131
:100F7000FFFF04010A287201FFFF04010A28720121
:100F8000FFFF0401AA287201FFFF0401AA287201D1
:100F9000FFFF0401AA287201FFFF0401AA287201C1
:100FA000FFFF0401094A1B01FFFF0401BBF210010E
:100FB000FFFF0401BBF21901FFFF0401BBF21001A6
:100FC000FFFF04010A287201FFFF04010A287201D1
:100FD000FFFF04010A287201FFFF04010A287201C1
:100FE000FFFF04010A287201FFFF04010A287201B1
:100FF000FFFF04010A287201FFFF04010A287201A1
:10100000FFFF0401AA287201FFFF0401AA28720150
:10101000FFFF0401AA287201FFFF0401AA28720140
:10102000FFFF0401FE00FF01FFFF0401BBF21001FE
:10103000FFFF0401BBF21901FFFF0401BBF2100125
:10104000FFFF04010A287201FFFF04010A28720150
:10105000FFFF04010A287201FFFF04010A28720140
:10106000FFFF04010A287201FFFF04010A28720130
:10107000FFFF04010A287201FFFF04010A28720120
:10108000FFFF0401AA287201FFFF0401AA287201D0
:10109000FFFF0401AA287201FFFF0401AA287201C0
:1010A000FFFF0401FE00FF01FFFF0401BBF210017E
:1010B000FFFF0401BBF21901FFFF0401BBF21001A5
:1010C000FFFF04010A287201FFFF04010A287201D0
:1010D000FFFF04010A287201FFFF04010A287201C0
:1010E000FFFF04010A287201FFFF04010A287201B0
:1010F000FFFF04010A287201FFFF04010A287201A0
:10110000FFFF0401AA287201FFFF0401AA2872014F
:10111000FFFF0401AA287201FFFF0401AA2872013F
:10112000FFFF0401094A1B01FFFF0401BBF210018C
:10113000FFFF0401BBF21901FFFF0401BBF2100124
:10114000FFFF04010A287201FFFF04010A2872014F
:10115000FFFF04010A287201FFFF04010A2872013F
:10116000FFFF04010A287201FFFF04010A2872012F
:10117000FFFF04010A287201FFFF04010A2872011F
:10118000FFFF0401AA287201FFFF0401AA287201CF
:10119000FFFF0401AA287201FFFF0401AA287201BF
:1011A000FFFF0401094A1B01FFFF0401BBF210010C
:1011B000FFFF0401BBF21901FFFF0401BBF21001A4
:1011C000FFFF04010A287201FFFF04010A287201CF
:1011D000FFFF04010A287201FFFF04010A287201BF
:1011E000FFFF04010A287201FFFF04010A287201AF
:1011F000FFFF04010A287201FFFF04010A2872019F
:10120000FFFF0401AA287201FFFF0401AA2872014E
:10121000FFFF0401AA287201FFFF0401AA2872013E
:10122000FFFF0401FE00FF01FFFF0401BBF21001FC
:10123000FFFF0401BBF21901FFFF0401BBF2100123
:10124000FFFF04010A287201FFFF04010A2872014E
:10125000FFFF04010A287201FFFF04010A2872013E
:10126000FFFF04010A287201FFFF04010A2872012E
:10127000FFFF04010A287201FFFF04010A2872011E
:10128000FFFF0401AA287201FFFF0401AA287201CE
:10129000FFFF0401AA287201FFFF0401AA287201BE
:1012A000FFFF0401FE00FF01FFFF0401BBF210017C
:1012B000FFFF0401BBF21901FFFF0401BBF21001A3
:1012C000FFFF04010A287201FFFF04010A287201CE
:1012D000FFFF04010A287201FFFF04010A287201BE
:1012E000FFFF04010A287201FFFF04010A287201AE
:1012F000FFFF04010A287201FFFF04010A2872019E
:10130000FFFF0401AA287201FFFF0401AA2872014D
:10131000FFFF0401AA287201FFFF0401AA2872013D
:10132000FFFF0401094A1B01FFFF0401BBF210018A
:10133000FFFF0401BBF21901FFFF0401BBF2100122
:10134000FFFF04010A287201FFFF04010A2872014D
:10135000FFFF04010A287201FFFF04010A2872013D
:10136000FFFF04010A287201FFFF04010A2872012D
:10137000FFFF04010A287201FFFF04010A2872011D
:10138000FFFF0401AA287201FFFF0401AA287201CD
:10139000FFFF0401AA287201FFFF0401AA287201BD
:1013A000FFFF0401094A1B01FFFF0401BBF210010A
:1013B000FFFF0401BBF21901FFFF0401BBF21001A2
:1013C000FFFF04010A287201FFFF04010A287201CD
:1013D000FFFF04010A287201FFFF04010A287201BD
:1013E000FFFF04010A287201FFFF04010A287201AD
:1013F000FFFF04010A287201FFFF04010A2872019D
:10140000FFFF0401AA287201FFFF0401AA2872014C
:10141000FFFF0401AA287201FFFF0401AA2872013C
:10142000FFFF0401FE00FF01FFFF0401BBF21001FA
:10143000FFFF0401BBF21901FFFF0401BBF2100121
:10144000FFFF04010A287201FFFF04010A2872014C
:10145000FFFF04010A287201FFFF04010A2872013C
:10146000FFFF04010A287201FFFF04010A2872012C
:10147000FFFF04010A287201FFFF04010A2872011C
:10148000FFFF0401AA287201FFFF0401AA287201CC
:10149000FFFF0401AA287201FFFF0401AA287201BC
:1014A000FFFF0401FE00FF01FFFF0401BBF210017A
:1014B000FFFF0401BBF21901FFFF0401BBF21001A1
:1014C000FFFF04010A287201FFFF04010A287201CC
:1014D000FFFF04010A287201FFFF04010A287201BC
:1014E000FFFF04010A287201FFFF04010A287201AC
:1014F000FFFF04010A287201FFFF04010A2872019C
:10150000FFFF0401AA287201FFFF0401AA2872014B
:10151000FFFF0401AA287201FFFF0401AA2872013B
:10152000FFFF0401094A1B01FFFF0401BBF2100188
:10153000FFFF0401BBF21901FFFF0401BBF2100120
:10154000FFFF04010A287201FFFF04010A2872014B
:10155000FFFF04010A287201FFFF04010A2872013B
:10156000FFFF04010A287201FFFF04010A2872012B
:10157000FFFF04010A287201FFFF04010A2872011B
:10158000FFFF0401AA287201FFFF0401AA287201CB
:10159000FFFF0401AA287201FFFF0401AA287201BB
:1015A000FFFF0401094A1B01FFFF0401BBF2100108
:1015B000FFFF0401BBF21901FFFF0401BBF21001A0
:1015C000FFFF04010A287201FFFF04010A287201CB
:1015D000FFFF04010A287201FFFF04010A287201BB
:1015E000FFFF04010A287201FFFF04010A287201AB
:1015F000FFFF04010A287201FFFF04010A2872019B
:10160000FFFF0401AA287201FFFF0401AA2872014A
:10161000FFFF0401AA287201FFFF0401AA2872013A
:10162000FFFF0401FE00FF01FFFF0401BBF21001F8
:10163000FFFF0401BBF21901FFFF0401BBF210011F
:10164000FFFF04010A287201FFFF04010A2872014A
:10165000FFFF04010A287201FFFF04010A2872013A
:10166000FFFF04010A287201FFFF04010A2872012A
:10167000FFFF04010A287201FFFF04010A2872011A
:10168000FFFF0401AA287201FFFF0401AA287201CA
:10169000FFFF0401AA287201FFFF0401AA287201BA
:1016A000FFFF0401FE00FF01FFFF0401BBF2100178
:1016B000FFFF0401BBF21901FFFF0401BBF210019F
:1016C000FFFF04010A287201FFFF04010A287201CA
:1016D000FFFF04010A287201FFFF04010A287201BA
:1016E000FFFF04010A287201FFFF04010A287201AA
:1016F000FFFF04010A287201FFFF04010A2872019A
:10170000FFFF0401AA287201FFFF0401AA28720149
:10171000FFFF0401AA287201FFFF0401AA28720139
:10172000FFFF0401094A1B01FFFF0401BBF2100186
:10173000FFFF0401BBF21901FFFF0401BBF210011E
:10174000FFFF04010A287201FFFF04010A28720149
:10175000FFFF04010A287201FFFF04010A28720139
:10176000FFFF04010A287201FFFF04010A28720129
:10177000FFFF04010A287201FFFF04010A28720119
:10178000FFFF0401AA287201FFFF0401AA287201C9
:10179000FFFF0401AA287201FFFF0401AA287201B9
:1017A000FFFF0401094A1B01FFFF0401BBF2100106
:1017B000FFFF0401BBF21901FFFF0401BBF210019E
:1017C000FFFF04010A287201FFFF04010A287201C9
:1017D000FFFF04010A287201FFFF04010A287201B9
:1017E000FFFF04010A287201FFFF04010A287201A9
:1017F000FFFF04010A287201FFFF04010A28720199
:10180000FFFF0401AA287201FFFF0401AA28720148
:10181000FFFF0401AA287201FFFF0401AA28720138
:10182000FFFF0401FE00FF01FFFF0401BBF21001F6
:10183000FFFF0401BBF21901FFFF0401BBF210011D
:10184000FFFF04010A287201FFFF04010A28720148
:10185000FFFF04010A287201FFFF04010A28720138
:10186000FFFF04010A287201FFFF04010A28720128
:10187000FFFF04010A287201FFFF04010A28720118
:10188000FFFF0401AA287201FFFF0401AA287201C8
:10189000FFFF0401AA287201FFFF0401AA287201B8
:1018A000FFFF0401FE00FF01FFFF0401BBF2100176
:1018B000FFFF0401BBF21901FFFF0401BBF210019D
:1018C000FFFF04010A287201FFFF04010A287201C8
:1018D000FFFF04010A287201FFFF04010A287201B8
:1018E000FFFF04010A287201FFFF04010A287201A8
:1018F000FFFF04010A287201FFFF04010A28720198
:10190000FFFF0401AA287201FFFF0401AA28720147
:10191000FFFF0401AA287201FFFF0401AA28720137
:10192000FFFF0401094A1B01FFFF0401BBF2100184
:10193000FFFF0401BBF21901FFFF0401BBF210011C
:10194000FFFF04010A287201FFFF04010A28720147
:10195000FFFF04010A287201FFFF04010A28720137
:10196000FFFF04010A287201FFFF04010A28720127
:10197000FFFF04010A287201FFFF04010A28720117
:10198000FFFF0401AA287201FFFF0401AA287201C7
:10199000FFFF0401AA287201FFFF0401AA287201B7
:1019A000FFFF0401094A1B01FFFF0401BBF2100104
:1019B000FFFF0401BBF21901FFFF0401BBF210019C
:1019C000FFFF04010A287201FFFF04010A287201C7
:1019D000FFFF04010A287201FFFF04010A287201B7
:1019E000FFFF04010A287201FFFF04010A287201A7
:1019F000FFFF04010A287201FFFF04010A28720197
:101A0000FFFF0401AA287201FFFF0401AA28720146
:101A1000FFFF0401AA287201FFFF0401AA28720136
:101A2000FFFF0401FE00FF01FFFF0401BBF21001F4
:101A3000FFFF0401BBF21901FFFF0401BBF210011B
:101A4000FFFF04010A287201FFFF04010A28720146
:101A5000FFFF04010A287201FFFF04010A28720136
:101A6000FFFF04010A287201FFFF04010A28720126
:101A7000FFFF04010A287201FFFF04010A28720116
:101A8000FFFF0401AA287201FFFF0401AA287201C6
:101A9000FFFF0401AA287201FFFF0401AA287201B6
:101AA000FFFF0401FE00FF01FFFF0401BBF2100174
:101AB000FFFF0401BBF21901FFFF0401BBF210019B
:101AC000FFFF04010A287201FFFF04010A287201C6
:101AD000FFFF04010A287201FFFF04010A287201B6
:101AE000FFFF04010A287201FFFF04010A287201A6
:101AF000FFFF04010A287201FFFF04010A28720196
:101B0000FFFF0401AA287201FFFF0401AA28720145
:101B1000FFFF0401AA287201FFFF0401AA28720135
:101B2000FFFF0401094A1B01FFFF0401BBF2100182
:101B3000FFFF0401BBF21901FFFF0401BBF210011A
:101B4000FFFF04010A287201FFFF04010A28720145
:101B5000FFFF04010A287201FFFF04010A28720135
:101B6000FFFF04010A287201FFFF04010A28720125
:101B7000FFFF04010A287201FFFF04010A28720115
:101B8000FFFF0401AA287201FFFF0401AA287201C5
:101B9000FFFF0401AA287201FFFF0401AA287201B5
:101BA000FFFF0401094A1B01FFFF0401BBF2100102
:101BB000FFFF0401BBF21901FFFF0401BBF210019A
:101BC000FFFF04010A287201FFFF04010A287201C5
:101BD000FFFF04010A287201FFFF04010A287201B5
:101BE000FFFF04010A287201FFFF04010A287201A5
:101BF000FFFF04010A287201FFFF04010A28720195
